:020000040800F2
:100000000000022079E90508C19C0008DD600208B3
:1000100029EA050829EA050829EA05080000000080
:1000200000000000000000000000000085B1000892
:1000300087B100080000000089B10008ED16010832
:1000400029EA050829EA050829EA050829EA050830
:1000500029EA050829EA05088FFE000893FE000832
:1000600029EA050897FE00089BFE000869A300081E
:100070007DA3000891A30008A5A30008B9A3000868
:10008000CDA30008E1A3000829EA0508000000004C
:100090000000000000000000000000009FFE0008BB
:1000A000A1A20008C9A20008F1A200088BA20008C2
:1000B00019A300082DA3000841A3000829EA050898
:1000C00029EA050829EA050829EA050829EA0508B0
:1000D00029EA0508DD9D0008E99D000800000000F0
:1000E000A3FE000829EA05088BB100080000000003
:1000F000000000000000000000000000F5A3000860
:100100000000000029EA050855A3000829EA0508AF
:1001100000000000000000000000000000000000DF
:1001200009A400081DA4000831A4000845A4000883
:1001300059A40008000000000000000000000000BA
:10014000000000000000000000000000D5B1000821
:100150006DA4000881A4000895A4000829EA0508F8
:1001600029EA050829EA050800000000000000004F
:10017000000000000000000000000000000000007F
:100180000000000029EA050800000000000000004F
:0801900029EA050829EA050827
:0801980024DA0500010000005B
:1001A000946301200201000002001400B4630120E6
:1001B0000202000002001400D4630120020A0000C1
:1001C00002001400F4630120020600000200140083
:1001D00014640120020700000200140034640120AE
:1001E000020300000400140054640120020800000F
:1001F0000400140074640120010B0000000077006B
:1002000094640120010C000000007600B464012019
:100210000110000000007600D4640120010D0100EF
:1002200000007700F4640120011200000000760055
:10023000146501200114000000001E003465012037
:10024000011A000000000D0054650120011B000090
:1002500000000E0074650120011C000000001E005B
:10026000946501200117000000000C00B465012016
:100270000118000000000E00D465012001280100D3
:1002800000001800F4650120012000000000480073
:10029000146601200121000000004900346601209D
:1002A0000122000000004A005466012001230000E2
:1002B00000004B00746601200124000000004C0087
:1002C000946601200125000000004D00B466012065
:1002D0000126000000004E00D46601200127000026
:1002E00000004F00F4660120012B000000002900EF
:1002F00014670120012C010000002900346701204F
:10030000012D01000000700054670120012F000042
:100310000000310074670120012E0100000052002E
:10032000946701200130010000002800B46701201B
:100330000131010000002800D467012002350400CB
:1003400000012C00F46701200134000000003C0093
:0C035000146801200137000000002000AC
:10800000D0E907239A423CBFC1685218D01A704782
:10801000D0E9092300699A4238BF1218D31A0138EF
:10802000C01A7047D0E90902131A584258417047E4
:10803000036A41690246C85CD16801338B4228BF9C
:10804000002313627047436A8269D154436A02690C
:108050000133934228BF0023426B4362D36843F04D
:108060008003D3607047436B188810F010001EBF68
:108070001A889B8801207047436B99891A88890662
:1080800010B592B2044607D5900605D5E26A2AB328
:108090009888216B80B29047636B99891A8809068A
:1080A00092B210D510060ED5D4E909128A4223D017
:1080B000A169895CC9B2998021690132B2FBF1F0F2
:1080C00001FB1022A262998A1A88C90592B204D5CE
:1080D000D20744BF4FF6F7721A8010BD9B88E26941
:1080E0006169DBB28B54E369E2680133B3FBF2F1FF
:1080F00002FB1133E361CFE7DA6822F08002DA6035
:10810000E1E7036941681F2B30B54FF0200285BFBE
:10811000A3F120054C680C68AA4098BF9A402242FF
:108120001DD0826900201074D0688468206820F017
:1081300001002060546820686579094C828934F810
:10814000154092B21F2B22EA0402828188BF203B95
:108150004FF020028BBF9A409A40CA608A6030BDBF
:10816000005A06080E4BDA68D20310D4DA68D1063A
:108170000FD4DA68D2050ED4DA6812F0E00F0CD111
:10818000DB6813F0020F0CBF0920082070470120A4
:10819000704706207047022070470720704700BFD5
:1081A000003C024007B509238DF80730FFF7DAFFDE
:1081B0008DF807009DF80730012BF7D09DF80700D8
:1081C00003B05DF804FB838A028B9BB243EA02434F
:1081D00099430CBF01200020704782B00023019317
:1081E0000093012300900193019B63B1009A21F059
:1081F0007F4314320092009A12681A4214BF012081
:10820000002002B07047009A1832F3E770477047B9
:10821000704701207047034BD3E90003C01AC0F335
:108220000A007047781A0020054AD2E900138B42F1
:10823000FDD0D1180133C3F30A03087A53607047A5
:10824000781A0020044BD3F8080820B1D3F80808A6
:10825000431F584258417047781A0020012380F884
:1082600049307047044BD3E90003C01AC0F30A0039
:10827000C0F50060704700BF781A002010B5D0F834
:10828000E83504461B699847032384F8123100201F
:1082900010BD08B590F8123180F81331042380F82E
:1082A0001231D0F8E835DB689847002008BD08B5E2
:1082B000D0F8E435DB6903B19847002008BD08B564
:1082C000D0F8E4351B6A9847002008BD08B5D0F8FF
:1082D000E4355B6A9847002008BD70B504460D463A
:1082E000164655F0C5FCC3B201335B0033802B70DA
:1082F00003236B70601E0223002410F8011F01B9D4
:1083000070BD5A1CD2B2E9540233AC54DBB2F4E76C
:1083100010B5074C2068FF2808D00649D1F80C2872
:1083200001F5016100F07CF8FF232360002010BDFF
:1083300000000020781A0020432301480B8070477A
:1083400004000020122301480B80704747000020E2
:10835000042301480B8070475900002010B5044CDD
:1083600004480A462146FFF7B8FF204610BD00BF6B
:1083700090220020F801070810B5044C04480A4672
:108380002146FFF7AAFF204610BD00BF9022002023
:108390000B02070810B5044C04480A462146FFF7B3
:1083A0009CFF204610BD00BF90220020100207084D
:1083B00010B5044C04480A462146FFF78EFF2046BC
:1083C00010BD00BF902200201A02070810B5044C0F
:1083D00004480A462146FFF780FF204610BD00BF33
:1083E00090220020250207087047704770477047A9
:1083F000704770477047054B00200522C3F80828D6
:10840000C3F81809C3F81C09704700BF781A002088
:10841000024B0020C3F80808704700BF781A0020FC
:10842000212838B50C461BD022282BD0202815D166
:10843000A1B1072A12D11A4DD5F81C3913B1096818
:10844000002098472368C5F82039237985F8243916
:10845000637985F82539A37985F82639002038BD58
:108460000029FBD0072AF9D10D4BD3F820290A6047
:1084700093F824290A7193F825294A7193F826392B
:108480008B71EBE70029E9D0022AE7D1044BD3F83E
:108490001839002BE2D0098800209847DEE700BF9A
:1084A000781A002030B50E4CD4E900329A1AC2F383
:1084B0000A020A44B2F5006F10D80144002281423A
:1084C00003D102B12360002030BDE21810F8015B37
:1084D00015720133C3F30A030122F0E70220F3E728
:1084E000781A0020034BD3F8280908B1036918470C
:1084F000704700BF781A0020034B93F850090038EA
:1085000018BF0120704700BF781A0020034B93F872
:108510005009032894BF002001207047781A0020DA
:1085200000487047CC230020837B042B0DD0074BE1
:10853000D3F898200132C3F8982042600422827355
:10854000D3F89C200132C3F89C207047A85E00201D
:10855000202301480B8070475D0000201223014852
:108560000B8070477D000020042301480B8070477A
:108570008F0000200A4608B5044920B90448FFF7D7
:10858000ACFE024808BD0348F9E700BFFC23002009
:10859000330207084B02070810B5044C04480A468A
:1085A0002146FFF79AFE204610BD00BFFC230020A5
:1085B0006302070810B5044C04480A462146FFF739
:1085C0008CFE204610BD00BFFC2300207602070869
:1085D00010B5044C04480A462146FFF77EFE2046AB
:1085E00010BD00BFFC23002081020708002370B5E6
:1085F0004D1C1E46040FB0F1204F34BF30343734C9
:1086000001F8134005F813600133DCB2A2424FEACF
:108610000010EFD870BD1A2310B50B80094BD3F8AA
:10862000E807D3F8EC2780180AD0D3F8EA470649C0
:108630000822FFF7DBFF042210312046FFF7D6FFA8
:10864000024810BD00F0FF1F95000020930000209D
:1086500008B5FFF747FF013840B208BD002070475A
:108660000020704770477047D0ED007AD0ED036A64
:1086700030EE677AE6EE877AB0EE670AC0ED007AF0
:10868000704790ED017AB5EE407AF1EE10FAF0EE17
:10869000407A09D19FED0E7A60EE870AF7EE006A04
:1086A00086EEA07A80ED017A90ED017A90ED000AD5
:1086B00080ED021A31EE077A77EEC07AC1EE076AD2
:1086C000A6EEA70AC0ED036A80ED000A704700BF5E
:1086D000DB0FC940D0ED056AD0ED017A90ED026A5A
:1086E000D0ED045AB0EE407A26EEA70AD0ED007A1B
:1086F00080ED057AA7EE870AD0ED067AC0ED066A0E
:10870000A6EE270AD0ED077A90ED036AA6EE670A77
:1087100090ED086AC0ED087AA5EEC60A80ED070A5A
:108720007047B0EE407AD0ED007A90ED050AD0EDBA
:10873000016AA7EE870AD0ED037A67EEC07AE6EE0B
:10874000877AD0ED066A76EEA77AD0ED026AC0EDA0
:10875000057AD0ED047A67EEC07AE6EE877AC0ED4E
:10876000067A704703685A1C0260197070472DE939
:10877000F04F89B083680793D0E90032029201324A
:1087800092FBF3F103FB11224260029ADFED967A2D
:1087900000EB820282ED200AB1EE400A82ED400A2F
:1087A00000F18006A3F1020E00F580700124B0EE06
:1087B000670A079AA24208DA30EE670AF6EE007AF4
:1087C00020EE270A09B0BDE8F08F029ACDF80CE040
:1087D0000EEB020191FBF3F203FB12114A1C92FB18
:1087E000F3F503FB152206EB810500EB8101D1EDCA
:1087F000006A0591A11895ED007A04951F1B91FB65
:10880000F3F503FB15110091F0460191154606970B
:10881000039F06998F420CDB049991ED007A05992C
:10882000D1ED006A0699884574DB0134AEF1020E81
:10883000BFE7AB42D8BF002506EB8509019999ED4A
:10884000000A8B42D8BF0021B4EEC70A00EB850AAC
:1088500000EB810BF1EE10FADAED007A9BED006A85
:1088600001914FEA810C10DCF4EEE67AF1EE10FA99
:108870002EDC0199039F01310137013501910397E6
:10888000F0EE676AB0EE407AC2E7B444DCED005A1D
:10889000B4EEE50AF1EE10FAE6DDF4EEC75AF1EEB9
:1088A00010FA58BFB0EE657A89ED007AAC464FF009
:1088B00001094C45D8D00CF1010C6345D8BF4FF0ED
:1088C000000C06EB8C0B8BED007A09F10109F0E747
:1088D000F4EEC67AF1EE10FACBDDB4EEE66AF1EE14
:1088E00010FA54BFB0EE460AB0EE660A8AED000AEE
:1088F000AC464FF001094C45BBD00CF1010C63456F
:10890000D8BF4FF0000C00EB8C0A8AED000A09F189
:108910000109F0E79342D8BF002206EB82070099D5
:1089200097ED000A8B42D8BF0021B4EEC70A00EBD6
:10893000820C00EB8109F1EE10FADCED007A99ED82
:10894000006A00914FEA810516D53544D5ED005AED
:10895000B4EEE50AF1EE10FA0ED5F4EEC75AF1EED8
:1089600010FAD4BFB0EE650AB0EE470A87ED000AF0
:1089700015460127BC4223D1F4EEE67AF1EE10FA57
:1089800013D5F4EEC67AF1EE10FA0ED5B4EEE66A1F
:10899000F1EE10FAD4BFF0EE467AF0EE667ACCED46
:1089A000007A15460127BC4214D1009901310132E9
:1089B000009108F10108F0EE676AB0EE407A31E705
:1089C0000135AB42D8BF002506EB850989ED000AC9
:1089D0000137CFE70135AB42D8BF002500EB850C4E
:1089E000CCED007A0137DEE70000000003690133B7
:1089F000012B036108D1DFED117A80ED010A80EDD2
:108A0000000AC0ED027A704790ED006A07EE903AD6
:108A100070EE466AF8EEE77A86EEA77AD0ED027A33
:108A200037EE067A30EE470A80ED017AE6EE807A7C
:108A3000B0EE470AC0ED037AE1E700BF0000000096
:108A400003685A1C026019707047007970470079FA
:108A5000C0F3401070470079400970472DE9F84392
:108A6000D0F8148007468946B8F1000F57D1056841
:108A7000C5F30D0606B3D9F80060FFF793FB09288C
:108A800040F08680444C236923F4407323612369BA
:108A900043F400732361236943F0010323612E60D3
:108AA000FFF780FB2369092823F0010323616FD1BD
:108AB0003B6804333B6032E0384B9D4229D303F5D9
:108AC00080439D4224D303F580439D422AD3344BF7
:108AD0009D4229D903F580339D4227D903F5003300
:108AE0009D4225D903F500339D4223D903F5003378
:108AF0009D4221D903F500339D421FD903F5802300
:108B00009D421DD9B5F1016F1CD305200BF0F0F883
:108B10000826FFF747FB092816D04FF0FF384046DC
:108B2000BDE8F8831026F4E71826F2E72026F0E7E0
:108B30002826EEE73026ECE73826EAE74026E8E785
:108B40004826E6E75826E4E7134C236923F44073EC
:108B50002361236943F400732361236923F0F8033D
:108B600023612369334343F002032361236943F400
:108B700080332361FFF716FB236923F0020323618F
:108B80002369092823F0F80323613FF474AFC4E795
:108B90006FF00108C3E700BF003C0240004000083E
:108BA000FFFF000803682DE9F0410D4641681344BA
:108BB0008B42044619D8AE1800F10C074FF000089C
:108BC000B54202D16069BDE8F08123695A1C226177
:108BD000234415F8011B1973042AF1D139462046A4
:108BE000FFF73CFFC4E90480EAE74FF0FF30EAE713
:108BF0002DE9F0479846444B914603EB8002054629
:108C00009468002C51D02833636004F13E03A361C3
:108C100004F59F73E3614FF48073C4E90433236860
:108C200094F83D00E160A36307F068FA064694F803
:108C3000440294F83CA0271D08B152F0ADF894F816
:108C4000450208B152F0A8F8D4F840321BB12F4ABF
:108C5000116B0B43136318F0080F2FD00135EDB2E1
:108C60001EB140F20673F380357218F0100F94F8BD
:108C700046221DD00221304607F000FAD4F84822DF
:108C800094F9471294F8473212010029D2B236DB28
:108C90001F49C81880F800235809012203F01F0358
:108CA00002FA03F341F820303C462046BDE8F08745
:108CB00018F0200F0CBF32211221DCE719F0020F4F
:108CC0000CD06B1CDBB21EB140F20652F280337244
:108CD00094F846220221304607F0D0F919F0010F2E
:108CE000CCD0504607F00AFA0135EDB218B140F287
:108CF0000663C380057294F846220221BCE7054949
:108D000003F00F03CA54CFE7005A060800380240A8
:108D100000E100E014ED00E02DE9F341038A8689CB
:108D2000B6B205460C461E404FF0004816B902B0D8
:108D3000BDE8F081B6FA86F328FA03F2D24391B285
:108D4000298216401B3B002C3ED0042BEED8DFE8D6
:108D500003F037312B250300E368EF6A23B19B68EA
:108D600013B1B9B2201D9847636A2BB19B681BB140
:108D7000B9B204F11C009847E36B2BB19B681BB19F
:108D8000B9B204F134009847636D002BCED09B68D4
:108D9000002BCBD0B9B204F14C0003E0E368696B5F
:108DA0005B68201D9847C1E7636AA96B5B6804F1A3
:108DB0001C00F7E7E36BE96B5B6804F13400F1E753
:108DC000636D296C5B68E6E7042B06D8DFE803F0E7
:108DD0000D0B09070300EB6A0193019BA6E76B6B80
:108DE000FAE7AB6BF8E7EB6BF6E72B6CF4E790F880
:108DF0004820531C0244DBB280F8483082F834101B
:108E000090F849200AB1132B01D954F087BC704760
:108E1000002280F8492054F081BC70B5124D044600
:108E200095F8833A002BFBD16618B44204D1002098
:108E300070BD01200AF002FCD5F8843AD5F8882AE2
:108E40000133C3F30A039342F3D0D5F8843A14F8FC
:108E5000012B2B4483F88C2AD5F8843A0133C3F3D1
:108E60000A03C5F8843AE0E7781A002038B50C46C2
:108E70001146FFF7E7F948B1054D002AD5F89431BE
:108E800004DD2046FFF7C9FFD5F8943138BD00BF97
:108E9000702B0020F0B585B0D0F8CC1590F8CC65DB
:108EA0000291D0F8D0150391012180F8111106F03C
:108EB0001F01B0F8D22590F8CD75B0F8CE35B0F8D6
:108EC000D055C0F840210129044600F0098102294B
:108ED00000F01A81002940F09381092F5ED8DFE865
:108EE00017F0B600F4005D00C8005D0057000A00EE
:108EF0005D00A90076001D0A022DADF806200BD0FA
:108F0000032D25D0012D49D1D0F8EC351B68A07870
:108F10000DF10601984709E0D0F8E43580789B6AA6
:108F20000DF1060198474570C4F8F005BDF806201C
:108F3000002A47D0BDF80E30002B43D09A4228BFFC
:108F40001A46ADF806200146204653F039FF39E0B5
:108F5000DBB2052B22D8DFE803F003070B0F131752
:108F6000D0F8EC355B68D2E7D0F8EC359B68CEE7FB
:108F7000D0F8EC35DB68CAE7D0F8EC351B69C6E7FA
:108F8000D0F8EC355B69C2E7D0F8EC359B69BEE7F9
:108F90002A4303D190F81211032903D1204653F03C
:108FA00039FE0FE003F07F05016980F8145163F387
:108FB0000A120B681A430A6053F016FF2DB1022300
:108FC00084F81231002005B0F0BD0123F8E7D9B2D2
:108FD0008D4D012985F89811E0D890F81231022BB7
:108FE0000FD0032BDAD1C1B9022380F81231D0F8A7
:108FF000E43580F810115B689847204653F0F4FE82
:10900000E0E70029F9D00121032380F8101180F84E
:109010001231204653F0C0FDEFE790F810110129FE
:10902000EBD0D0F8E4355B68984795F8981184F850
:109030001011EEE7012AB1D190F81231022B04D0C1
:10904000032BABD100F588717EE770497CE790F87F
:109050001231023B012BA1D86B4B0022C3F8A02197
:10906000D0F8182112B10222C3F8A02168490222C7
:109070006AE7012B08D1C4F81831D4F8E43502A905
:109080009B6820469847B8E7022B9BD1EBB2002B98
:1090900098D103692D0A023D5A68032D13D8DFE8E1
:1090A00005F0020C0E10022363F30612564BC3F8B0
:1090B000A421012384F816319FE70323F4E7042356
:1090C000F2E70523F0E70123EEE790F81221023AD8
:1090D000012A3FF663AF012B7FF474AF0023CAE788
:1090E00090F81231032B7FF459AFEDB2012D3FF60A
:1090F00055AFD0F8E43502A99B689847BDF80E300B
:10910000002B7FF45FAF78E706F06006202EE9B20F
:1091100005D1D0F8E43502A99B68984752E7012FA2
:1091200035D0032F23D0002F7FF44CAF90F81231AD
:10913000022B5FD0032B7FF431AF15F0800F4FF07F
:1091400028031BBF01F07F0103FB010103FB0101A9
:1091500091F81E3108BF91F876332B49003B18BFB8
:109160000123C1F8A831022201F5D471ECE690F890
:109170001221022A3ED0032A7FF410AF002B7FF485
:109180007CAF4A063FF479AF53F012FD75E790F8D3
:109190001221022A2ED0032A7FF400AF002B7FF485
:1091A00011AF11F07F023FF428AF6DB22823002DDC
:1091B000B5BF03FB020303FB010303F58E7303F545
:1091C0005D73002199701A70E90F00EB82025970EB
:1091D000002DB4BF9269526DD9781368023923F417
:1091E000001301298CBFC3F30071012161F31C73CB
:1091F000136042E74B063FF4E5AE53F0D9FCE1E6DD
:1092000006F08001F9E700BF702B00200C2D002034
:10921000102D002010B5044671BB90F81131032BBE
:109220001BD1D0F89023D0F87C339A4217D9C1785B
:10923000012908BFD0F88013A2EB030204BFC918AC
:10924000C0F88013934228BF1346C0F890239BB206
:10925000D0F88023002153F077FE002010BDD0F815
:10926000E4351B6923B190F81221032A00D19847F5
:10927000204653F0B9FDF0E7D0F8E4359B69002BA8
:10928000EBD090F81221032AE7D19847E5E770B5B3
:109290000A7812F0600305460C4628D0202B2DD109
:1092A000CB884E78EBB112060AD51D491A463046D6
:1092B000FFF7B6F8E2881A49284653F081FD0EE020
:1092C000184A1660184A0321C2F80C3880F81111A8
:1092D000C0E9E43302F50162002153F035FE0020BD
:1092E00070BD022211443046FFF79AF8F7E74B7839
:1092F0000A2B08D00B2B09D0062BF0D1284653F0AF
:1093000089FC0220ECE709490122D6E78B781BB9DA
:10931000074AC2F8AC31E2E753F07CFCDFE700BF5C
:109320008822002000000020781A00201C2D002038
:10933000702B002038B5282303FB0101074DB1F83D
:109340008C1304462846FFF7ADF8204640232A46F2
:10935000012153F0F9FD002038BD00BF202D002071
:1093600070B50E4BD3F8FC2193F8F051044632B19E
:1093700093F800322B4302D1012153F019FC8121D3
:10938000204653F015FC022D07D12046044ABDE8C3
:1093900070401F23012153F0D7BD70BD702B0020FA
:1093A000642D0020002310B519460446402253F0D6
:1093B00069FC402280212046002353F063FC0123F6
:1093C00084F81231D4F8E835A0785B68984700201B
:1093D00010BD38B5402204460223812153F052FCCF
:1093E000204602234022012153F04CFC2046032357
:1093F0000822822153F046FC084B0222002583F804
:109400004B2083F84C500121FEF7F5FF2046044A1B
:10941000402353F099FD284638BD00BF00000020CE
:10942000202D002010B58121044653F001FC204678
:10943000012153F0FDFB2046822153F0F9FBFEF79A
:10944000E7FF002010BD10B58121044653F0F0FB6A
:109450002046012153F0ECFB024B002083F814025C
:1094600010BD00BF702B0020F8B5224C94F8832A61
:10947000012A03462ED1204FD7F8185215B984F887
:10948000835A23E0402D23D8AEB2402E02D10222CF
:1094900084F8832AD4F8881A184A0A44C3E9542263
:1094A00040F201110022A3F84411C3E9566203F50A
:1094B000A271184653F0AFFCD4F8883A3344C3F392
:1094C0000A03AD1BC4F8883AC7F818520020F8BD4B
:1094D0004026DFE7022AF9D1002540F20112C0E957
:1094E0005455C0E95655A0F8442100F5A27153F037
:1094F00092FCC4E7781A0020702B0020042500207D
:10950000F8B5284FD7F81C320F2B03F1010203D016
:10951000C7F81C220020F8BD234C0023C7F81C32DA
:1095200094F8833A002BF5D1D4F8882AD4F8843AF9
:109530009A42EFD0D4F8882AD4F8843A9A4295BF58
:10954000D4F8845AD4F8885AD4F8883AC5F5006516
:1095500098BFED1A402D22D8AEB2402E0CBF022388
:109560000123D4F8882A84F8833A104B1344C0E9C5
:10957000543340F201120023C0E95663A0F844219D
:1095800000F5A27153F047FCD4F8883A3344C3F392
:109590000A03AD1BC4F8883AC7F81852BAE701238A
:1095A0004026DEE7702B0020781A002004250020DA
:1095B000064BD3F880391A79022A05D19A689207A6
:1095C00002D5586952F0A8BF704700BF781A002032
:1095D00010B50A4CD4F8800906F02EFB58B9D4F81F
:1095E00080090379022B08D183689B0705D5BDE864
:1095F000104008F0ABB800BFECE710BD781A0020AF
:1096000073B50A4E441C0025D6F8800901230022B8
:109610000DF1070154F0C4F89DF80700FF2802D1AE
:109620000135A542F0D102B070BD00BF781A00200C
:1096300070B5044608200D46FFF7E2FFFF2812D060
:10964000FE2812D10A4E2B46D6F880090022214668
:1096500054F0A6F80022D6F880090223114654F0EF
:109660009FF8002070BD0120FCE70220FAE700BF50
:10967000781A002037B5124D4FF6FF530024D5F865
:109680008009ADF8043001AA02232146C5F84C49EF
:1096900054F086F80120FFF7B3FFFF2805D104231B
:1096A00085F85039022003B030BD092385F85039C0
:1096B000044BD3F89431C5F840392046F3E700BF96
:1096C000781A0020702B002013B540F040038DF86D
:1096D00000300B0E8DF801300B0C8DF802300B0AA8
:1096E0008DF80330952304468DF804108DF805306D
:1096F00054F07CF800B964B907480623D0F8800913
:109700006A46002154F04CF80820FFF779FF02B0B8
:1097100010BDFF20FBE700BF781A00202DE9F041C3
:10972000194C1E4694F85039042B054688461746B6
:109730001CD1FFF73DFF94F84639FBB969021120AF
:10974000FFF7C2FFE0B9052384F850390F4BC4F886
:109750002C89D3F89431C4F83059C4F83879C4F856
:109760003C69C4F840390120BDE8F081082B03D1E1
:10977000FFF780FF0228DCD00020F5E72946DEE76E
:10978000FFF726FFF8E700BF781A0020702B0020B3
:1097900038B500220D233521022006F06DFE224C43
:1097A000C4F8800910B984F8500938BD002106F0CA
:1097B000D1F8012009F042FFD4F88059686906F019
:1097C0002AFC95F910301948194D142202FB0300A8
:1097D0000022D0F8B0000A23114653F0B7FFD4F8A6
:1097E000800906F029FA50B9124B84F84409D3F8DD
:1097F0009431C4F84039012384F85039D5E7013D4C
:10980000EDD1D4F88009022106F0A4F8D4F880093B
:1098100006F073F894F84439C4F88059013384F899
:10982000505984F84439C0E7781A0020000000201D
:10983000A1860100702B002038B5134C0023A07BBB
:10984000E0B125688D4219D1104C03F581751AB924
:1098500004EB0514A27138BD04F1180101EB432398
:109860009A4209D1831E5842584104EB051453F023
:1098700095F80123A371EEE70020F6E70133082BEA
:1098800004F11004DBD1E6E7C05E0020A84E002002
:10989000174838B5002380F8A03000F11804256877
:1098A0008D421ED1A57B032D1BD1124C03F5817572
:1098B0004AB904EB05140423A371D0F89C3001339A
:1098C000C0F89C3038BD04F1180000EB4320131A97
:1098D0005842584104EB051453F060F80123A3717A
:1098E000F0E70133082B04F11004D8D1EAE700BFF8
:1098F000A85E0020A84E0020F8B50446144EFFF7DD
:10990000A2FD204602234022812153F0BBF94022D0
:1099100001212046022353F0B5F9D6F82032002564
:109920001B6886F81452284686F8F0519847E76875
:10993000384653F03FFD3846012153F051FD204693
:109940001F2306F5FA72012153F0FEFA2846F8BDEE
:10995000702B0020002108B5084606F01DFF094BBA
:10996000094A03F58071C2F82819D3F800319847E5
:10997000FEF7B8FD0028FBD00121002006F00CFF07
:10998000002008BD00000020781A00202DE9F84FC3
:109990000E460121084615461F4606F0FDFEDFF87B
:1099A0004CA00024A74219DD06EB442905EB04086E
:1099B00001E0FEF797FDDAF82839002BF9D0D3F84B
:1099C00004B000231A4649464046D8470028F0D044
:1099D000FEF788FD0028FBD00134E3E700210120D9
:1099E00006F0DAFE0020BDE8F88F00BF781A0020EC
:1099F0002DE9F84F0E460121084615461F4606F090
:109A0000CBFEDFF848A00024A74218DD06EB44296E
:109A100005EB040801E0FEF765FDDAF8283943B1EB
:109A2000D3F80CB000231A4649464046D8470028D0
:109A3000F1D1FEF757FD0028FBD00134E4E7002107
:109A4000012006F0A9FE0020BDE8F88F781A00205A
:109A5000024BD3F8240207F09FBD00BF702B0020FB
:109A60000068F022FF2107F0A1BECB4341EA0311B9
:109A7000CAB20068D22107F099BE0068B422FF2163
:109A800007F094BE0A460068A52107F08FBE552155
:109A9000F8E700689622FF2107F088BE0A460068B2
:109AA000872107F083BECA01006802F08002782196
:109AB00007F07CBE38B50446154600680A46E12129
:109AC00007F074FE30B120682A46FF21BDE8384017
:109AD00008F0E2BD38BD0A46E121EBE70A46C321A2
:109AE000E8E738B5021D0D46F0210446FFF7E2FF16
:109AF00008B123792B7038BDF8B504460E461546DB
:109B0000071D20683A46FF2108F0C6FD30B116B1A6
:109B10002379DB07F5D40DB123792B70F8BD002232
:109B20000121E9E710B50446FFF7A7FF18B1204669
:109B3000BDE81040F3E710BD10B50446FFF7A2FFE3
:109B400018B12046BDE81040E9E710BD70B50646E3
:109B50000C468D18AC4201D1012006E014F8011B1F
:109B60003046FFF7E9FF0028F4D170BDCC21E3E7D0
:109B700038B504460D46FFF78CFF40B12046FFF78D
:109B8000CEFF20B129462046BDE83840A3E700209B
:109B900038BD70B506460C468D18AC4201D1012087
:109BA00006E021463046FFF7E3FF01340028F4D1F8
:109BB00070BD38B505461446FFF770FF2846FFF71D
:109BC000AEFF20B11CB12B79C3F34013237038BD15
:109BD00010B50446FFF7A6FF38B12046FFF7C6FFD1
:109BE00018B12046BDE8104099E7002010BD73B5BC
:109BF0000546CDE90023FFF795FFA8B12846FFF7FA
:109C000046FF88B12846FFF78AFF68B16E460824F0
:109C100016F8011B2846FFF78FFF28B1013C14F00E
:109C2000FF04F5D102B070BD0020FBE7C90138B5D3
:109C300001F0800104461546FFF735FF08B9002002
:109C400038BD002201212046FFF756FF0028F6D03C
:109C500023795B092B70F3E710B5021D0446FF2141
:109C6000006808F019FD18B12079C04300F0010028
:109C700010BD0F49D1F8883043F47003C1F8883023
:109C80000C4B1A68002042F001021A6098601A68B2
:109C900022F0847222F480321A60074A5A601A68ED
:109CA00022F480221A60D860044B8B60704700BF9A
:109CB00000ED00E0003802401030002400000008F1
:109CC000704782B00023019300933C4B1A6842F422
:109CD00080321A601A6802F400320092019A01324E
:109CE0000192009A1AB9019AB2F5A04FF2D11B68FD
:109CF00013F4003318BF01230093009B012B57D1AD
:109D00002E4B2F491A6C42F080521A640A6842F4B2
:109D100040420A609A689A609A689A609A6842F427
:109D200080529A60274A5A601A6842F080721A601C
:109D30001A689001FCD5244A40F2027111609A68B9
:109D400022F003029A609A6842F002029A601B4B6A
:109D50009A6802F00C02082AFAD19A6802F00C0202
:109D6000042A27D0082A27D159685A685B68490213
:109D7000C3F388134CBF1549154902F03F02B1FBEC
:109D8000F2F253430D4A5268C2F3014201325200CB
:109D9000B3FBF2F3094A91680E4AC1F303110A4476
:109DA00092F85C20D3400C4AC2F8203102B07047D0
:109DB00000BFFDE7054BEDE7054BEBE70038024040
:109DC0000070004019304004003C024040787D01A2
:109DD0000024F400005A0608000000200148FEF7A5
:109DE0004BB900BF280100200148FEF745B900BF6C
:109DF00074030020064A002352F83310814201D137
:109E0000D8B2704701330E2BF6D1FF20704700BF48
:109E10006C5A0608704770B5002828D04C684CB9B9
:109E2000426815685679AB8902229BB2B24023EA98
:109E30000203AB818A683AB943681D68AB8923F095
:109E400001031B041B0CAB81816044B1436819689A
:109E50005D798C890223AB4023439BB28B8132B165
:109E600043681A6893899BB243F00103938170BDE4
:109E70000B4B30B51A4600241D79854208D1DD68A8
:109E8000294203D0142303FB042030BD0029F9D05C
:109E900001340A2C03F11403EED10020F5E700BFD2
:109EA000BC0500200028ACBF00F16040064B4FEA23
:109EB0000111ACBF00F5614000F00F00C9B2B4BFA2
:109EC000195480F80013704714ED00E038B50368AA
:109ED0001B681C68244B07EE902A93ED487AF8EE35
:109EE000677AB8EE477A013987EE270A8DB2DFED3F
:109EF0001F7A30EE270A55F0B5FB1D4A238801383A
:109F0000944280B29BB212D002F5806294420ED08D
:109F1000B4F1804F0BD0A2F58032944207D002F505
:109F20008062944203D002F58062944206D123F00D
:109F300070039BB223F440739BB206E00D4A944237
:109F400003D002F580629442F4D12380084BE5628D
:109F50009C42208503D003F580639C4201D10023FD
:109F600023860123A38238BD000000200AD7233CAA
:109F70000000014000100040F0B543689A795D7917
:109F800012F0040002F0020C11BF0022E6464FF46A
:109F9000807284460FBF0124964604201446032D88
:109FA00038D8DFE805F0023872AC1B681D8C25F04C
:109FB00001052D042D0C1D841D8C9F881E8B25F002
:109FC00002052D0444EA0E042D0C26F073062543E9
:109FD000634C3604360CA342BFB246F0600603D091
:109FE00004F58064A34209D14FF6F3742C4044EA8F
:109FF0000C0427F4407744EA000517439F801E8332
:10A0000059631D841A8B22F008021204120C42F0CC
:10A0100008021A83F0BD1D682B8C23F010031B046B
:10A020001B0C2B842B8CAF882E8B23F020031B045E
:10A0300044EA0E041B0C26F4E64643EA0413484C9B
:10A040003604360CA542BFB246F4C04603D004F530
:10A050008064A5420CD123F0800343EA0C1323F063
:10A0600040039BB227F4406743EA001347EA8207A4
:10A07000AF802E83A9632B842B8B23F400631B04F6
:10A080001B0C43F400632B83C4E71D682B8C23F463
:10A0900080731B041B0C2B842B8CAF88AE8B23F49A
:10A0A00000731B0444EA0E041B0C26F0730643EAFB
:10A0B00004232B4C3604360CA542BFB246F0600692
:10A0C00003D004F58064A5420CD123F4006343EA75
:10A0D0000C2323F480639BB227F4405743EA002308
:10A0E00047EA0217AF80AE83E9632B84AB8B23F082
:10A0F00008031B041B0C43F00803AB838AE71B68AF
:10A10000188C20F480500004000C1884188C9E8851
:10A110009D8B20F40050000444EA0E04000C25F44A
:10A12000E64540EA04300E4C2D042D0CA342B6B295
:10A1300045F4C04503D004F58064A34203D126F45E
:10A14000804646EA82169E809D83196418849A8B05
:10A1500022F400621204120C42F400629A8359E75E
:10A160000000014043685A79032A0FD8DFE802F063
:10A170000205080B1868343070471868383070478B
:10A1800018683C30704718684030704700207047AE
:10A1900010B543681A685879084B0344012093F8B6
:10A1A000DC40138CA0409BB223EA00031384138C81
:10A1B000A140194389B2118410BD00BF005A06089E
:10A1C000F0B5EFF31184102383F31288C568466855
:10A1D000AA68136823F00103136032687779104E80
:10A1E000938936F817609BB223EA060393812A69A4
:10A1F0006D681F2A4FF0200385BF203A934093409B
:10A20000EB6098BFAB60E3B283F31188C3689B68CF
:10A2100059601A6842F001021A6001230374F0BD0C
:10A22000005A06080268137D012B04BF0223137530
:10A2300092F82C100CBF4FF400730023012904BFC7
:10A24000022182F82C1092F8441008BF43F4806376
:10A25000012904BF022182F8441092F85C1008BF63
:10A2600043F4006301290DD1022182F85C1043F40C
:10A2700080534268126800215162918989B20B4370
:10A28000938101E0002BF4D17047034B0348D3F8CE
:10A290002812FEF741BD00BF702B002000000140D6
:10A2A00010B5064C0648D4F82812FEF735FDD4F850
:10A2B00048120448BDE81040FEF72EBD702B002068
:10A2C000000001400040014010B5064C0648D4F89B
:10A2D0002812FEF721FDD4F84C120448BDE81040C6
:10A2E000FEF71ABD702B0020000001400044014021
:10A2F00010B5064C0648D4F82812FEF70DFDD4F828
:10A3000050120448BDE81040FEF706BD702B002037
:10A310000000014000480140034B4FF08040D3F85B
:10A320002C12FEF7F9BC00BF702B0020024B034833
:10A33000D3F83012FEF7F0BC702B00200004004070
:10A34000024B0348D3F83412FEF7E6BC702B002012
:10A3500000080040024B0348D3F83812FEF7DCBC7B
:10A36000702B0020000C00400348D0F8903613B149
:10A3700000F2846018477047000000200348D0F8BE
:10A38000B03613B100F2A4601847704700000020F7
:10A390000348D0F8D03613B100F2C46018477047B4
:10A3A000000000200348D0F8F03613B100F2E4605A
:10A3B00018477047000000200348D0F8103713B149
:10A3C00000F2047018477047000000200348D0F8DE
:10A3D000303713B100F22470184770470000002096
:10A3E0000348D0F8503713B100F244701847704753
:10A3F000000000200348D0F8703713B100F26470F9
:10A4000018477047000000200348D0F8903713B178
:10A4100000F2847018477047000000200348D0F80D
:10A42000B03713B100F2A470184770470000002045
:10A430000348D0F8D03713B100F2C4701847704702
:10A44000000000200348D0F8F03713B100F2E470A8
:10A4500018477047000000200348D0F8103813B1A7
:10A4600000F6040018477047000000200348D0F8A9
:10A47000303813B100F62400184770470000002060
:10A480000348D0F8503813B100F64400184770471D
:10A49000000000200348D0F8703813B100F66400C3
:10A4A0001847704700000020036823F00103036091
:10A4B0000023036043608360C36003612123436121
:10A4C0002A4B984203D13D2243F8082C7047284B71
:10A4D000984204D14FF4746243F8202C7047254B06
:10A4E000984204D14FF4741243F8382C7047224B31
:10A4F000984204D14FF0746243F8502C70471F4BC0
:10A50000984203D11E4A43F8642C70471D4B984271
:10A5100003D11D4A43F87C2C70471C4B984203D151
:10A520001B4A43F8942C70471A4B984204D14FF0C1
:10A530003D5243F8AC2C17E0174B9842C3D0174B51
:10A540009842C7D0164B9842CCD0164B9842D1D0E7
:10A55000154B9842D6D0154B9842DAD0144B9842FE
:10A56000DED0144B9842E2D0704700BF106002402A
:10A570002860024040600240586002407060024023
:10A580003D00002088600240400F0020A060024093
:10A5900000003D20B8600240106402402864024080
:10A5A0004064024058640240706402408864024083
:10A5B000A0640240B86402402DE9F0410022012667
:10A5C00003250B6806FA02F737EA030334D1036860
:10A5D000540005FA04FE23EA0E0303600B79D0F859
:10A5E00000806FEA0E0C03FA04FE013B4EEA080EEF
:10A5F000012BC0F800E014D883680CEA03038360E1
:10A600004B79D0F808C0A34043EA0C038360436849
:10A6100023EA070343608B79476893409BB23B432F
:10A620004360C36805FA04F723EA0703C360CB79E4
:10A63000C768A3403B43C3600132102AC1D1BDE8C3
:10A64000F081204B9A6802F00C02042A10B534D035
:10A65000082A34D159685A685B684902C3F38813E1
:10A660004CBF1949194902F03F02B1FBF2F25343C2
:10A67000144A5268C2F3014201325200B3FBF2F3B2
:10A68000104C0360A168124AC1F30311114491F800
:10A69000E010CB404360A168C1F38221114491F8DE
:10A6A000E01023FA01F18160A168C1F342310A444C
:10A6B00092F8E020D340C36010BD034BE0E7034BAA
:10A6C000DEE700BF0038024040787D010024F4003E
:10A6D000005A0608F0B5446B8668A38923F400533A
:10A6E0001B041B0CA3818579290201F4806C41793C
:10A6F00001F001038907218A4FEA053289B221F46A
:10A70000405102F4005242EA01022282A289C5F3BA
:10A71000800722F4B0524FEA83034FEA073722F052
:10A720000C0248BF43F008034CEA07011204120C64
:10A730000B431343A381A38A23F440731B041B0C14
:10A7400085B0A3826846FFF77CFF204B9C4203D074
:10A7500003F580639C4237D1039BA289192117041A
:10A7600001FB03F34FF064014CBF7600B600B3FB6E
:10A77000F6F3B3FBF1F001FB10330201A0890004F2
:10A780004BBFDB001B01323332334BBFB3FBF1F362
:10A79000B3FBF1F303F0070303F00F0313439BB282
:10A7A0002381A38A2A0755BF23F008039BB21B0409
:10A7B00043F0080358BF1B0CA382A3899BB243F448
:10A7C0000053A38105B0F0BD029BC6E70010014015
:10A7D0002DE9F8431E46204B9DF820509DF824702B
:10A7E0009842894690462CD13B462A463146002065
:10A7F000FEF7FEF904460020C4E90700C4E9090099
:10A80000C4E90B986571A660A7712046FFF762FF47
:10A81000EA0707D5636B4FF6DF721A80DA6842F0F9
:10A820002002DA60626BAB0742BFD36843F080035B
:10A83000D36093899BB243F4005393812046BDE8D3
:10A84000F883064B984204D13B462A463146012004
:10A85000CEE70024F2E700BF0010014000440040B2
:10A86000816037E7417135E7817133E72DE9F043C6
:10A87000654F07EBC00985B005464FEAC00899F857
:10A88000880805F03BFC064699F8890805F036FC77
:10A89000044699F88A0850F07FFA6B1CDBB21EB1AF
:10A8A00040F60C12F28033721CB140F60C22E280AA
:10A8B000237204223A21304605F0E0FB20460422B0
:10A8C0003A2105F0DBFB07EB0803D3F884484F4B34
:10A8D0009C4263D103F5F2331A6A42F400121A6201
:10A8E0001A6A22F400121A62474497F88B38022B36
:10A8F0006ED0032B6ED0464E464A012B18BF16462B
:10A90000A78827F03F0768463F04FFF79AFE3F0CF1
:10A91000029A414BB2FBF3F398B20743A780218818
:10A9200021F001010904090C21803C498E4253D1D8
:10A930003B4BB2FBF3F2013091B2042980B238BF35
:10A9400004212084A18323889BB243F00103238048
:10A95000238823F4816323F002031B041B0C43F4BC
:10A96000806323804FF480432381238823F0800376
:10A970001B041B0C238023889BB243F0010323801C
:10A98000284B03EB4513012283F86122002283F850
:10A99000605283F8622205B0BDE8F083224B9C42EE
:10A9A00009D103F5F0331A6A42F480021A621A6A76
:10A9B00022F4800297E71D4B9C4295D103F5EE33BC
:10A9C0001A6A42F400021A621A6A22F400028AE742
:10A9D000124E95E7124E93E706EB4606B2FBF6F2EF
:10A9E00091B2C2F30B020AB941F001014FF4967221
:10A9F00053434FF47A72B3FBF2F301339BB241F449
:10AA0000004123849EE700BF000000200054004066
:10AA100000350C00801A060040420F00A08601009D
:10AA2000400D0300702B002000580040005C0040E7
:10AA30002DE9F047BE4D460105EB401908F00CFD2D
:10AA400099F96022BB4B8846D10003EBC20207464E
:10AA5000D2F8844899F86222013A142A00F28380DD
:10AA6000DFE812F0790089009F00B800C300CD0034
:10AA7000D600EB00F600FF000A014C0174019A01B8
:10AA8000FD010E022002290249026D0215005F1825
:10AA90004FF0090A97F8880805F030FB044697F84C
:10AAA000890805F02BFBB5F8C03201339BB207468D
:10AAB0002046A5F8C03205F0AEFA384605F0ABFAEC
:10AAC0001121204605F0B1FA1121384605F0ADFA02
:10AAD0004FF0650803E00520002108F00FFD204637
:10AAE00005F090FA10B9B8F10108F4D1204605F04C
:10AAF00097FA0021052008F001FD204605F08BFAA9
:10AB00000520002108F0FAFCBAF1010AE0D1204644
:10AB100005F086FA0021052008F0F0FC384605F023
:10AB20007FFA0021052008F0E9FC204605F073FAC1
:10AB30000520002108F0E2FC384605F06CFAAB195C
:10AB400093F96002431C01D0FFF790FEAB1900227D
:10AB500083F8622207E0238813F4007340F0BA817F
:10AB6000AA1982F86232AB1993F86232002B7FF493
:10AB700065AFBDE8F087238823F400631B041B0C3A
:10AB8000238023889BB243F48063238023889BB275
:10AB900043F480732380AB19C3E99A78032283F8C6
:10ABA000622265492046FDF70EFB002800F09281E5
:10ABB000AB1993F872225AB993F87322FF2A04D181
:10ABC00093F870220AB10A22C2E7AB190422BFE748
:10ABD0000F22BDE7AB1993F8712202F0FE02228228
:10ABE000C3E99A78052283F8622254492046FDF78A
:10ABF000EAFA002800F06681AB190622A8E7AB1933
:10AC000093F873222282C3E99A78072283F862229A
:10AC10004B492046FDF7D7FA002800F05381AB19C5
:10AC2000D3F874223AB9228892B242F40072228098
:10AC3000C3E99A7804E108228AE723889BB243F4A7
:10AC400080732380AB19C3E99A78092283F86222C2
:10AC500039492046FDF7B7FA002800F03B81AB19CF
:10AC6000B1E7AB1993F8712242F001022282C3E9E5
:10AC70009A780B2283F8622232492046FDF7A3FA24
:10AC8000002800F01F81AB19D3F87432012B1AD1C0
:10AC9000238823F480631B041B0C2380EFF31182B1
:10ACA000102383F31288238B23889BB243F4007311
:10ACB0002380D3B283F311880C22AB19C3E99A78AD
:10ACC00083F862224FE7022B15D123889BB243F40D
:10ACD00000632380EFF31182102383F31288238B08
:10ACE000238823F480631B041B0C2380D3B283F3DB
:10ACF00011880D22E1E7238B0E22DEE71249204660
:10AD0000FDF76BFA002800F0E580AB19D3F8782244
:10AD1000511CC3F87812218A1170D3F87422013AB9
:10AD2000C3F874220122C3E99A7883F87C220FE7E2
:10AD3000702B0020000000200100030082000700AB
:10AD400084000700020003004000001081492046F3
:10AD5000FDF743FA002800F0BD80EFF311821023C5
:10AD600083F3128823889BB243F400732380AB19CA
:10AD7000D2B2D3F87812481CC3F87802208A08703F
:10AD800082F31188D3F87822511CC3F87812218AF3
:10AD900011706FF00102C3E76E492046FDF71DFAFE
:10ADA000002800F09780AB1903F51A71D3F87422CC
:10ADB000032A30D1228822F480621204120C2280ED
:10ADC000EFF31180102282F31288D3F8782202F177
:10ADD000010CC3F878C2B4F810C082F800C0228811
:10ADE00092B242F400722280C2B282F31188D3F888
:10ADF0007822501CC3F87802208A1070D3F874228D
:10AE0000023AC3F874220C2283F86222C3F86872F3
:10AE1000C1F80480A7E6022A14D8228822F48062AE
:10AE20001204120C2280228892B242F40072228014
:10AE3000228AC3F86872002283F87C22C1F8048059
:10AE4000012285E6D3F87822501CC3F87802208AC4
:10AE50001070D3F87422013AC3F87422D6E723881D
:10AE600023F480631B041B0C2380AB1993F871221D
:10AE700002F0FE022282C3E99A78102283F862224D
:10AE800035492046FDF79FF9E0B1AB1993F87322DD
:10AE9000FF2A04D193F870220AB1132258E6AB19A5
:10AEA000112255E6AB1993F873222282C3E99A78EE
:10AEB000122283F8622229492046FDF784F908B15D
:10AEC000AB19EAE726492046FDF787F910B1AB191F
:10AED00014223DE6A919D1E99A2342F21070BA1A58
:10AEE00068EB0303824273F10003FFF43CAE1523C9
:10AEF00081F8623237E6AB1903F51A70D3F8742281
:10AF000082B1D3F87812013A11F801CBA4F810C03D
:10AF1000C3F87422C3F86872C3F87812C0F80480CA
:10AF2000122215E6228892B242F400722280012297
:10AF3000C3F8687283F87C22C0F8048008E623888E
:10AF40009BB243F4007323804FF6FF33A382AB1907
:10AF50006EE600BF040000108200070084000700B6
:10AF60000004001038B5114C04EB401494F8615201
:10AF7000D5B1C4F87432049BC4F87832002384F845
:10AF80007C320223490084F8732284F86232012261
:10AF90009DF8143084F8711284F8722284F87032AB
:10AFA000FFF746FD94F87C52284638BD702B0020F0
:10AFB00038B5114C04EB401494F86152CDB1C4F88B
:10AFC0007432049BC4F878320223490084F8732257
:10AFD00084F8623200229DF8143084F8711284F8EB
:10AFE000722284F87C2284F87032FFF721FD94F8F5
:10AFF0007C52284638BD00BF702B002082B0002351
:10B000000193054B0193019B03EB80030193019B8B
:10B01000196002B0704700BF5028004082B0002382
:10B020000193054B0193019B03EB80030193019B6B
:10B03000186802B0704700BF5028004010B51C20AF
:10B0400005F05CF81121044604F0EFFF204604F0FF
:10B05000E7FFC82008F0F2FA2046BDE8104004F0EF
:10B06000DABF436D064A1A61C278012A06D100F29E
:10B07000CC5058611A684FF080221A60704700BFA8
:10B080001800086038B5044600296DD190F81131D8
:10B09000022B28D1D0F83821D0F824118A4230D997
:10B0A000C378012B02BFD0F828315B18C0F82831D3
:10B0B000521AD0F82831C0F838214FF48071002599
:10B0C00092B2A0F81C11C0E94A33C0F83451C0F85C
:10B0D000302100F58E7151F01FFE2B462A4629467D
:10B0E000204651F031FF94F81631012B07D1244A44
:10B0F0002369D2F8A4215A60002384F81631002075
:10B1000038BDD0F83C31B3FBF1F501FB1535A5B9DD
:10B11000994212D8D0F8402193420ED24FF4807356
:10B12000C0E94A55C0E94C55A0F81C3100F58E71B4
:10B1300051F0F2FDC4F84051CFE7D4F8E435DB68B4
:10B140002BB194F81221032A01D1204698470523F8
:10B1500084F81131002320461A46194651F0F4FEB6
:10B160002046FFF77EFFBEE7D0F8E4355B69002B91
:10B17000C5D090F81221032AC1D19847BFE700BF7C
:10B18000702B002070477047704710B50F4C94F833
:10B19000CE32B3B14FF0E022D2F8103D23F00603D7
:10B1A000C2F8103DFEF765FDD4F8D4329B68DB078A
:10B1B00007D5D4F8D023136823F0030161F3070304
:10B1C0001360034B4FF480225A6110BD702B002096
:10B1D000003C01402DE9F04FB14CD4F8D0325A690F
:10B1E000D0078BB000F196815A699B6912EA030A75
:10B1F00000F09081CAF307431AF4002F01930FD097
:10B20000D4F8D432DFF8A0829E69DB691E40360C88
:10B2100004F5467B04F531790027002E40F07D814E
:10B22000019B59070DD5D4F8D4329E4D9F69DB6937
:10B230001F40BFB205F118064FF00008002F40F084
:10B24000AD811AF0020F1FBF954BD3F8D032022206
:10B250005A61BAF1000F5FFA8AF51BDA904B93F846
:10B26000CE223AB1D3F8D023136823F0030161F35F
:10B2700007031360D4F8D4228A48536823F00103EB
:10B280005360894BD3F8B4389847D4F8D0324FF094
:10B2900000425A611AF4006FCAF307262FD0002328
:10B2A0008DF8173094F8D6338DF817307E4B7D48E3
:10B2B000D3F8B0389847D4F8D022D4F8D4324FF429
:10B2C00000619B68516194F8CE22C2B1DB0716D5AC
:10B2D00094F8D933012B12D19DF81730032B0ED1DE
:10B2E000D4F8D0331A6842F001021A601A6842F0AA
:10B2F00003021A606D4A136943F0060313612F07B6
:10B3000008D5694B6748D3F8A8389847D4F8D032A5
:10B3100008225A61ED0614D5D4F8D002836923F0CF
:10B3200010038361036AC3F34341022903F00F0250
:10B3300000F0E981062900F00D82836943F01003D3
:10B340008361F00633D5D4F8D452D4F8D0826B6838
:10B35000002723F001036B603946404652F040F865
:10B3600094F8C5C25249B9463B46FF206345C0F038
:10B37000FF814FF0FF33AB614FF00113EB610B2303
:10B3800063F3070763F307096F61C5F810902B6833
:10B39000444823F4FE632B60FFF763FE4FF48053B1
:10B3A000C8F81430404B3F48D3F8AC389847B10642
:10B3B0006DD5D4F8D462D4F8DC22B3681168C3F335
:10B3C0004103022B14BF0023032363F30A0111601E
:10B3D000736843F48073736006A8FFF732F9D4F8FA
:10B3E000D0520799E86820F47050E860B36813F011
:10B3F000060FC3F3410200F0C2812E4B2E4A0B44CC
:10B40000934240F2C0812D4AA1F57403A3F5105375
:10B41000934240F2BC812A4B2A4A0B449342C0F02B
:10B42000BA81294AA1F18C73A3F54343934240F2B8
:10B43000B681264B264A0B449342C0F0B481254B7B
:10B44000254A0B449342C0F0B281244AA1F1B7735C
:10B45000A3F558539342C0F0AD81214B214A0B44D0
:10B460009342C0F0AB81204B204E0B44012240217F
:10B47000B34234BF06230523094E63F38D204FF4F6
:10B480000053E86086F8C622A6F8C8126B61019BDB
:10B49000DA0632D5044B0348D3F8B838984727E08A
:10B4A000702B0020342E00200000002000ED00E072
:10B4B000482E0020401E1BFF3F420F00DFC8100037
:10B4C0002013FBFE20D61300FF69180000D3CEFE28
:10B4D00040771B00C05BB3FEC091210040AC270049
:10B4E000C01D6AFE40E13300803C36FEE09C410016
:10B4F000D4F8D0324FF480125A61019B9B0609D5D3
:10B50000B04BB148D3F8BC389847D4F8D0324FF498
:10B5100000125A610BB0BDE8F08FF10737D5DBF8A8
:10B520000010D4F8D4328D685B691D40EA071ED53F
:10B5300094F8C7320125AB428D6007D10969D9F86B
:10B540007C33C1F312015B1AC9F88C33D8F89C38EC
:10B550009D48F9B2984794F8C732012B07D137B903
:10B5600094F8D533052B02D19748FFF77AFDAB0746
:10B5700042BFDBF8003002259D60280707D5D8F8C8
:10B58000A43891489847DBF8003008229A600137C8
:10B5900076080BF1040B09F128093EE6FA0772D58B
:10B5A000D4F8D43232681869D3F83490916829FA03
:10B5B00008F94FEAC9195FFA89F949EA000909EA65
:10B5C000010919F0010F1FD0596B012000FA08F092
:10B5D00021EA000159637B4B7B48D3F8A0384FF038
:10B5E0000109C2F808905FFA88F1984794F8C732C9
:10B5F0004B4509D1B8F1000F06D194F8D533042B8F
:10B6000002D17148FFF72DFD19F0080F1EBF3368F6
:10B610004FF00809C3F8089019F0100F1EBF3368E7
:10B620004FF01009C3F8089019F0400F1EBF33689F
:10B630004FF04009C3F8089019F0020F1EBF33689D
:10B640004FF00209C3F8089019F0800F1BD0D5E91C
:10B650004C329B1AD5F82421D6F800B0934228BF6B
:10B6600013465A4ADBF8180092F8C7C2D2F8D492AF
:10B6700003339B080293029B80B2984203D9D5E919
:10B680004C03984205D808F101087F082835043694
:10B69000D4E5C01AD5F82431984228BF1846C31CF7
:10B6A0009B080293BCF1000F1BD0D5F82811D5F8E8
:10B6B00034210144C5F82811D5F8301102448A42DA
:10B6C000DBF81800C5F83421D5D195F81C11D9F84C
:10B6D0003420012303FA01F122EA0102C9F83420DF
:10B6E000C9E782B2D6F8B810D5F828E10332931032
:10B6F00003930A466146039B8B42D6D05EF8213005
:10B7000013600131F7E747F6F07119423FF415AEC7
:10B71000282101FB0241C3F30A13DD1CD4F894C3B2
:10B72000D1F84476AD1000218D420DD1282101FBC6
:10B730000242D2F844161944C2F84416D2F8501600
:10B740001944C2F85016F8E5DCF800E047F821E0AB
:10B750000131E9E7D4F894130D68C4F890580968EA
:10B76000C4F89418282101FB0242C3F30A13E5E749
:10B7700051F8042F9060CA6B01339060F6E54FF4E6
:10B780000071092378E6012240210E2374E601228C
:10B7900040210D2370E6012240210C236CE601229A
:10B7A00040210B2368E6012240210A2364E601229E
:10B7B0004021E6E70122402108235DE601224021E5
:10B7C000072359E600000020342E0020702B0020B3
:10B7D000034BD3F87C0908B104F014BC0120704776
:10B7E000781A002008B5FFF7F3FF0A4A18B90023BA
:10B7F00082F8503908BD92F844390133DBB2072B87
:10B8000082F84439F3D8044BD3F89431C2F8403964
:10B810000123EDE7781A0020702B0020F0B5C54C0D
:10B82000D4F8800985B0002861D094F85039013BE4
:10B83000082B44D8DFE813F009005D00DF00430067
:10B84000AA01300186014300E601FDF7B1FE0021A7
:10B850000846FDF739FF0546FDF7BAFE012D29D14F
:10B86000002684F84569FDF7A3FE40F2AB110820DD
:10B87000FDF72AFF05280AD184F84559FDF7A8FEEF
:10B8800094F84539A3B1022384F85039CDE7012853
:10B89000F4D10423D4F880093246694651F080FF80
:10B8A0009DF80330AB2B04BF022384F84539E5E74C
:10B8B00084F85039D4F88009022104F04BF894F848
:10B8C0005039013B022B09D89B4BD4F84029D3F8BF
:10B8D00094319B1AC82B01D9FFF784FF94F85009C3
:10B8E000042800F0A081A0F108035842584105B097
:10B8F000F0BDFDF75DFE94F84559AA1E554255412D
:10B90000AD0700213720FDF7DFFE29462920FDF78E
:10B91000DBFE0546FDF75CFE002DCBD194F84539E2
:10B92000022B17D1FDF744FE29463A20FDF7CCFE45
:10B93000042306462A46D4F88009694651F030FFB0
:10B94000FDF746FE16B1FFF74DFF6EE7009D2DBADD
:10B95000C5F3807584F84659FDF72AFE00210920B9
:10B96000FDF7B2FE10B1FDF733FEA3E773481021D7
:10B97000FDF75EFE06460028F5D101217F204FF03D
:10B9800073F801280546EED1022130464FF06CF8DD
:10B9900050B10128E7D116213A204FF065F8013067
:10B9A0008002C4F8540918E004212C204FF05CF800
:10B9B000032107464E204FF057F80C21064636204B
:10B9C0004FF052F80236431CB340BD40A3FB05358F
:10B9D0005B0A43EAC553C4F85439FDF7F9FDFDF796
:10B9E000E7FD00210A20FDF76FFE08B903234BE7AE
:10B9F000FDF7EEFDA7E710216846FDF719FE0028C8
:10BA00007FF458AF9DF8003084F85A39BDF8013002
:10BA10005BBAA4F858399DF8033084F85B39019B70
:10BA2000C4F85C399DF808301A0903F00F0384F854
:10BA30006539DDF8093084F864291BBAC4F8603927
:10BA40009DF80D309DF80E201B01DBB243EA121366
:10BA500003F5FA6302F00F02A4F8663984F8682946
:10BA6000FDF7B6FD94F846394BB1D4F880090221B0
:10BA700003F070FF0023C4F84C39042304E7FDF7FA
:10BA800097FD4FF400711020FDF71EFE0546FDF7EF
:10BA90009FFD002DE9D056E794F83419D4F82C29ED
:10BAA000D4F88009802302EBC112002151F078FE06
:10BAB00094F834390133DBB2042B84F834397FF441
:10BAC000FEAE1F4AD4F880090223002151F068FE1F
:10BAD0000123D4F880090022694651F061FE9DF8E7
:10BAE000003003F01F03052B15D1072384F85039CC
:10BAF000114BD4F83859D3F89431C4F84039002D9B
:10BB00003FF4DDAED4F83C39D4F82C29D4F8301900
:10BB10000120A847D3E6FFF765FED4F83859002D79
:10BB20003FF483AED4F83C39D4F830190022012018
:10BB3000A8477AE6781A0020702B0020E423002022
:10BB4000F05A060851F052FE002862D0002384F813
:10BB50004439D4F84C39012B0BD9013BC4F84C398A
:10BB6000D4F848390133C4F84839082384F85039E7
:10BB7000A5E607D1FDF77EFD02287FF4A0AEFDF714
:10BB800027FD9CE6042384F85039F8E7D4F82C0903
:10BB90004FF40071FDF74CFD0128054619D002282D
:10BBA00020D000287FF48BAEFDF712FDD4F8386961
:10BBB00084F84459042384F85039002E3FF47FAEB2
:10BBC000D4F83C39D4F82C29D4F830192846B04799
:10BBD00075E6164BD3F89421D4F840396433934278
:10BBE000BFF46DAEFDF7F4FCFFF7FCFDD4F8385957
:10BBF000002D3FF41AAE0022D4F83C39D4F83019A5
:10BC0000104695E751F0F2FD18B1FDF7E1FC042371
:10BC1000ACE7064BD3F89421D4F84039FA33934279
:10BC2000FFF491AE4BE6012061E600BF702B0020CF
:10BC30002DE9F341284C05460E4690461F4694F8E0
:10BC40005039042B0DD0082B07D1D4F84839AB421A
:10BC500019D0FDF70FFD0228F1D0012002B0BDE898
:10BC6000F081FDF7A5FC94F8463953B96902182014
:10BC7000FDF72AFD38B1FDF7ABFCFFF7B3FD03205C
:10BC8000ECE72946F3E794F85039D4F88009082BFB
:10BC900014BFFE23FC23FF228DF804208DF805300D
:10BCA00001AA0223002151F07BFDD4F880098023F2
:10BCB0003246002151F074FD012384F83439062303
:10BCC000C4F82C69C4F83059C4F83889C4F83C79F0
:10BCD00084F850390020C1E7781A002070B51C4C58
:10BCE00094F85039042B05460E4610D1FDF760FC40
:10BCF00000213720FDF7E8FC31461720FDF7E4FC72
:10BD000090B1FDF765FCFFF76DFD032002E0082B05
:10BD100001D0012070BDD4F84839834214D0FDF71A
:10BD2000A9FC0228F5D1E1E794F8463973B9690214
:10BD30001920FDF7C9FC0028E3D1082384F8503905
:10BD4000C4F84C69C4F848590220E3E72946EFE7F4
:10BD5000781A0020034BD3F8280908B14369184723
:10BD6000704700BF781A0020034BD3F8280908B1A8
:10BD700083691847704700BF781A0020034BD3F837
:10BD8000280908B1C3691847704700BF781A002016
:10BD900038B50D461446FFF7F1FF03682B604FF4EA
:10BDA00000732360002038BD034B1B78032B14BFA6
:10BDB0004FF4807080207047A84E002008B50B4AD1
:10BDC00068B1816811B10723937008BDFFF7ECFFDC
:10BDD000C2E90311C2E9010011750423F4E702F579
:10BDE0008051012381F8B4315370EEE7A84E002052
:10BDF00010B502784368022A0B4A06D1D2E98021A5
:10BE000002EB410202EB532010BD0169D2F8180287
:10BE1000D2F8104218400239D2F80C32400A04FB22
:10BE200001001844F0E700BFA85E0020064B1B7815
:10BE3000022B0BBF030AC0F3D413C0B200F07F0083
:10BE40000B601060704700BFA84E002090F91A30B8
:10BE50005A1C0AD003F58172124B03EB0213DA79F4
:10BE600022F00102DA71FF23837690F91B104B1C3C
:10BE700016D00C4A01F5817102EB011302EB01129D
:10BE8000DB79D179C3F34503012B86BF03F1FF337F
:10BE900003F03F03002363F34601FF23D171C37610
:10BEA000704700BFA84E002008B5FFF77DFF034B89
:10BEB000D3F810325843400208BD00BFA85E0020EE
:10BEC0000378022B09D10E4BD3F820224368B3EB41
:10BED000422F2CBF012000207047006970B1094B30
:10BEE0001B78032B0EBF084B80B24FF6F7739842B6
:10BEF00094BF0020012000F0010070470120FAE704
:10BF0000A85E0020A84E0020F7FFFF0F4368F7B59A
:10BF1000C3F308020A44B2F5007F04460D4604D27A
:10BF20002B446360012003B0F0BDFFF78FFF03785F
:10BF3000022B01D16368F3E7154BD3F81022B5EB60
:10BF4000422F4FEA422706DCD3F8183246681E40DB
:10BF50007342AB4201DD0020E5E7AB19BB4210D3D1
:10BF60000169007E01AA50F0F9FD0128F3D123698F
:10BF70006361019B236163683B449B1BEF1B636010
:10BF8000BD192046FFF79CFF0028CBD1D2E700BFA8
:10BF9000A85E002070B504460E461546FFF7B6FFB2
:10BFA00020B10DB12046A847012070BD94F82800AB
:10BFB000022320B9C4E90B5684F82830F5E7184667
:10BFC000F3E738B5174D05F58054014694F8E001C4
:10BFD00030BB49B191F828302BB9442204F5DC700C
:10BFE00057F0BEFA012038BD44220F4858F0DAFB62
:10BFF0004FF6FF73A4F8D231032384F8D0312B78A5
:10C000000948022B18BF032384F8B831D4F81C3236
:10C01000C4F8DC31102384F8D1314EF0EFFEE1E7B3
:10C020000020E0E7A84E002060600020044A92F85B
:10C03000B411012309B982F8B431024A5370704730
:10C04000A85E0020A84E00202DE9F74F12F002094B
:10C050008A461546019304D018B9FFF7E7FF02207E
:10C060000CE0684AD2F808625EB1D2E9831404FB9E
:10C070000611884205D3FFF7D9FF002003B0BDE8C1
:10C08000F08F4FF0FF31604EDFF880B18C468E4666
:10C09000884600243368B77B984221D1002F46D0D0
:10C0A000D2F89810594E0131C2F8981004F58172F7
:10C0B0001201B1502146554C01F5817604EB061270
:10C0C0009279042AC9D801A757F822F063C1000861
:10C0D000B9C100087BC00008B9C10008CDC1000883
:10C0E0000FB3012F10D104F581770BEB0717FF7900
:10C0F000FB0709D417F07E0F06D1FF0915D1B768E9
:10C1000047453CBFA446B8460134082C06F110064A
:10C11000C0D100290CDABEF1000F20DABCF1000F0B
:10C12000ABDB614604E02146EEE7A646ECE721469C
:10C13000364E41F2180406EB01173851D2F89840F8
:10C140000134C2F8984041F21C02BC5001F58172E2
:10C15000170106EB0212F45100245460ABE771465C
:10C16000E6E715F0010213D0294BD3F82839002B4C
:10C1700083D0284F5D68284A002307EB4121A84758
:10C1800000283FF47AAF04EB06140223A37174E78E
:10C1900004EB0610019B90F807C0EF1067F3C71C73
:10C1A000032B80F807C02BD94FF6FF72934228BFAC
:10C1B000134604EB06129380B9F1000F06D004EB8E
:10C1C000011000F580501830FCF7AEF96A0741BF46
:10C1D00004EB0612D37943F00103D371EB0608D5C3
:10C1E00004EB0614E379C3F34502013262F346031C
:10C1F000E371084B03EB4123CAF8003001203DE70F
:10C200001346D6E7A85E0020C05E0020A84E00209E
:10C21000781A0020C04E0020399800087FB50F4DD5
:10C2200001AA0C4602A9FFF701FE05F58053029E04
:10C23000D3F800020322002303A93044FFF704FFD0
:10C24000012808D12978039B019A02290CBF23F801
:10C25000124043F8224004B070BD00BFA84E002039
:10C260002DE9F04FD1F8009085B01646074601AA97
:10C2700048460D4602A9FFF7D9FD374A0299D2F880
:10C28000003201EB0308019B013B9C19FFF78CFD79
:10C29000A4EB09040444A2F5805AB4FBF0F408EBC3
:10C2A00004092B68B342A9EB080103D3012005B0B0
:10C2B000BDE8F08FDDF804B00BEB0604E41AFFF7DD
:10C2C00073FD844228BF0446BBF1000F1AD1A0427F
:10C2D0008CBF0B220A220B46404603A9FFF7B4FE8F
:10C2E0000128E4D19AF800102B68039A022903F17F
:10C2F000010358460CD0A0420CD242F82030013045
:10C300000133F8E70B22E6E722F810300130013361
:10C31000A042F9D32B68A3EB0B032344012F2B601E
:10C3200014D1B34212D102290BBF04F1004404F12D
:10C33000804304F1FF3403F1FF330BBF4FF6FF736B
:10C340004FF0FF3122F8143042F82310002308F197
:10C3500001080193A5E700BFA85E00202DE9F04F7A
:10C3600085B00546FFF720FD0C461746814601AA19
:10C37000206802A9FFF75AFD6B1E012B66D9019BAD
:10C380004BB94E46DFF8C880012D8CBF0025012532
:10C39000A8F5805A1BE0FFF749FE02202BE0D8F8F1
:10C3A0007831C3B1D8F89411914214D1D8F8102241
:10C3B000013B500203EB4223B3FBF0F30B44B3FB0E
:10C3C000F6F206FB12320AB133449B1A236022684C
:10C3D000BA42E4D32BE0DDF808B0D8F8000200231D
:10C3E000092203A95844FFF72FFE012806D002288E
:10C3F000D3D00028EBD105B0BDE8F08F9AF800103B
:10C40000019A022907D00329C7D1039B53F8223090
:10C4100023F0704302E0039B33F81230D4F800C0DD
:10C42000B3FA83F35B09AB4204D16745E3D82760D5
:10C430000320E0E732440CEB060391452360E0D88B
:10C440000BF10103029300230193C0E7012699E752
:10C45000A85E002037B50446C0690D4610B901201A
:10C4600003B030BD0023032201A9FFF7EDFD012831
:10C47000F6D1B4F92030002B17DB019A012D4FEAD9
:10C48000431102EB431316D0022D12D0E268DA6199
:10C490002278032A04D100221A775A779A77DA771A
:10C4A000626A5A83110C9982D9E7FFF7BFFD022017
:10C4B000D6E7E5205054A268E9E738B5044694F879
:10C4C0003430052B2FD8DFE803F00727353C444DE7
:10C4D000022084F83400F2E7294DD5F8082204F14F
:10C4E000300102320120FFF739FF012805D0023860
:10C4F000C0B2012817D80520EBE7D5F81012E26882
:10C50000236BC5F8143202EB4122E260E26A236138
:10C51000002ADED16362DCE7206B4FF0FF31FFF7CA
:10C520007DFE012801D0002038BDE36A002BCFD169
:10C530000320CEE7D4E90B01FFF770FE0128F7D006
:10C54000F1E700212046FFF785FF0128EBD1042009
:10C55000BFE794F82830082B04BF002384F8283064
:10C560000120E1E794F82830082B04BF002384F869
:10C570002830034B012283F8B5210220D4E700BF05
:10C58000A85E00202DE9F341044694F83830032BCF
:10C590000ED8DFE803F00611767F032084F8380018
:10C5A000F3E72046FFF789FF0128F7D00228F4D0EF
:10C5B000002002B0BDE8F08123786568DFF8E480F0
:10C5C000022B1CBF374BD3F81832204618BF1D4032
:10C5D000FFF70EFCC5F34F252D1A0646ADB200231A
:10C5E000022201A93046FFF72FFDAF190128BFB283
:10C5F000DFD101984FF40072002158F0D3F8E369BD
:10C600002BB363681BBB019B4FF020322E211970A6
:10C61000C3F80120C3F80520A3F80920606A5883F5
:10C620004FEA104C102083F8201083F82110D872A4
:10C63000C3F82220C3F8262083F82A20E26BA3F84F
:10C6400014C022FA00F199865A8783F82B00D8F893
:10C6500010124B1E9F4208D24FF400712046FFF784
:10C6600055FC50F09BF90136B9E7C1EBC1514902C5
:10C6700001F500712046FFF749FC50F08FF90220C8
:10C680008CE7002384F82830236C0BB120469847B0
:10C6900001208EE7236C002084F8280003B198471E
:10C6A000022086E7A85E002010B5044694F83830D2
:10C6B000032B53D8DFE803F00631434D022384F8FF
:10C6C0003830F3E72649D1F894212261FFF7ECFBDB
:10C6D000E3680344E360FFF767FB1044C1F894018B
:10C6E000FFF7E2FBD1F878311B1AC1F87831FFF778
:10C6F000DBFBD1F87C311B1AC1F87C312263FFF7D8
:10C7000053FBE36A1044606313B962620123D6E706
:10C71000FFF74AFB121A2263F8E712480021FFF7DD
:10C7200099FE0128CAD0431EDBB2012B06D894F82B
:10C730002830062B04BF002384F8283010BD626B1C
:10C7400004F130010120FFF78BFD0128EBD1032319
:10C75000B5E700212046FFF77DFEE4E70220E2E78F
:10C76000A85E0020186000202DE9F74306460C461D
:10C770004FF6F77596F83C30042B73D8DFE803F0DA
:10C78000290736416300032086F83C00F2E73A4F60
:10C79000DFF8EC8007F580593B78306B032B4FD1E5
:10C7A00040454BD801A94EF03BF9012857D1306BD9
:10C7B0000021FFF733FD012851D1019B3363D9F8E4
:10C7C0001422013B934294BFC9F81432C9F81422D1
:10C7D000E2E7610001F0FE013046FFF73BFE012871
:10C7E0000CD1736B002B18BF0220CDE7726B06F1E2
:10C7F00030010020FFF734FD0128C4D002282ED1DB
:10C8000031E01E48F26AD0F89431C0F894219B1AA6
:10C81000D0F810225343D0F8782102EB4322C0F81D
:10C820007821D0F87C2102EB4322C0F87C21002142
:10C8300000F5B870FFF70EFE0128DFD10420A3E752
:10C8400083B2AB42ADE796F82830042B04BF002337
:10C8500086F82830B36B0BB130469847012003B0FF
:10C86000BDE8F083022096F82830042B04BF002393
:10C8700086F82830F3E700BFA84E0020A85E00200D
:10C88000F7FFFF0F70B50378027E023B012B0446D1
:10C890001CD8237E990622D42046FFF7D7FA237EA0
:10C8A0001A070AD51E4D95F89801C31F58425841E2
:10C8B00050F074F8002385F898310023237084F831
:10C8C0002830E36A53B1BDE87040184712F0060FF4
:10C8D000DFD00121FFF7BEFD0128DAD070BDE2698B
:10C8E0001049002318010858824211D10E4903F55E
:10C8F000817201EB0213DB79C3F34503012B0BD8E3
:10C90000002301EB0212D17963F34601D171C3E731
:10C910000133082BE6D1BFE7013B03F03F03F0E70B
:10C92000A85E0020C05E0020A84E002010B580B197
:10C93000027872B190F828206AB9D0E901249442B3
:10C940002CBF84608260032280F82820C162FFF738
:10C9500099FF012010BD0020FCE7B1F904300F2B36
:10C960002DE9F34104460D4616460BD14FF40071F4
:10C97000FFF7CCFA18B9002002B0BDE8F0814FF6FD
:10C98000FF73AB802046FFF733FA94F91B20531C4A
:10C99000074624D0244B41F2180103EB0210415802
:10C9A0008F4212D1183303EB42230193019A72B1E3
:10C9B000AB8801331BB202EB4312AB8020463260DE
:10C9C000FFF716FA28600120D6E7FFF72FFB204675
:10C9D000FFF776FA0028CED000233360F3E7204635
:10C9E000FFF76EFA80460028F1D1381E18BF0120EB
:10C9F0004FF0D4FF4346112201A93846FFF724FB2C
:10CA00000128E4D1094A019B9B1A48BF03F2FF1396
:10CA1000B3F5805F4FEA632203D3FFF707FB4FF0C4
:10CA2000FF32E276C2E700BFA84E0020C04E0020D1
:10CA30002DE9F0414FF0FF31304A314C0D460023D3
:10CA4000107804280ED103F5817004EB0010C07932
:10CA5000C60707D4681C52F80A0C01D0884201D2DC
:10CA600001461D460133082B02F11002E8D1002DCA
:10CA700041DB234CDFF8988005F5817704EB071341
:10CA80002E01998841B1D8F828392BB1A01941F26B
:10CA900018029B688058984741F218032644F058C2
:10CAA000D8F828396BB1174ED3F80C80164A0023FA
:10CAB00006EB4521C04720B1022810D00020BDE878
:10CAC000F081124BD3F89C2004EB0714013AC3F811
:10CAD0009C200322A271012283F8A020EEE706F633
:10CAE000E87604EB0714D6F89C30013BC6F89C307E
:10CAF0000123A371E2E70120E1E700BFCE5E002041
:10CB0000A84E0020C04E002091980008A85E00208A
:10CB1000781A002070B5124D124BC5F8B83840F2A3
:10CB20000112002385F81432A0F84421C0F85C31CA
:10CB300005F6B8020D23C0E95422044685F8C4184E
:10CB4000C0F8583100F5A27150F065F905F5FA7298
:10CB500020461F23BDE87040012150F0F5B900BF09
:10CB6000702B00205553425370B50B7813F06002C0
:10CB7000044638D0202A1ED14A78FE2A05D0FF2A42
:10CB80001DD050F047F8022016E04A88AAB9CE8896
:10CB9000012E12D11A0610D5314DD5F820329B69DD
:10CBA0009847C0B285F8C80838B1324605F6C801C2
:10CBB000204650F005F9002070BD2046E1E74A8884
:10CBC000002AFAD1C9880029F7D11B06F5D4244AD6
:10CBD00082F81412012182F8F0111F2302F5FA7273
:10CBE00050F0B2F9E7E74B780A2B24D00B2B25D075
:10CBF000012BE0D191F904600D79C068002E22DA92
:10CC000005F07F0150F0ECFB2946204650F010F86B
:10CC10002946134D02234022204650F033F895F860
:10CC2000F031022B12D1812120464FF0C1FF0023A9
:10CC300085F8F031BFE70B490122BAE7084B4A8873
:10CC400083F8C928B7E750F0B5FBDDE7002EB2DA6C
:10CC5000012BB0D001212046FFF75CFFABE700BFFE
:10CC6000702B00203934002010B50B4A92F8143292
:10CC7000022B044607D0033B012B02D80021FFF70B
:10CC800049FF002010BD92F8011250F07BF90028F6
:10CC9000F7DA01212046F2E7702B002070B5314C05
:10CCA00094F8146205461EB1012E50D0002070BDCC
:10CCB000D4F8F831C4F8BC38D4F8FC31C4F8C03822
:10CCC000B0F8B4331F2B0DD1D4F8F421264B9A427F
:10CCD00008D194F80112012904D894F80232013BDA
:10CCE0000F2B0AD9202105204FF0DAFD022384F80A
:10CCF000F0312846FCF734FBD8E750F043F9002820
:10CD0000F7DB94F81432013B022BCFD9B4F8CA18E0
:10CD100021B3D4F8FC3184F8C468994228BF19467D
:10CD2000D4F8C0385B1AC4F8C038042384F814322D
:10CD300040F20113A5F844310C4BC5E95616C5E97C
:10CD4000543305F5A271284650F065F8AEE794F823
:10CD5000011250F017F90028A8DA31462846FFF7EB
:10CD6000D9FEA3E7702B002055534243A63E002076
:10CD7000F0B59C0827010E46154600EB0414A042AE
:10CD800006F1100605F1100508D103F0030339443C
:10CD90003A4404EB83039C4223D1F0BD84469CEDCE
:10CDA000006A16ED045AD0ED016A56ED037A90ED53
:10CDB000027A56ED025A26EE056A66EEA76AD0EDB3
:10CDC000037A05ED046A16ED016A45ED036A27EE64
:10CDD000257A67EE867A103005ED027A45ED017A04
:10CDE000CDE7F4EC017AB1EC017A67EE877AE2ECF8
:10CDF000017AD0E74A09012350F8222001F01F01EF
:10CE00008B40134214BF01200020704710B54C091D
:10CE1000012250F8243001F01F018A40134340F8EA
:10CE2000243010BD80EA0120082241F2210103B222
:10CE3000002BB5BF81EA4303400098B280B2013AAB
:10CE4000F5D1704738B50C468D18AC4200D138BDCD
:10CE500014F8011BFFF7E6FFF7E74840082243B24A
:10CE6000002BBBBF5B0083F0D5034000D8B2A8BF46
:10CE7000C0B2013AF3D1704738B50C468D18AC42B8
:10CE800000D138BD14F8011BFFF7E7FFF7E770B5D5
:10CE9000066805460C460020B44203D3731C2B6081
:10CEA000307070BD14F8011BFFF7D7FFF4E7DFED1A
:10CEB0000A7AC0ED020A20EE270AB7EE007AC7EE22
:10CEC000007A00230360C0ED017A70EEA77A80EE4D
:10CED000A77A80ED037A7047DB0FC94090ED017AA5
:10CEE000D0ED007AC0ED020A30EE877AC0EE876A94
:10CEF00030EE677AE6EE877AB0EE670AC0ED007A28
:10CF00007047012303700023C364836403650364D3
:10CF100043644365836283657047DFED157A80ED76
:10CF2000010AF4EEE70AF1EE10FAC0ED020A80ED14
:10CF3000031AC0ED051A18DDB4EEE70AF1EE10FA97
:10CF400008DC9FED0C7A80ED047A80ED0F2AC0EDAD
:10CF50000E2AD6E781EE007AC0EE207AF0EE006A63
:10CF600077EE877A86EEA77AEDE700238360E8E71D
:10CF7000BD378635000000000F29A8BF0F21012909
:10CF800070B5B8BF01214C00013400260460A40034
:10CF900005468160466022463146803057F002FCEB
:10CFA0002246314605F58070BDE8704057F0FABB67
:10CFB000FDEEC07A17EE903A2033402B43D8DFEDD8
:10CFC000237A9FED237AB4EEE70AF1EE10FA28DC1B
:10CFD000DFED207A9FED1E7AB4EEE70AF1EE10FA4B
:10CFE00022D4DFED1D7AB4EEE70AF1EE10FA1EDD71
:10CFF00030EE670A37EEC00A60EE007ADFED176A9E
:10D000009FED177AA7EEA67ADFED166AE7EE876A3C
:10D010009FED157AA7EEA67A20EE276AA6EE070AFC
:10D02000704730EE470ACEE730EE070AD4E79FEDAF
:10D030000F7AB4EEC70AF1EE10FA44BF30EE270AB9
:10D0400037EE400AD8E79FED0A0A7047DB0F4940E8
:10D05000DB0FC940DB0F49C0DB0FC93F9A7C2E367E
:10D06000FAAF4FB93587083CA4AA2ABEDB0FC9BF67
:10D0700000000000DFED027A30EE270A98E700BFDB
:10D08000DB0FC93F10B51C46334BB3FBF2F399429B
:10D090009FED325AF0EE404AF7EE005A53D207EEB7
:10D0A000901A9FED2F7ADFED2F6AF8EE677AF8EE8F
:10D0B000002A67EE877A07EE102AB8EE477A27EE45
:10D0C000267AC5EE876A87EEA64AB0EE440AFFF7D5
:10D0D0006FFFF0EE403AB0EE440AFFF7CBFF74EE7C
:10D0E000A44A012C83EEA43A1CBF35EEC04AF6EEEA
:10D0F000006A33EE257A12BF64EE266AF0EE656AA6
:10D1000020EE224A86EE876AC4EE074A60EE227A53
:10D1100075EEC35AC7EE876AC5EE877AF0EE465AB7
:10D12000C0ED005AC0ED014A80ED026AC0ED036A0D
:10D13000C0ED047A80ED065A80ED055A80ED085A5C
:10D1400080ED075A10BDF0EE454AB0EE456AF0EEAC
:10D15000456AF0EE457AE3E720A1070000000000F1
:10D16000DB0FC940BD378635B0EEE06AF0EEC07A1D
:10D17000B4EEE76AF1EE10FAF0EE406A4BDCB5EE81
:10D18000400AF1EE10FA4BD0B4EEE76AF1EE10FA75
:10D19000F0EE675A41D5B0EE465A85EE257ADFEDBE
:10D1A000225A9FED225ADFED224AA7EE255ADFEDE3
:10D1B000215AE5EE075A9FED205AA5EE875ADFED7A
:10D1C0001F5AE5EE075A9FED1E5AE7EE054AB7EEE5
:10D1D000005AA4EE875AB1EE657A87EE050AB4EEDE
:10D1E000E76AF1EE10FA48BFDFED167AF5EEC00AF5
:10D1F00048BF37EEC00AF1EE10FA48BFDFED127AF1
:10D20000F5EEC06A48BF37EEC00AF1EE10FA48BF2B
:10D21000B1EE400A7047F0EE465AB0EE675ABCE7EE
:10D220009FED0A7ABBE700BF39094E3DE3B59EBECC
:10D2300069A2163E88FA16BE45FE7FBFA7DFA8B4D6
:10D2400099FB243FDB0FC93FDB0F49400000000082
:10D2500044F25063984203DDA0F50C40A0387047BB
:10D26000034B9842BCBF00F50C40A030704700BF94
:10D27000B0B9FFFF48F69F43984203DDA0F50C408C
:10D28000A03870470028BCBF00F50C40A0307047A4
:10D2900091ED005A08B5B0EE450AFFF7EBFEF0EE4F
:10D2A000405AB0EE450AFFF783FE91ED015AF0EEC9
:10D2B000404AB0EE450AFFF7DDFEF0EE403AB0EE30
:10D2C000450AFFF775FE91ED023AB0EE405AB0EE16
:10D2D000430AFFF7CFFEB0EE404AB0EE430AFFF735
:10D2E00067FE25EE806A63EEC07A24EE847AC0ED94
:10D2F000017AF0EE467AE5EE077A25EE843A64EE9E
:10D30000806AC0ED037AF0EE437AE5EE667AA5EE28
:10D31000067AE5EE436A23EE844A64EEE34A65EE5C
:10D32000A35A80ED004A80ED025AC0ED047AC0EDA8
:10D33000054AC0ED066A80ED077AC0ED085A08BDBF
:10D34000034600F1400100221A615A619A61DA61D4
:10D3500010338B42F8D11022002157F023BA91EDFF
:10D36000007AD0ED047AE7EE077AC0ED047AD1EDC9
:10D37000006A91ED017AD0ED057AE6EE877AC0ED8C
:10D38000057AD1ED006A91ED027AD0ED067AE6EEEB
:10D39000877AC0ED067A91ED007AD0ED077A77EEC4
:10D3A000877AC0ED077AD1ED016A91ED007AD0ED70
:10D3B000087AE6EE877AC0ED087A91ED017AD0ED31
:10D3C000097AE7EE077AC0ED097AD1ED016A91EDAD
:10D3D000027AD0ED0A7AE6EE877AC0ED0A7A91ED0C
:10D3E000017AD0ED0B7A77EE877AC0ED0B7A91ED6A
:10D3F000007AD1ED026AD0ED0C7AE6EE877AC0EDC4
:10D400000C7AD1ED026A91ED017AD0ED0D7AE6EE5B
:10D41000877AC0ED0D7A91ED027AD0ED0E7AE7EEC3
:10D42000077AC0ED0E7A91ED027AD0ED0F7A77EEA1
:10D43000877AC0ED0F7A91ED007AD0ED107A77EE11
:10D44000877AC0ED107A91ED017AD0ED117A77EEFE
:10D45000877AC0ED117A91ED027AD0ED127A77EEEB
:10D46000877AB7EE007AC0ED127AD0ED137A77EEB4
:10D47000877AC0ED137AD1ED017AD1ED006A91ED92
:10D48000027A67EEA77AE6EEA67AE7EE077A90EDE3
:10D49000007AA6EEA77A80ED007AD1ED016A90EDD0
:10D4A000017AA6EEA77A80ED017AD1ED026A90EDBD
:10D4B000027AA6EEA77A80ED027A90ED037A77EEF3
:10D4C000277AC0ED037A70472DE9F043034685B013
:10D4D00000F11007054600261C46AC4612E0F8ECA9
:10D4E000016A1EED047AD4ED007AE6EEC77AC4ED47
:10D4F000007A98450EF1100EF1D10434BC420CF1C3
:10D50000040C03D0A7F11008E646F2E701361C46EA
:10D51000B646BEF1040F1DD000EB0E1CA84604F168
:10D52000100907E0FCEC016A18ED047AE6EEC77A10
:10D53000C4ED047ACC45D4ED047A08F11008F1D199
:10D54000D3ED006A87EEA67A0EF1010E84ED047A1F
:10D550006446DEE7042E03F1140305F1040507F128
:10D560001007B9D1002300930193029303936C46F3
:10D5700000231427F2EC017A00EB031507FB030CE0
:10D580006E466545C4ED007A1FD10133042B04F1CA
:10D590000404EFD104AD103100F1400275ED017AC1
:10D5A00000EB03170E461446BC4241ED017A13D13D
:10D5B00052ED016A87EEA67A013BA2F1140221ED39
:10D5C000017AEBD105B0BDE8F083F5EC016AB6EC69
:10D5D000017AE6EEC77AD4E7F4EC016AB6EC017A98
:10D5E000E6EEC77AE0E71FB50C4602466946103002
:10D5F000FFF76AFFDDED007AB6EE007A67EE877A14
:10D600000120C4ED007ADDED017A67EE877AC4ED82
:10D61000017ADDED027A67EE877AC4ED027A04B012
:10D6200010BDF8B510EE100A10EE904A50F08CFCC8
:10D63000064620460F4650F087FC324604460D460B
:10D640003B463046394650F0D7FC2246064601F1AB
:10D6500000472B462046294650F0CEFC02460B469A
:10D6600050F014FB02460B463046394650F0EEFDB2
:10D6700041EC100B51F024FE51EC100B50F0B4FFB4
:10D6800000EE100AF8BDB5EEC00AF1EE10FA08B5CA
:10D6900006DB51F03DFFB4EE400AF1EE10FA01D77F
:10D6A0009FED010A08BD00BF000000002DE9F04118
:10D6B000044626461C3004F1640250ED017AB1ECB8
:10D6C000010A77EE807A40ED017AFBF78FF9183086
:10D6D0009042F2D12C4F6268D7F8943125699B1A99
:10D6E000A2680135934225612BD904F13008F36A11
:10D6F000012BC3BF03F1FF3307EE903A96ED0A7A90
:10D700009FED220AC4BFF8EEE77A87EE270AFFF7FB
:10D71000BAFF4645D4ED057A15D0F4EEC07AF1EEA5
:10D7200010FA06F11806E2D5237B4BBBD7F89421FB
:10D73000626000222361A261E36222636364A264E7
:10D74000E365BDE8F081F4EEC07AF1EE10FAEBD4B7
:10D7500007EE905AD4ED066AF8EE677A022386EE59
:10D76000A77AD4ED0C6A84ED067A86EEA77AD4ED1A
:10D77000126A84ED0C7A86EEA77A84ED127A00E0C4
:10D7800003232370DDE700BF702B002000000000A2
:10D7900070B52DED028B0378012B04463CD1056951
:10D7A000254E25B9426812B9D6F89421426094ED0D
:10D7B000068A30EE088A013584ED068A256104F177
:10D7C0001C00FBF713F96268D6F894319B1AA26823
:10D7D000934221D9E36A012BC3BF03F1FF3307EE64
:10D7E000903A94ED0A7A9FED150AC4BFF8EEE77AF5
:10D7F00087EE270AFFF747FFD4ED057AF4EEC07AEB
:10D80000F1EE10FA0ED5237B4BB9D6F89421626065
:10D8100000222361A261E362BDEC028B70BD032391
:10D820002370F9E707EE905AF8EE677A022388EE44
:10D83000277A84ED067AF3E7702B002000000000C1
:10D8400008B52DED028BF0EEC08AB0EE408AB7EE3F
:10D85000000A30EE680AFFF716FF9FED0E7ADFED43
:10D860000E7AE8EE877A9FED0D7AA7EEA87ADFEDC3
:10D870000C7AE7EE287AB5EEC08ABDEC028BF1EEA9
:10D8800010FA20EE270A44BFDFED067A37EEC00A11
:10D8900008BD00BF306E99BC2716983D843459BE30
:10D8A000A40DC93FDB0F494060EEA00AE0EE000A7C
:10D8B000B0EE600AE7E660EEA00AE0EE000AE1EEF4
:10D8C000010AB0EE600ADEE62DE9F74F90469DF8BA
:10D8D0003020002A0CBF4FF0200A4FF0300A0D9A7A
:10D8E0001C1E05460F46BABF64424FF0010B4FF0B5
:10D8F000000B12F8011B01B14CB9BBF1000F2DD187
:10D90000264636B9A1464FF0FF340D9E0FE0013C8C
:10D91000EFE7BD4202D251462846C047013EF0E73C
:10D92000BD4203D201922846C047019A16463246AC
:10D9300012F8011B0029F3D10D9BA9EB03094E44FA
:10D94000BBF1000F06D0A146B9F1000F09DC002C95
:10D95000A8BF3619304603B0BDE8F08F4FF000097C
:10D96000D3E7BD4202D251462846C04709F1FF39EC
:10D97000EAE70FB437B50C4D06ABD5F8D01853F81D
:10D98000042BD5F8CC0801934FF060FF0446D5F87E
:10D99000240203F02BFE0028F9D0204603B0BDE896
:10D9A000304004B0704700BF702B00200EB403B5A8
:10D9B00003AB084953F8042BCDE9003001A84FF020
:10D9C00045FF019B00221A7002B05DF804EB03B022
:10D9D000704700BF418A00080CB430B52C4CD4F815
:10D9E000D438A5B01BB9D4F8D838002B39D094F866
:10D9F000DC38994206D9012303FA00F0D4F8E03864
:10DA000018422ED0D4F894114FF47A7304A8B1FBC5
:10DA1000F3F203FB12131F49FFF7C8FF04AB0344E3
:10DA2000289A1D490393054629AB03A802934FF09A
:10DA30000DFF039B591C03910A211970039B591C6C
:10DA40000391002119700246D4F8D40890B10368FC
:10DA50005B6A03B19847D4F8D45804AC14F8011B9E
:10DA600021B925B0BDE8304002B07047284603F028
:10DA700093FDF3E7D4F8D838002BF2D015440222F6
:10DA8000009204A9AA18FD2028F018FBE9E700BFBE
:10DA9000702B00208F02070865870008174A38B5E9
:10DAA000D2F8E458033005EB9003B3F5007F19D8A2
:10DAB00002F6E804C2F8E438114A02EB810120F0D2
:10DAC000030051F8102CC3F50073024441F8102CE8
:10DAD0009B000C4A0421002004EB8504FFF77CFF27
:10DAE000204638BD0021084A0846FFF775FF074A5F
:10DAF000136843F0007313600024F1E7702B0020DB
:10DB0000683C00209B020708BF02070888690120C3
:10DB10002DE9F0470368214F0546002457F83420CB
:10DB2000934213D11E4E06EB84094FEA8408D9F8BC
:10DB300028A2BAF1000F21D107216420FFF7AEFF20
:10DB40000146C9F8280260B9164A04E001340E2CD7
:10DB5000E4D1154A00210520FFF73EFF0020BDE873
:10DB6000F0876422514656F01DFED9F8283207EBA3
:10DB7000C407C3E90073DB615B63DB644644687917
:10DB8000D6F82832182404FB003200211046C2E9DE
:10DB90000311956011750430E1E700BF6C5A060867
:10DBA000702B0020F2020708CD02070803685A1CF8
:10DBB000026019700368090A5A1C026019707047E4
:10DBC00003685A1C0260197003685A1C02600A0A32
:10DBD0001A7003685A1C02600A0C1A700368090E56
:10DBE0005A1C02601970704738B504460068154623
:10DBF00055F0B6FC23682B44236038BD03685A1CDB
:10DC000002601878704703685A1C02601A4612F8BE
:10DC1000021B0260587841EA00207047026810B584
:10DC2000531C0360134613F8021B0360D31C547883
:10DC3000036093781B0443EA04230B43111D016026
:10DC4000D07843EA006010BDD1E900329A4206D094
:10DC50005A1C0A6008B11B7803700120704700202D
:10DC60007047D1E900239B1A012B10B504460846E2
:10DC700004DDFFF7C8FF2080012010BD0020FCE775
:10DC8000A0F16103192B98BF2038704738B50546BD
:10DC9000002428464FF0ECFFA04200D838BD2B5D91
:10DCA000A3F16102192A9CBF203B2B550134F0E7F8
:10DCB00030B50A440546914201D1002011E015F823
:10DCC000013B11F8014BA3F141001928A4F14100D7
:10DCD00098BF2033192898BF2034181B01D1002C7D
:10DCE000E9D130BD6FF00042E2E710B503888278D9
:10DCF00003F003010C24013A04FB01221149847949
:10DD000001EB4202A3F5FA63B2F8F22040F2B551FA
:10DD10009B0801FB0323C278013A134402791821BE
:10DD200001FB0323427900893C2101FB0322064BBE
:10DD3000234401FB02334FF47A720021C3FB02013A
:10DD400010BD00BF005A060880436D38F8B519466B
:10DD50000446002310464FF47A7250F0A3FD244B82
:10DD60003C25034493FBF5F005FB103390FBF5F1E4
:10DD700005FB110060711820A37191FBF0F300FB0B
:10DD8000131140F2B550217193FBF0F100FB1133F8
:10DD9000B3F5896F4FEA810526DA40F2DA218B422A
:10DDA00024DCB3F5B77FB4BF00200120114E182149
:10DDB00001FB00660B2136F811709F4201DD01392D
:10DDC000F9D105F5FA65054425804D1CA5700C2593
:10DDD00005FB00110848228100EB41010133B1F835
:10DDE000F2105B1AE370F8BD0320DFE70220DDE7E5
:10DDF00080BC92C7F25A0608005A0608F0B5294DB1
:10DE000007460E460FCD8DB06C460FC40FCD0FC424
:10DE100095E80F0084E80F0017F003033FD1642159
:10DE200097FBF1F201FB127242B94FF4C87297FBF3
:10DE3000F2F302FB1373003B18BF01237A1EC3F1F8
:10DE40001D03002A019340F26D13114607FB03F3F3
:10DE5000B8BFB91C03EBA1036FF0630192FBF1F1B2
:10DE60000B444FF4C87192FBF1F21344253307249D
:10DE700093FBF4F2C2EBC2029B1A013E6D460021F5
:10DE800055F8040F01310344B14293FBF4F2C2EBA5
:10DE9000C202A3EB0203F3D1C01A0DB0F0BD0123FF
:10DEA000CCE700BF545B0608084BD3E91E1251EAC9
:10DEB000020309D0064BD3F894315B1842F10002FB
:10DEC000C0E900320120704700207047683C002004
:10DED000702B002037B505466846FFF7E5FF04467E
:10DEE00038B1DDE900232846FFF730FF204603B0B4
:10DEF00030BD40F2011328806B80A880A871288172
:10DF0000F4E737B50546FFF7E5FF044650B1074B88
:10DF10000DF10602B3F88030ADF8063029462846E8
:10DF20004CF0EEFC204603B030BD00BF683C002042
:10DF30002DE9F041044686B094F83030042B13D814
:10DF4000DFE813F0150005005D00E9003601DFF899
:10DF5000688204F11C0701AA39464046FEF7FDFC21
:10DF600001280CD002282AD006B0BDE8F0819248E2
:10DF70004CF044FF4FF6FF73238401233CE0019DE6
:10DF80000DB12B7863B98C48FDF760FF237EDD0669
:10DF900018D54CF033FF4FF6FF73238402232BE098
:10DFA000EE7A3007D7D40B2204F13101284655F020
:10DFB00053FA0028CFD1637E7340D90604D57E483A
:10DFC000FDF744FF042317E0AA8A6B8B43EA024360
:10DFD0007A4A6362D2F81022EB69A3605202B3FB63
:10DFE000F2F102FB113109B113445B1A7248E3608C
:10DFF0006676FDF72BFF032384F830309CE76F4EE5
:10E0000096F8E031002BAFD104F11C0806F5DC775F
:10E0100001AA41463846FEF7A0FC012859D1019DCE
:10E02000002D38D02B78E52B01D0002BF0D1644B9C
:10E03000EB1A48BF03F2FF13B3F5805F4FEA63208A
:10E0400003D3FDF7F3FF4FF0FF305E4901EB001003
:10E05000FAF76AFA01F5D070FDF7F8FE20220021E8
:10E06000284656F09FFBD4F831302B60D4F8353079
:10E070006B60B4F839302B8194F83B30AB72637E1F
:10E08000EB7203A8FFF73DFF38BB6FF07E032B74E4
:10E0900047236B743AE096F8B831022B92D096F889
:10E0A000E031002B8ED10922C6E97D3386F8E021CC
:10E0B00086F8F031D6F8CC2186F8EC313E48D6F817
:10E0C0001432C6F8E421C6F8E831FEF75BFA0128FD
:10E0D0009ED002283FF476AF46E79DF80E209DF8CB
:10E0E0000F3043EA4213BDF80C20A2F2BC7243EA9F
:10E0F00042232B829DF811309DF812205B0143EAE8
:10E1000052039DF8102043EAC223EB812B8A2B8314
:10E11000EB89EB826FE7237E9A0608D5E06900233E
:10E12000112202A9FDF790FF01287FF41DAF2046C0
:10E130004CF064FE2269237E9AB91B0708D51F4B59
:10E1400093F89821002A7FF40FAF072283F89821D3
:10E15000002384F82830E36A204606B0BDE8F04189
:10E16000184703F0F70213F0040322760AD0E26A9C
:10E17000A1680023204684F8283006B0BDE8F041AD
:10E18000FDF708BF122AE3D1E26AA263626A84F84B
:10E190003C3004212046C4E90B22C4E9023384F850
:10E1A00028106363636206B0BDE8F0414CF026BE00
:10E1B0000020E36A2070D0E760600020A85E0020A5
:10E1C000C04E0020C05E00202DE9F34103780446D4
:10E1D000002B76D090F82830013B082B71D8DFE86F
:10E1E00003F00509475B4C6170666B0002B0BDE847
:10E1F000F0419DE6344B4568D3F81072D3F81832DD
:10E200007F021D40216B2046FDF75AFE05EB0108F9
:10E210004745064626D880B1D4E901329A422CBF40
:10E22000A260A360002384F82830E36A002B48D062
:10E23000204602B0BDE8F04118472169207E01AABE
:10E240004EF08CFC01283CD123696361019B236162
:10E2500063683B445B1B6360236BDB1B2B442363C2
:10E260003546CFE70028D7D163680B446360D3E716
:10E2700002B0BDE8F041FEF705BB0121FEF774FADC
:10E2800001281ED1216C0023204684F8283002B0DA
:10E29000BDE8F041FEF74ABB002102B0BDE8F04105
:10E2A000FEF762BA02B0BDE8F041FEF7FDB902B078
:10E2B000BDE8F041FEF701B902B0BDE8F041FEF75C
:10E2C00061B902B0BDE8F081A85E0020F0B501247C
:10E2D000B0FBF4F58D4203D200261CB91C70F0BDD2
:10E2E0004C43F5E7B0FBF4F5B4FBF1F704FB150084
:10E2F0002EB9002D03DC8C420CD33C46EDE7092DF2
:10E3000008DD002A0CBF572437242C4403F8014BA6
:10E310000136F2E73024F8E703463038C2B2092A62
:10E320000FD9A3F16102052A02D8A3F15700704763
:10E33000A3F14102052A02D8A3F1370070474FF03C
:10E34000FF30704770B50446944208461546B4FB4A
:10E35000F2F602D33046FFF7F5FF05FB1644024BF9
:10E360001B5D00F8013B70BD17030708B5EEC00A3E
:10E37000DFED2D7AF1EE10FACCBF30EE270A30EE49
:10E38000670ADFED2A7A20EE270A30B5FDEEC07A63
:10E3900087B017EE904A054684EAE470002303A98B
:10E3A000A0EBE470CDE9003302934CF017FD002C94
:10E3B000B4BF2D23202303A88DF800304FF058FC64
:10E3C000012822D130238DF8013043F23003ADF81B
:10E3D000023003A9684657F09DF868464FF048FCA4
:10E3E000C41EE4B222466946284655F0B9F8002317
:10E3F0002B550F49284657F08DF80DEB04012846A0
:10E4000057F088F8284607B030BD022805D13023E0
:10E410008DF801308DF80230DBE7032804BF30238C
:10E420008DF80130D5E700BF6F12033A00007A443F
:10E43000483A070830B50278202A034600F1010067
:10E44000F9D0092AF7D02D2A4BD10346BFEE000A96
:10E450009FED3C7A1A46F2EE046A134612F8010B5D
:10E46000A0F13001CCB2092C41D92E280BD1F2EE0B
:10E47000046A1146B0EE666A0B4611F8012B303A79
:10E48000D0B209283CD91A7802F0DF02452A53D1CC
:10E490005A782D2A3FD102330120013B00220A2560
:10E4A00013F8011F3039CCB2092C3AD9B2F59A7F52
:10E4B0001346DFED256A28BF4FF49A731A46F7EE2C
:10E4C000007A072A30D8DA086FF0070101FB02331F
:10E4D000F2EE046A63BB88B3C7EE276A20EE260A11
:10E4E00030BD2B2A08BF0346B7EE000AB0E707EE9F
:10E4F000901AF8EEE77AE7EE267AB0EE677AACE7A4
:10E5000007EE902AF8EEE77AC7EEA65A66EE866A1C
:10E5100037EE257AB0E72B2A14BF013302330020EF
:10E52000BBE705FB0212BBE767EEA67A083AC8E72D
:10E5300067EEA67A013BCDE7F7EE007A67EE276A31
:10E54000CCE700BF0000000020BCBE4C70B5034605
:10E5500010F8012B202AFAD0092AF8D02D2A0ABF58
:10E56000034601254FF0FF35591E00240A2611F8F5
:10E57000010FFFF7D1FE092802D905FB04F070BD99
:10E5800006FB0404F3E710B50023802804D8934267
:10E590000AD2C854581C10BD934205D060F07F04C5
:10E5A000CC54C0090133F0E74FF0FF30F3E7F8B582
:10E5B000144D2B787E2B23D1012229460020FEF713
:10E5C00041FC114F6C1C228862B1A31DBB4217D2C3
:10E5D000A618BE4214D2052A12D92146FEF732FCF3
:10E5E0003446F0E702222146FEF72CFC6388074AF6
:10E5F000C31A0434641B5842A2F81A425841F8BDA9
:10E600000020FCE70040000800800008683C002073
:10E610002DE9F04F724BDFF8DCB18FB0A3EB0B02AA
:10E62000CDE901234FF00308102200210AA856F07B
:10E63000B9F8019B0993029B08936A4BCDF81CB073
:10E640001A69002ABFBF684A5A6002F188325A60CC
:10E650000124F322DA604FF000097E23224604A948
:10E6600007A88DF83440CDF830908DF81030FAF7C7
:10E6700099FA4845C0F2A180224604A94846FEF70F
:10E68000E1FB5A4CADF81200594B9C423CD300249C
:10E69000022205A907A8ADF81440FAF783FAA042B0
:10E6A000C0F28B80BDF81200022205A9FEF7CAFB5A
:10E6B0000222ADF812000DF1120107A8FAF772FA62
:10E6C000A0427ADB0B9880B1079B089A03449342DF
:10E6D00073D80AABC0F104022146184456F062F820
:10E6E0000AA907A8FAF7BAF90C900C9B002B64DB77
:10E6F0009DF8342022B13B490A6942F000420A6188
:10E70000B3FA83F35B0959E062888DF81990C2F37C
:10E710000B06B31DADF814302388C3F30B011B0B9C
:10E720008DF818301304ADF816101ED4062205A972
:10E7300007A8FAF737FA00283FDBBDF812000622D7
:10E7400005A9FEF77FFB676805463246394607A8EC
:10E75000FAF728FA002830DB324639462846FEF719
:10E7600071FBADF8120014348EE700273D460135E9
:10E77000EDB2062205A907A88DF81950FAF712FA8A
:10E7800000281ADBBDF81200062205A9FEF75AFB85
:10E79000616882463944324607A80391FAF702FAC3
:10E7A00000280ADB039932465046FEF74BFB032D47
:10E7B000ADF812003744DAD1D5E70023B8F10108EB
:10E7C00008D0002B3FF430AFFFF7F1FE20B10FB0BF
:10E7D000BDE8F08F002BF7D1052005F089FA00BFC6
:10E7E00000800008003C024023016745A86207083A
:10E7F000F867070800400008034AD2F81C3223EAF1
:10E800000003C2F81C327047683C002003460649EA
:10E810000648884201D3002070470288C2F30B02E9
:10E820009342F9D01430F4E7F8670708A8620708A4
:10E8300070B544880B460546C4F30B0422460021FC
:10E84000184655F0AFFF2969084A9142034607D39D
:10E85000074A914205D22246BDE8704054F080BE7E
:10E8600019B1BDE870401846084770BDF867070841
:10E87000FF6C070810B4B0F902404288002C0B4628
:10E8800041685DF8044BBEBFC2F30B02DBB203FB71
:10E890000211CDE730B5094B094CA34200D330BD7E
:10E8A000B3F902205988002A06DA5A68DD68C1F3F4
:10E8B0000B0100FB01222A601433EEE7A86207086F
:10E8C000F867070830B502460144002012F8015BE2
:10E8D000082480EA050343F3000323F0730383EA6B
:10E8E0005003D8B2631E13F0FF044FEA5505F0D170
:10E8F0009142EBD130BD2DE9F04F87B0CDE9032334
:10E900000025804601910095039B4046EC0003EBF7
:10E91000C50AFBF707F9002800F0978000220121C3
:10E920004046FBF7E9F80290002800F08E8098F846
:10E9300004309A0706D4029A049B10461D7007B053
:10E94000BDE8F08FF0214046FBF7F6F800287CD0B8
:10E95000039BA4F108024FF0000B01261344344638
:10E960005F460593019BB3B3082C34D804F1FF39FB
:10E9700043FA09F909F0010949464046FBF793F8C3
:10E98000002862D0002201214046FBF7B5F802467C
:10E9900000285AD098F8041001F0600CBCF1600F08
:10E9A0004FEAD11037D0019B1BB1082C01D881450B
:10E9B000C1D120B31AF8071031437600013416F0A4
:10E9C000FF060AF80710E4B2CCD10137FFB2082FD6
:10E9D00021D00126C6E75DB1009BA34208D9059B63
:10E9E000DA5D164214BF4FF001094FF00009C3E78A
:10E9F000009B1B1BD3F1000949EB0309BCE7880905
:10EA000040EA511111F0010F1AF8071008BFA34690
:10EA100021EA0601D1E7402C11D907215046029284
:10EA2000FFF750FF9AF80740029A844207D1013558
:10EA3000EDB2BBF1000F3FF47FAFCDF800B0049B07
:10EA40001B78AB423FF660AF76E7002274E700BF69
:10EA500090F83C20034602F0FF0012B1002283F838
:10EA60003C2070474FF48053838170474FF400631C
:10EA7000838170474FF40063838170474FF40063D4
:10EA8000838170474FF40063838170474FF40063C4
:10EA9000838170474FF400638381704710B5064A45
:10EAA0000423002152F8044B844208BF42F8041C9E
:10EAB000013BF7D110BD00BFD0600020324BF0B554
:10EAC000188ADC8BB3F92850B3F92270B3F918E037
:10EAD000B3F93060001B9C8B6043B3F9264005EB13
:10EAE000E035E40294FBF5F404EBE034A4F57A603D
:10EAF000B3F91650DC6200FB00FC4FEA2C3C4543A6
:10EB00000CFB07F700FB0EFEED12B3F9200005EB3E
:10EB1000E725B3F914700CFB00F0001405EB870532
:10EB2000B3F81AC05B6B00EB6E30B54002300235B3
:10EB3000A3EBA50580104CF2503300F500403341A3
:10EB40006B430CFB00F04FEAD03055BF5B00B3FBCA
:10EB5000F0F3B3FBF0F35B0071B1181240F6DE3551
:10EB600040436843094D00145D4300EB254000F627
:10EB7000CF6003EB20130B6022B10A235C430834FF
:10EB8000241114600120F0BDD060002043E3FFFF9A
:10EB900001207047012070472DE9F74F604E9046E5
:10EBA000B38FB26BB6F94CC0B6F94A70B6F948B03B
:10EBB000C3EB22155B00C3EBE203B6F93E206D43C5
:10EBC0005343B6F940202D135543AD1305EBE32510
:10EBD000B36D0093A5F5FA30B6F9463075658946F0
:10EBE00080FB001EDA1703FB0EF401FB0244A3FBBB
:10EBF00001321444B6F9442082FB00A21B0A12031E
:10EC000043EA046342EA1A524FEA0A3A13EB0A0350
:10EC100042EB2422B6F842A002F500420192A3FB87
:10EC20000A23019A0AFB023A4FEAEA734FEA6A02A0
:10EC300053EA6A0A4FF000045ED087FB00704FEA87
:10EC4000EC7A0CFB0EFE400401FB0AEE40EAD730E2
:10EC5000ACFB011C7F047F180099F4444CEB0000CE
:10EC6000C1F5801C0CF00041E71941EA5C014FEA54
:10EC7000CC7CBCEB070C40F6354400EBCB0061EBE1
:10EC80000001ACFB040C04FB01C14FF00BFE8446F9
:10EC90000746430BB6F952004A1343EAC14300FB4F
:10ECA00002FEC41703FB04EEA0FB03407044624362
:10ECB00003FB0022A4FB03431A44B6F95030640E50
:10ECC00044EAC2144FEAE37E03FB01F0E4190EFBB1
:10ECD0000C00A3FB0C3738444FEAD34343EA4033DC
:10ECE00041EB6262E41842EBE042B6F94E30240A8E
:10ECF00044EA026404EB0314B9F1000F02D0240AC1
:10ED0000C9F80040B8F1000F05D005EB8505803546
:10ED10002D12C8F80050012003B0BDE8F08F00BFED
:10ED2000D060002031B10A4BD3ED1E7AFDEEE77AB8
:10ED3000C1ED007A52B1064B9FED067AD3ED1F7AF2
:10ED400067EE877AFDEEE77AC2ED007A0120704720
:10ED5000D06000200000C8422DE9F74FCDE9001235
:10ED6000574AB2F88E30D2F88010B2F88A60B2F802
:10ED700090701B02C91AB2F88C306EEB0E0EA3FB1A
:10ED8000010403FB0E44B2F88830C00940EA446035
:10ED90001B04C018A6FB013506FB0E55B2F88660B1
:10EDA0004FEA132343EA05634FEAC6364FEAE414F9
:10EDB00044F100049B19A7FB012607FB0E664FEAEE
:10EDC000D25242EA46224FEA252545F10005F615C2
:10EDD00012F5FA6C46F1000BBCF5FA6F7BF10007F7
:10EDE00050DA02FB06F8A2FB02794FF0050A09EBA4
:10EDF0004809A7FB0A780AFB09884FEA570949EA3C
:10EE0000C879BF08B0EB090947EA887764EB680462
:10EE1000DF1B3B462B4F65EBA805BC454FF0FF378A
:10EE20007BEB0707484622DA40F6AC57D21946F189
:10EE300000065643A2FB027202EB46024FEAC208EA
:10EE4000FE00BE1B48EA577862EB0808361844EB10
:10EE500008044FF00B083046A7FB087608FB026257
:10EE60007F0847EAC277DF1B3B4665EB620501FB83
:10EE70000EFEA1FB011202EB4E02C90F41EA420154
:10EE8000BCEB010C009A9AB10D4AD2F89410A1FB88
:10EE9000033201FB05225B0D43EAC2231B1A4FEA32
:10EEA000625262EB0402DB0B43EA4243009A1360B6
:10EEB000019B0BB1C3F800C0012003B0BDE8F08F87
:10EEC000D060002024FAFFFF01207047B0F9003025
:10EED0005943084B994208DBB1F5000F07DA0029C6
:10EEE000B8BFFF31081200B270470348FBE747F68E
:10EEF000FF70F8E701FF7FFF0080FFFF064B002255
:10EF0000C3F89820C3F89C20C3F8A0200022C3F8BF
:10EF1000A4200120704700BFD0600020104B1A6869
:10EF2000104BD3F8A410521AFA2A16D8D3ED267A29
:10EF3000FDEEE77A17EE902AD3ED277AC286FDEE32
:10EF4000E77A17EE902AD3ED287A0287FDEEE77A6A
:10EF500017EE903A4387012070470020704700BFAA
:10EF6000042D0020D060002090F85F3230B53BB90E
:10EF700090F85D1290F85E320124DAB2914200D826
:10EF800030BDB0F8665204FA03F22A43A0F86622B4
:10EF90000133F2E74379024613F0010006D0D2E9CB
:10EFA0000731D2685B1A013A03EA020070474379DD
:10EFB000024613F0020007D0936A516A1269013BBE
:10EFC0005B1A013A03EA0200704710B5437913F067
:10EFD000010304460ED0FFF7DDFF034650B1226A5D
:10EFE0006369E1689B5C0132B2FBF1F001FB102226
:10EFF000DBB22262184610BD43799B070AD5436AEB
:10F000008269D154436A02690133B3FBF2F102FB16
:10F010001133436270474171704781717047D0E985
:10F020000920131A584258417047024BD3F8A830B0
:10F030005B681847D0600020024BD3F8A830083036
:10F040009B681847D060002001207047012070475E
:10F0500001207047012070470120704731B10C4BEF
:10F06000D3ED2B7AF8EEE77AC1ED007A7AB1084B4E
:10F07000DFED086AD3F8B030A3F5D543333B07EE94
:10F08000903AF8EEE77A87EEA67A82ED007A70473A
:10F09000D06000200000C842012070470120704766
:10F0A000094A30B505460A2400201368AB4205D151
:10F0B000D3688B421EBF431CD160D8B2013C02F121
:10F0C0001402F2D130BD00BFBC0500207047054BD3
:10F0D00040F2FF7203EBC0039142A8BF1146998032
:10F0E000704700BF383D0020112807D8044B03EBC0
:10F0F0008003D3F8B4300BB19B681960704700BF30
:10F10000D060002008B5FFF7EFFFBDE8084021F010
:10F1100007B80C4A13787BB10B4B93F8FC1059B12C
:10F1200093F8FD1059B150680021FA2883F8FD10BA
:10F13000A8BF4FF0FF3070476FF0010070476FF0CD
:10F1400002007047F0100020D06000200B4B93F8B5
:10F15000FE206AB193F8FF206AB1002283F8FF20F5
:10F16000074B9868B0F5967FA8BF4FF0FF30704707
:10F170006FF0010070476FF002007047D060002010
:10F18000F0100020024BD3F800315B68184700BF35
:10F19000D0600020024BD3F800319B68184700BFB5
:10F1A000D0600020024BD3F80031DB68184700BF65
:10F1B000D0600020014BD868704700BFF0100020DD
:10F1C000044B93F8043113B1034B186970476FF087
:10F1D00001007047D0600020F0100020014BD3F8F0
:10F1E00008017047D06000202DE9F041062592F912
:10F1F000007086B06B43144612F80580A0EB080E31
:10F20000A0EB070CBEF1000FB8BFCEF1000EBCF1B1
:10F21000000FB8BFCCF1000CE645B8BF541905F19A
:10F220000605B8BF4FFA88F7AB421646E4D11A4438
:10F2300033786588BB420BD173884D1BCB1A002DE8
:10F24000B8BF6D42002BB8BF5B429D42C8BF344679
:10F250000636B242ECD16379049323790393638831
:10F2600002932378054ACDE90013034603210120C8
:10F27000FEF7B2FB204606B0BDE8F081D0030708D8
:10F280004B1EDBB2062B9CBF1C4AD25C1C4BF0B55C
:10F29000A3F1580488BF4FF48072002808BF1C46B1
:10F2A000234687B013F9087B1888C8B9154B93F823
:10F2B0000C01A3790593A3880493A378039323886F
:10F2C0000091CDE90123104A104B0321002818BFFB
:10F2D00013460F4A0120FEF77FFB204607B0F0BD22
:10F2E000161AD51B002EB8BF7642002DB8BF6D424E
:10F2F000AE42BCBF1C4647B20833D5E7C05B060828
:10F300005C110020D0600020D31C0708F63A0708E3
:10F310000904070808B500684DF015F9024BC3F859
:10F320008000012008BD00BFD060002008B5006843
:10F330004DF009F9024BC3F89400012008BD00BF4D
:10F34000D060002038B514460D46002943D0344B18
:10F350009FED347AD3ED447AB3F92C21F8EEE77AB5
:10F3600006EE102AC7EE876AB3F92821D3ED457A55
:10F37000F8EEE77AB8EEC66AC7EE875A07EE102AAB
:10F38000D3ED477AB3F92421B8EEC77AB8EEE70A8D
:10F39000A6EE867AD3ED487AF8EEE77AE6EE877A3B
:10F3A000A6EEA70A07EE902AB3F92A21B3F926316F
:10F3B00006EE102A07EE103AB8EEC66AB8EEC77A23
:10F3C000F8EEE77AA6EE867AE6EE877AA5EEA70A49
:10F3D00050F048F928600CB3114BDFED126A93ED41
:10F3E000457AB3F91821B3F91A31B8EEC77A07EEA6
:10F3F000902A87EE260A07EE103AB8EEC77AF8EEA2
:10F40000E77A20EE070AB6EE007AA7EE870ADFED6C
:10F41000067A20EE270A50F025F92060012038BD39
:10F42000D06000200000F04A0000C842094B10B52F
:10F4300053F8304007EE901A5CB1F8EEE77A94ED9D
:10F44000047A94ED030AA7EE870A50F00BF9A3683B
:10F45000186010BD383D002010B50C4B0C4C1B68DB
:10F46000D4F830011B1AFA2B06D904201AF08CFAB2
:10F47000002084F8340110BD11B1D4F838310B608C
:10F4800012B1D4F83C3113600120F4E7042D0020C0
:10F49000D06000202DE9F0410C4DDFF834802C685D
:10F4A0006B6901271C400CB9BDE8F081B4FA84F304
:10F4B000C3F11F0307FA03F608EB830324EA0604EB
:10F4C000D3F84001036898476E61ECE7003C0140C7
:10F4D000D060002038B5104CD4F8805125B10F4AC7
:10F4E00064212846FAF7F2FC00212846FAF744FD89
:10F4F0006B681A68B2F844306FEA43436FEA5343CB
:10F500009BB2A2F8443013889BB243F001031380EE
:10F51000012384F8843138BDD0600020009F24008E
:10F520000A4B10B5D3F8804124B1094A0321204683
:10F53000FAF7CCFC20460021FAF71EFD20460549CB
:10F54000BDE8104040F62B424BF062BBD06000207B
:10F55000009F2400BC9B0020F8B583681C68637979
:10F56000DB0724D5A57994F85C3205F001073D4608
:10F57000F3B1E06B43681A68D36AC3F34E03536276
:10F5800094F86D32012B07D094F8613223B1B4F8AE
:10F5900068320133A4F8683285F001014BF084FA37
:10F5A0000023A4F866324FF08073C4F85C32F8BDD3
:10F5B00094F85F62012E04BF94F85D3284F85E32E5
:10F5C0002046FFF7D1FC4EB9012384F85F3287EA69
:10F5D0000301E06BBDE8F8404BF066BA002384F805
:10F5E0005F323946F5E7F0B52DED028B83B00E465C
:10F5F000154646F0EDFA002869D022F065FE354B3D
:10F60000354C1B6803F00203002845D0002B59D06D
:10F61000324F0DF1060022F065FED7F87425BDF8D3
:10F6200006309FED2F7A9B1A07EE903AF8EEE77AB4
:10F63000F0EE408A67EE877A9FED2A0A27EE800A6D
:10F64000FDF718FD07F5B16797ED008AA0EE688A0F
:10F6500040F08EFD54ED2A0AD0ED057AB0EE480A4E
:10F6600070EEA70AFEF720F97EB1DFED1F7A9FED5D
:10F670001F7A20EE000A20EE270AC0EE077A9FEDDF
:10F680001C7A77EE877AC6ED007A0DB1194B2B60A4
:10F6900003B0BDEC028BF0BDA3B134F98C3C01EE9C
:10F6A000103A34F98E3C00EE903A34F9903C00EE7A
:10F6B000103AB8EEC11AF8EEE00AB8EEC00AFEF74A
:10F6C000FAF8D1E754F8743C93ED330ACCE79FED98
:10F6D0000A0AC9E7306A0120C8710020D060002002
:10F6E0000AD7233C35FA8E3CCDCC9C3F00409C464B
:10F6F00082E6C547331390430000000070B504460E
:10F70000012024F059FF58B103684BB11C4A2379FA
:10F7100092F83D10994231D092F83C209A422DD077
:10F72000184B5E68730612D500212720FAF7A0FB5C
:10F73000002105462620FAF79BFB1DB12A682368A5
:10F740009A421BD018B1026823689A4216D0F5037A
:10F750000CD521680C4B0A221868814202D1D86866
:10F76000C0010BD4013A03F11403F5D1207911281B
:10F7700004D0A0F121035842584170BD0120FCE79C
:10F7800070030020306A0120BC05002008B520214C
:10F7900055F0CFFE0346184623B10278202A03F124
:10F7A0000103F8D008BD70B50D461446FFF7EEFF13
:10F7B0000646A0B1FEF7CAFE40F634039842A8BF41
:10F7C0001846B0F5617FB8BF4FF46170A0F5617362
:10F7D0001922B3FBF2F32B702378013323703046E8
:10F7E000FFF7D4FF0646A0B1FEF7B0FE40F63403A3
:10F7F0009842A8BF1846B0F5617FB8BF4FF461705A
:10F80000A0F561731922B3FBF2F36B702378013317
:10F810002370304670BD154B53F8200070B508B307
:10F82000134D0C2202FB005212F96F3C591C1AD0E6
:10F8300012F8670CB0B1E9188C2411F81C6C12F89E
:10F84000681C0020142263435C1805EB4404013A51
:10F8500034F8184C314410FA84F0F5D11423B0FB7D
:10F86000F3F080B270BD0020FCE700BFD060002044
:10F87000C871002038B503200D461446FFF7CBFFB2
:10F8800007EE900A8DB19FED0B7AF8EE677AF0EEF5
:10F89000006A67EE877AB8EE047AA7EEA67ADFED03
:10F8A000067A67EE277AC5ED007A0CB1034B236028
:10F8B00038BD00BF6740533A00007A443313904389
:10F8C00010B5427A044632B10146406851F80A3B0D
:10F8D00098470023637210BD10B4447A621C04443C
:10F8E000D2B24272A172037A934202D85DF8044BFD
:10F8F000E6E75DF8044B7047EEE710B503681A7948
:10F90000022A044602D1987A4CF00EFE002323719D
:10F91000236010BDF0B50D4B0D4E0446B34201D32C
:10F920000020F0BD587988420DD11D79A54200D044
:10F930004CB9D879904206D118680779AF4202D104
:10F9400005689D42EDD00C33E8E700BFA001000838
:10F950005C03000837B503460079022830D11B4A02
:10F9600093F91030009214225343194C194AE3586A
:10F97000934227D0A2F57842934225D002F58062C7
:10F9800093421DD101F108020DEB02011A8811F812
:10F99000085C22F040021204120C14211A8001FBB0
:10F9A00000441A88E16822F0380231F82510120468
:10F9B000120C0A431A801A8892B242F040021A804E
:10F9C00003B030BD0020DDE70120DBE700010203CA
:10F9D000B000002000300140C36910B5044623B9CF
:10F9E00009211420FEF75AF8E061E06910BD10B556
:10F9F00004460068FFF7F0FF8378DBB1B0F90A3006
:10FA000007EE903AF8EEE77AC4ED057AB0F90C30DB
:10FA100007EE903AF8EEE77AF1EE677AC4ED047AF1
:10FA2000B0F90E3007EE903AF8EEE77A0120C4ED17
:10FA3000067A10BD1846FCE710B504460068FFF7CB
:10FA4000CBFF8378CBB1B0F9043007EE903AF8EEF3
:10FA5000E77AC4ED047AB0F9063007EE903AF8EE92
:10FA6000E77AC4ED057AB0F9083007EE903AF8EE7F
:10FA7000E77A0120C4ED067A10BD1846FCE710B500
:10FA800004460068FFF7A8FF8378CBB18388DBBA10
:10FA900007EE903AF8EEE77AC4ED047AC388DBBA51
:10FAA00007EE903AF8EEE77AC4ED057A0389DBBAFF
:10FAB00007EE903AF8EEE77A0120C4ED067A10BD21
:10FAC0001846FCE710B500680C46FFF785FF0346B3
:10FAD000807840B15B892222DBBA93FBF2F303F218
:10FAE0006D132380012010BD38B500680D46144603
:10FAF000FFF772FFD0F8013007EE103ACDB1D0F821
:10FB00000530DFED176A9FED176A07EE903AF8EEC1
:10FB1000677A77EEE67A77EEA77AC7EE866AF7EE2F
:10FB2000007A76EEE77ADFED106A67EEE67AC5EDE9
:10FB3000007A9CB1DFED0D7ADFED0D6AB8EEC77A81
:10FB400027EE277AC7EE267A9FED0A7A77EEC77AF4
:10FB50009FED097A77EE877AC4ED007A38BD00BF51
:10FB60009AC9CC449AC94C460E76D7450000484302
:10FB700000E0FF44000048423393884337B50068F3
:10FB80000D461446FFF728FFD0F805309FED237A85
:10FB900007EE903AF8EE677AF2EE046A77EEC77AEB
:10FBA0009FED1F7AD0F8013067EE877AB3EE097ABD
:10FBB00067EE877A07EE103AF4EEE67AF1EE10FA85
:10FBC00006DCFAEE046AF4EEE67AF1EE10FA0CD5F1
:10FBD00017EE900A4EF0B8F9124ACDE9000104215F
:10FBE0000320FDF7F9FE03B030BD2DB1DFED0E6A45
:10FBF00067EEA67AC5ED007A002CF4D0B8EE477A0D
:10FC0000DFED0A6ADFED0A7AE7EE267A9FED097AE0
:10FC100077EE877AC4ED007AE5E700BF0000004682
:10FC200000008038530407080AD778430319C83DF9
:10FC3000000048C2339388430379022B0DD190F919
:10FC4000103014225343064AD3581A89920746BFEC
:10FC50001889C0F3C010012070470020704700BF12
:10FC6000B00000200368DB6B13B504462BB9236892
:10FC70005B6B3BB9FF23E38202E098470028F6D193
:10FC800002B010BD214601A898470028F2D0BDF867
:10FC90000630013B9BB2EEE7036810B59B68044653
:10FCA000984701236374FF23A37410BD036810B544
:10FCB00004461B689847236820469B689847E37C66
:10FCC0000133E37410BD036810B504465B689847C0
:10FCD000236820469B689847E37C013BE37410BD92
:10FCE0002DE9F3410446184616460D461F464DF0D1
:10FCF000BFFF2368E67328440022A0730092D3F864
:10FD0000148032463B4629462046C04702B0BDE833
:10FD1000F08130B5046885B0E469089D34B10DB94F
:10FD20000DF10F050095A04705B030BD2046FBE75B
:10FD300003685B6A184703689B6A184710B5037B22
:10FD400004460BB1437B13B92046FFF7F4FF236849
:10FD50002046DB68BDE81040184703685B6C03B1C0
:10FD60001847704738B504468B6801600D469847C0
:10FD70000B4B2361002323752B6B13B1204698474F
:10FD80002075084B93F830331BB1237D23F001031A
:10FD900023750023E3822046BDE8384062E700BFB8
:10FDA0000001FF00C871002003681B6803B11847F9
:10FDB000704703685B6803B11847704703681B6AA4
:10FDC00003B11847704703685B6A03B1184770476F
:10FDD00030B40468029DA46A1CB10295A44630BCEC
:10FDE000604730BC704730B40468029DE46A1CB1BF
:10FDF0000295A44630BC604730BC704703685B6C1A
:10FE000003B11847704703689B6C03B118477047EC
:10FE100003689B6F03B1184770470368D3F88030BD
:10FE200003B1184770470368D3F8843003B118470B
:10FE300070470368D3F8883003B11847704721B181
:10FE40000B68D3F88C3003B118470020704738B5E1
:10FE5000094C052303FB0044A13C0025013514F89F
:10FE6000010FEDB24CF093FA052DF7D1BDE8384003
:10FE700000204CF08CBA00BFC75B060810B5441ECA
:10FE800014F8010F00B910BDFFF7E1FFF8E7FFF725
:10FE900001BBFFF7FFBAFFF7FDBAFFF7FBBAFFF7A9
:10FEA000F9BAFFF7F7BA18B103689B6803B11847AE
:10FEB000002070470C4B93F8312370B506460D4671
:10FEC0008AB9D3F8344374B123681B685BB1204608
:10FED000FFF7E9FF38B123683246196820462B4600
:10FEE000BDE87040084770BDC87100200120704710
:10FEF00018B103689B6803B11847002070470B4B8B
:10FF000070B5D3F8384306460D4674B123681B68B4
:10FF10005BB12046FFF7ECFF38B123683246196821
:10FF200020462B46BDE87040084770BDC8710020D0
:10FF3000034620B1026812B1D26902B1104793EDB5
:10FF4000017A084BB8EEC77AD3EDD06AF6EE007AA4
:10FF5000E7EE267AFDEEE77A17EE900A00F30B0043
:10FF6000704700BFC8710020034620B1026812B17B
:10FF7000126A02B1104793ED027A084BB8EEC77AC5
:10FF8000D3EDD16AF6EE007AE7EE267AFDEEE77A57
:10FF900017EE900A00F30B00704700BFC8710020F5
:10FFA000034628B102681AB1516A09B1936918472A
:10FFB00093ED037A074BB8EEC77AD3EDD26AF6EE2B
:10FFC000007AE7EE267AFDEEE77A17EE900A00F364
:10FFD0000B007047C87100204FF47A7300F5006081
:10FFE000584340F6FF7390FBF3F000F57A70B0F5DC
:10FFF000FA6FA8BF4FF4FA60B0F57A7FB8BF4FF43C
:020000040801F1
:100000007A70704730B1036882881B691A4214BF46
:1000100001200020704710B1036882881A8370475E
:1000200010B1036882885A83704773B50C46054641
:1000300000B30668104B06F13F4202F57E0203EB67
:10004000922393F8AA024AF0A7FEAB88009304F02B
:1000500003038DF80430C4F381038DF8053069463D
:10006000C4F30013304664098DF806308DF807405C
:10007000FAF7A2FA02B070BDC05B0608F7B50C46ED
:1000800015460746A8B306681B4B06F13F4202F52A
:100090007E0203EB922393F8AA024AF07DFEB88811
:1000A0000090B0FA80F3C3F11F0303F00702C3F31B
:1000B000CC0306EB83039200196A0F27974021EACD
:1000C00007011962196A95400D431D6204F003038C
:1000D0008DF80430C4F381038DF805306946C4F30C
:1000E0000013304664098DF806308DF80740FAF7A2
:1000F00063FA03B0F0BD00BFC05B060838B5040961
:10010000013C032C00F00F0219D80E4D05EB4403FF
:10011000B3F8B01241FA02F313F001000ED001233C
:100120009340013B03EA0100254455F0F7FA95F8A6
:10013000B832034404480C2202FB030038BD0020FF
:10014000FCE700BFC05B0608147500202DE9F04FE6
:10015000542204460021BE4891B054F023FBBD490F
:10016000621E0846033412F8013F5D1E052D88BF4C
:100170000023944240F8043BF5D1B64A002352F8DC
:10018000040B012800F05A810133042BF7D100231E
:1001900051F8042B022A00F047810133042BF7D1D8
:1001A0000320FEF77BFC0420FEF778FC0520FEF719
:1001B00075FC0620A64EDFF8B882FEF76FFC3446C9
:1001C0004FF01A0B4FF0000A08F52F79277B57B331
:1001D000384694F90D50FFF791FF28B1052383713C
:1001E000002380F807B003721321FFF71EFF0023DE
:1001F00019F83310B94240F0DE8008EBC303D3F89E
:10020000C032954A2361182303FB0525D5F8E03059
:100210002375591C0723A3750123C5F8E0106375E6
:1002200085F8DC309A440BF1010B5FFA8BFBBBF1D4
:10023000200F04F10C04C9D1BAF1000F00F0B8800E
:10024000864DDFF8308200272B7C002B00F0A88041
:1002500068794AF0A1FD28794AF09EFDD5F808A0FA
:100260005046FAF721F92C68D5F81490CDF80C8097
:100270000023CDE90C33CDE90E330493069304F14A
:100280004C030293EB680193142303FB09F34FF42F
:10029000806205934FF40063CDE907234FF40051CA
:1002A0004FF48073CDE9091350464FF4003301A990
:1002B0000B934AF083FCDAF80030694A43F00103FB
:1002C000CAF800305168674B0B4043F44033536029
:1002D0006268B9F1010F22F04072D4BF00230123FC
:1002E00022F4807242EA03226260A2685E4B1340ED
:1002F00043F00203A360E26A09F1FF3322F47002C3
:10030000DBB242EA03530122E362304694464FFADD
:1003100087FE437D6BB390F90D30734529D1037C83
:1003200090F81690092B4CD9A3F10A01D4F80CA02F
:1003300001EB41014FF0070B0BFA01FB2AEA0B0A14
:1003400009FA01F141EA0A01E160062A48D8511E82
:10035000D4F8349001EB81014FF01F0A0AFA01FA38
:1003600029EA0A0903FA01F141EA0901616301324C
:10037000D2B20CF1010CBCF1070F00F10C00C8D196
:10038000A36843F40073A360A36843F48073A3607D
:10039000A36843F00103A360A36843F08043A36014
:1003A0000137032F05F1180508F58C787FF44CAF61
:1003B00011B0BDE8F08F0133102B7FF419AF00238B
:1003C0001FE7216903EB430B4FF0070A0AFA0BFA08
:1003D00021EA0A0A09FA0BF141EA0A012161B4E7AC
:1003E0000C2A10D8D11FD4F8309001EB81014FF0C6
:1003F0001F0A0AFA01FA29EA0A0903FA01F141EA95
:1004000009012163B3E7A2F10D01D4F82C9001EBAF
:1004100081014FF01F0A0AFA01FA29EA0A098B4002
:1004200043EA0903E362A2E7104B212203F8582CA8
:1004300013F81C2C013203F81C2CB1E60B4B1122D3
:1004400003F8642C13F81C2C013203F81C2C9EE6D4
:1004500058710020D0600020F0100020BC11002056
:1004600000230140E030FCFFFDF7FFC0C871002011
:10047000C05B0608B07100202DE9F04F85B0B04D8B
:100480000293B04B9D4220D26C798C4240F0708137
:100490002C79844202D0002840F06A81EC799442A1
:1004A00040F066812C6884B11C220021201D54F08C
:1004B00079F925602B792371AA79A2600192012B29
:1004C0002A7AE26006D0022B0DD00024204605B027
:1004D000BDE8F08FE87AFFF711FE6B7A2374AB7AF0
:1004E000A0616374F2E7E87AFFF708FE95F90980E6
:1004F000A06184F81080A87AFFF700FE07466061CB
:10050000002800F0318114238F4E03FB08F3F2180A
:10051000F558002D00F02881937C002B40F0CB8013
:1005200092F8089048464AF037FC09F01F024FEA5B
:1005300059190123A9F102099340B9F1030F08D811
:10054000DFE809F07872026C80490A6922EA030345
:100550000B61142303FB086308F101095879FFF7C5
:10056000CDFD5FFA89F9034620B140F60A32C28018
:1005700080F80890142202FB08620393D079FFF7F9
:10058000BDFD039B824620B140F60A52C28080F82E
:100590000890142202FB086203939079FFF7AEFDE6
:1005A000039B834620B140F60A42C28080F808903F
:1005B000142202FB086292F80990019A12F00402D8
:1005C00001924A463CD04A211846FFF757FD4A4659
:1005D0002A215046FFF752FD4A460A215846FFF7A6
:1005E0004DFD142303FB086393F804A0BAF1000F38
:1005F00006D05046FFF782FD4A460921FFF73EFD2F
:10060000534B9D4223D103F584335A6A42F48052FE
:100610005A625A6A22F480525A6225E04B494A696A
:1006200022EA03034B6194E748490A6A22EA03037A
:100630000B628EE745494A6A22EA03034B6288E768
:100640000A211846FFF71AFD4A460A21C1E7414B25
:100650009D423ED103F500331A6A42F480421A6289
:100660001A6A22F480421A62019B002B65D1012292
:1006700002212B880A4303F44153134343F4457387
:100680002B80AB8B23F400631B041B0CAB83072371
:100690002B822B889BB243F040032B80BAF1000FD2
:1006A00004D05046FFF72AFDFFF7B5FC142303FBE7
:1006B00008660123B374029BBB710E23FB710023F8
:1006C00038463B720921FFF7B0FC3846FFF7A3FC20
:1006D000FCE6214B9D4209D103F5FE331A6A42F430
:1006E00000421A621A6A22F40042BCE71B4B9D4288
:1006F00009D103F582335A6A42F400525A625A6AA7
:1007000022F4005288E7164B9D4209D103F5684355
:100710005A6A42F480125A625A6A22F480127BE7C3
:10072000104B9D42A0D103F564435A6A42F4001273
:100730005A625A6A22F400126EE70022114698E7C4
:10074000A00100085C030008B0000020003802404F
:100750000030014000380040003C004000340140BF
:1007600000500140005401402046FFF7C6F8ACE6B7
:100770000C3587E6074B03EB8003D3F83C333BB1E2
:100780009A881B6859690A4201D05A8370471A83B4
:10079000704700BFC05B0608064B03EB8003D3F82D
:1007A0003C332BB11A689B8809B913837047538374
:1007B000704700BFC05B06082DE9F84F6B4B93F8FC
:1007C00084E1BEF1000F40F0CE80D3F8809199F81B
:1007D0001030002B40F0C780DFF898C19CF89A35A4
:1007E0009CF89B259CF89C55ACF898E50CF29E5023
:1007F000F0463C268178C778C1F1FF0189B2002913
:1008000000F0AD80C1F1FF0179430488B4FBF6FA32
:100810000912BAF1050F20D8DFE80AF0030D64725F
:1008200083917A1A6243B2FBF6F252FA81F2CDB2A8
:10083000D2B23B460FE0B4FBF6F306FB13439BB288
:10084000C3F13C037A1A5343B3FBF6F353FA81F333
:10085000CDB2DBB23A464FF0010E1F0247EA024723
:1008600047EA050B00210127C1F1170A07FA0AFA26
:1008700008EB01041AEA0B0F04F12A0408BFBA4678
:10088000A4B23B4F01F1010118BF4FF0020A182931
:1008900047F824A0E7D108F118081FFA88F8B8F53E
:1008A000406F00F10400A5D18021ACF89E17BEF185
:1008B000000F05D08CF89C558CF89B258CF89A3548
:1008C0004FF44063ACF898359CF8A037002B4AD021
:1008D000484640F62B41F9F773FC4846BDE8F84F0F
:1008E000F9F7A0BCB4FBF6F206FB12427D1A92B2F5
:1008F0005543B5FBF6F555FA81F5CBB2EDB2A9E754
:10090000B4FBF6F206FB124292B2C2F13C027C1A30
:100910006243B2FBF6F252FA81F2CBB2D2B23D465A
:1009200099E7B4FBF6F506FB15447B1AA4B26343C2
:10093000B3FBF6F353FA81F3CAB2DBB2EFE7B4FBD1
:10094000F6F306FB13439BB27C1AC3F13C03CAB215
:100950006343B3FBF6F353FA81F1CDB269E73D4649
:100960003A463B4677E7BDE8F88F00BFD0600020ED
:10097000BC9B0020C871002070B500212520F9F72C
:1009800077FAC36813F08073044607D12A4A1446E5
:10099000D168C90126D5142202FB03442046FDF785
:1009A000B7F8264B0546C3F8800100B32079244EE2
:1009B000FFF7A4FBC6F8A40720B140F21523C380BB
:1009C00000230372227A4A21FFF758FB96F8A837D2
:1009D000022B0DD1FEF77EFD2846F9F7C3FB00235D
:1009E000036004E001330A2B02F11402D0D170BD80
:1009F000032B06D1FEF76EFD2846F9F7B3FB6423FF
:100A0000EEE7FEF78DFD10B986F8A007EFE743F299
:100A1000AC020C48002153F0C5FE96F8A837012B14
:100A200002BF094BFF22C3F8A820012386F8A03794
:100A3000BDE87040C0E600BFBC050020D0600020CB
:100A4000C8710020BC9B0020BCCB0020F8B5134B24
:100A5000D3F88041054604B393F88411C9B9E0681E
:100A600066688268136823F001031360326877793F
:100A70000B4E938936F817609BB223EA06039381E5
:100A8000217413889BB243F0010313800177FEF7B2
:100A900021FD2046F9F766FB0560F8BDD060002017
:100AA000005A060838B5114BD3F8800158B193F8B5
:100AB000842142B10E4C94F8A827032A04D1F9F7F7
:100AC00051FB6423036038BD022A4FF0000503D1B7
:100AD000F9F748FB0560F6E783F88451FEF720FD3F
:100AE0000028F0D184F8A007EDE700BFD060002017
:100AF000C87100200346806B9B7903F00103994283
:100B000001D0FFF788BAFFF78BBA10B5837913F0DD
:100B1000010F03F020020446C36B13D05B68002A68
:100B20001A7A08BF4221606B18BF0221FFF7A6FAAC
:100B3000012184F86012A4F85C12E06BBDE810405B
:100B4000F9F726BB5B68002A08BF22211A7AEAE778
:100B5000036C806B23B15B6801211A7AFFF78EBAB0
:100B60000121FFF762BA2DE9F04183681C686679BC
:100B7000B1072FD594F86152C5B194F962528DB185
:100B8000B4F864124B08A4F86432204601F0010165
:100B9000FFF7B0FFA379013D6DB2580684F86252A9
:100BA00018D5BDB9002384F8613213E0A36A626AE4
:100BB00094F860129A4225D161B9A3791A0709D530
:100BC000236CA06BD3B15B681A7AFFF757FA204603
:100BD000FFF79BFFF10740F1818094F85C32002B16
:100BE0007CD194F85D320133DBB2092B84F85D329D
:100BF00035D12046BDE8F041FEF7B6B91946FFF7FA
:100C000014FAE4E75A1CA069A262C35C2069A779C0
:100C10005B0043F40073A4F864320A23824228BFC5
:100C2000002284F862320123A26284F8613299B111
:100C30003B0711D5D4F83C8029464046F9F7A8FA7D
:100C4000D8F80430606B1A7A2946FFF717FA84F84F
:100C500060522046FFF77CFF7D068ED4BAE70A2B50
:100C60003CD194F85F322BB9B4F8663243F00103FB
:100C7000A4F86632B4F86602820501D4C3071AD418
:100C8000B4F86A320133A4F86A3294F85F5201234F
:100C90009D42A4F85C3221D1A179E06B002384F855
:100CA0005F3201F0010149F0FFFEE06B2946BDE82B
:100CB000F041F9F76DBAE36AC0F3470013B1216B55
:100CC0009847E2E7E3696269D054E369E268013377
:100CD000B3FBF2F102FB1133E361D6E7BDE8F0812B
:100CE000F8B51E4B46681A6804461346B3FBF1F08C
:100CF000B0F5803F2ED281B22046F9F7E7F823689D
:100D00001F687C7974B165B203212846F9F7CAF8E7
:100D1000002D07DB6109124A04F01F040123A340E0
:100D200042F82130BC7974B165B203212846F9F745
:100D3000B9F8002D07DB6109094A04F01F040123FB
:100D4000A34042F82130326813889BB243F001037C
:100D50001380F8BD012BCBD95B08C7E72001002029
:100D600000E100E08160C06BBAE7002ABCBF8018D8
:100D70005242002BBCBFC9185B420028BCBF121AEC
:100D80000020F0B584180029A4F11D04BCBF5B1835
:100D90000021002CC8BF121BCC180F3C002CC8BF70
:100DA0001B1B0B4E02440B443C274FF0200C90427F
:100DB0000CDC06EB40050C4604E007FB04FE0134A6
:100DC00025F80EC09C42F8DD0130F0E7F0BD00BF11
:100DD0007479002008B5114B1A6C42F080521A64E5
:100DE0000F4A012111620F4AFF215162CA2151624B
:100DF000532151625B6FDB0009D400210120FAF717
:100E0000FDF8BDE8084008490020FAF7F7B80020CF
:100E1000FAF704F9044B9842EFD108BD00380240BC
:100E200000000E420028004076614E6938B50C463D
:100E300005461946046014B12046F9F747F8BDF895
:100E400010102046F9F798F863681A68B2F8443031
:100E50006FEA43436FEA53439BB2A2F844301388CE
:100E60009BB243F0010313802046F9F77BF900237E
:100E7000A860036038BD2DE9F04F85B006469DF8A7
:100E80003CA0039289469846FCF742FE834648B14F
:100E9000214C94F86C2B082A09D9204A00210420FF
:100EA000FCF79AFD0025284605B0BDE8F08F531CDD
:100EB0005C21DFB284F86C7B04F5376501FB0244EA
:100EC00002FB01550022C4F8702B84F8742B307992
:100ED000FFF714F9044620B1022280F80690C2718F
:100EE0000772BDF838300093039A434659462846A6
:100EF000FFF79CFFBAF1000F05D0327A022120469D
:100F0000FFF7BCF8CFE720461121FFF78EF8204607
:100F1000FFF786F8C7E700BFC8710020750407080F
:100F200030B51E4B2DED028B1C68B4FBF1F303F5BD
:100F30007F4383B0FF331B0CB4FBF3F40023B4FBFB
:100F4000F1F5019200932246ABB20221F0EE408A05
:100F5000B0EE608AFFF78FFFE0B107EE904AB5EE82
:100F6000408AF1EE10FAF8EE677A0ABF07EE105ADF
:100F700068EE270AF8EE470A9FED097AC0EE876A05
:100F80000123037127EE667AC0ED046AA8EEA77A02
:100F900080ED037A03B0BDEC028B30BD2001002050
:100FA00000007A440023064910B51C46984200DC34
:100FB00010BD51F833200AB1926814600133F5E78F
:100FC000383D002013B50F4C8DF80700D4E90423F9
:100FD000A16853438B4212D06368E0680DF10701AA
:100FE000184452F0BDFA636822691344A268B3FB47
:100FF000F2F102FB1133636063690133636102B094
:1010000010BD00BF103D00200F4B1B78062B14D8DD
:10101000DFE803F0041316070A0D10004FF4C87040
:1010200070470A4B588870474FF47A6070474FF406
:10103000FA5070474FF47A5070474FF47A70704707
:101040004FF4FA60704700BFEC3C0020783E00206F
:101050002DE9F04F2DED028BA54FA64D3B78DFF823
:10106000D0B299B000240393AA462646A946DAF8DE
:1010700000804046F8F7BEFE584490F8AC2E022A95
:101080006FD0032A76D0012A09D1DAF80C2022F099
:10109000807222F0080242F00402CAF80C20504686
:1010A000FEF72CFB70B9142202FB0692D16801F006
:1010B0000C02042A06D14046FDF7F2FF0134E4B2E7
:1010C0000444E4B201360A2E0AF1140ACFD18A4E42
:1010D000A6F1C8084046FEF711FBC0B9D8F80C10BD
:1010E0004A0714D501F00C03042B10D0039B9C423B
:1010F00047D221F0080141F00401D8F80000C8F8F7
:101100000C10FDF7CDFF0134E4B20444E4B208F161
:101110001408B045DED14FF000094C464E46C84693
:101120002846FEF7EBFAA8B3744A4346012104208F
:10113000FCF752FC08F10108B8F10A0F05F114059B
:10114000EED13E780C2E40F38F8001238BF8BA3E0F
:101150006B4A0C230093334600210420FCF73CFC2F
:10116000A7E0DAF80C2022F0807222F0040242F0AC
:10117000080292E7DAF80C2022F00C0242F08072AA
:101180008BE721F00401D8F80000C8F80C10FDF737
:1011900087FFBCE7E9684B070AD5039B9E4207D24D
:1011A00021F008012868E960FDF77AFF0136F6B200
:1011B000EA6810071AD5286805A900239C420DDCAF
:1011C0000823EB6018AB03EB890209F1010A08213F
:1011D00042F8245CD146FDF763FFABE751F804CF3A
:1011E000DCF800C0604501D00133E7E751071AD5AC
:1011F00028680EA900234B450DDB0423EB6018ABD8
:1012000004F1010A03EB8404042144F8485CFDF76F
:1012100047FF54468EE751F804CFDCF800C0604524
:1012200001D00133E7E7D30184D5286805AA00235C
:101230009C4202DC0EAA00230EE052F8041F09684B
:1012400088423FF477AF0133F2E752F8041F096890
:1012500088423FF46FAF01334B45F6DB4FF08071AE
:10126000E960FDF71DFF65E7264B1979264B032939
:10127000197035D90B1F022B34D8FFF7C5FE234A4E
:10128000234B9FED197B80B2B3FBF0F31360002377
:101290005360204B83ED007B1F4BCBF8BC3E1F4BB4
:1012A00013F81130002B45D11D4A02210420FCF710
:1012B00093FB20F0A9FE9BF8C03E0446002B40F0B3
:1012C000BE80184A02210420FCF786FB9BF8BA0E68
:1012D000B0FA80F0400919B0BDEC028BBDE8F08F88
:1012E000114BDAE7114BD8E70000000000000000C6
:1012F0002C6A0120BC05002084060020B0040708E9
:10130000C8040708783E0020EC3C0020F83C002090
:1013100040420F00003D0020CFF00008845B06082B
:10132000F4040708700507082DF40008CDF0000844
:10133000C8710020A64217DC754F9FED768A0DF12B
:1013400014080024A642B4DD734B58F8045F5B68B0
:10135000C3F3007A714B1B78062B6CD8DFE803F0DF
:10136000621B220B2B2B2B0003238BF8BA3E6C4AFB
:1013700000943346F0E6FFF747FEDFED6A0A0146C8
:101380005246B0EE600A2846FFF7CAFD47F834001F
:10139000002845D125E0FFF737FEDFED630A01465F
:1013A0005246EEE7FFF730FEDFED600A9FED600A80
:1013B00001465246E7E7052B1DD05E4A5E49062BE3
:1013C00018BF0A46CDF804A04FF0000A2846CDF811
:1013D00000A014230221FFF74EFD054668B947F827
:1013E000340005238BF8BA3E544A234600210420DA
:1013F000FCF7F2FA5DE7524AE4E700F114031946FC
:1014000000680393122249F003FC039B30B1184695
:101410004822514653F0C6F901232B7147F8345046
:1014200001348FE7FFF7F0FD9FED3A0A014652467F
:10143000F0EE480AA7E7002347F83430D1E7122836
:101440000BDD02238BF8BA3E3E4A122300930021A3
:1014500003460420FCF7C0FA38E79BF8CA3E012B8C
:101460000CD0022B0ED0384BCBF8D03E9BF8CA3EA6
:10147000002B38D0022B09D0344A23E74AF08AFBEC
:10148000334BF1E74AF086FB324BEDE74B46122B2C
:10149000B8BF12239BB29C4227DC4C45A8BF4C46E8
:1014A0002D4FDFF8B880DFF870900EAE0025A54212
:1014B000BFF60CAFD9F80420BBF8C43EB8FBF3F379
:1014C000C2F300720192BBF8C22E00920321234A9C
:1014D00056F8040F9BB2FFF7CEFC014670B147F8F7
:1014E000040B0135E3E74B46D4E704208BF8BA0E32
:1014F0001B4ACDF8009023460021ABE705238BF86B
:10150000BA3E184A2B460420FCF766FADEE600BF16
:10151000383D00206F12833A306A0120EC3C0020F5
:1015200012050708000000006F120339ACC5A73789
:10153000ACC5A736001BB700C0C62D004B05070879
:10154000808D5B008A050708E9F00008B6050708EA
:101550002101030805F100088461002040420F00CA
:10156000F205070828060708034AD2F8D02E12B160
:10157000112800D810477047C871002040B10138C9
:101580000023FF2803F1010203D840EA032080B2C0
:10159000704740081346F4E703681B681847036860
:1015A0005B68184703689B68184703681B6A70B537
:1015B00006460C46154683B1BDE8704018473046D4
:1015C000FFF7F0FF0028FAD014F8011B3046FFF7B0
:1015D000E3FF2B1B002BF2DC70BD0D44F9E7E4E7C1
:1015E0000368DB68184703681B69184703685B6971
:1015F00018470368DB6A03B11847704703681B6B21
:1016000003B118477047164B1B6813F0100F154BAA
:1016100005D0B3F8D42E12F0040F18BF002093F8B1
:10162000EE2E72B1D3F8F02ECAB1926838B1B3F889
:10163000F41E0D4BB3FBF1F35B10136070471060A9
:101640007047D3F8F82E93F8FC3E0BB980F00100F8
:101650002AB11368928808B11A8370475A83704779
:1016600088690120C871002040420F00BFF34F8FEE
:101670000549064BCA6802F4E0621343CB60BFF32E
:101680004F8F00BFFDE700BF00ED00E00400FA054A
:1016900008B572B600224FF0FF31930003F16043AA
:1016A00003F561430132082AC3F88010C3F88011A2
:1016B000F3D1FFF7DBFF012108B50846F9F79EFCDF
:1016C000FFF7E6FF08B50120F9F7A8FC012809D1CA
:1016D0000021F9F793FC044B1A6882F308885B68D1
:1016E0009847FEE708BD00BF0000FF1FEFF311831E
:1016F000102282F3128809490A6801320A604FF009
:10170000E02207499069C1F8000F0020C1F8040FDA
:101710001269DBB283F31188704700BF042D0020EB
:10172000C8710020074A084B5168D3F8083F584356
:101730004FF47A73B0FBF3F053685B1A8342FBD922
:10174000704700BF001000E0C871002010B50446CB
:101750004FF4FA70FFF7E6FF6069BDE81040FEF74E
:101760005ABC90F910302DE9F0411646142253432B
:101770000D4A52F80380836813F0020504460F46B1
:1017800002D140694AF0C8FE394640464CF046F85E
:10179000314640464CF042F815B92046FFF7D6FFD7
:1017A0000120BDE8F08100BFB00000207FB50379C3
:1017B000012B0D460AD0022B19D18368DB0758BFD5
:1017C00001F07F0104B0BDE87040CAE781688DF880
:1017D0000F2001F001010DF10F0200920191417CF7
:1017E00090F910002A46F9F7BDFB04B070BD002047
:1017F000FBE700682E22F421D8E7044B00681A8E1C
:101800009201343202F0FC02F421CFE7D0600020D4
:1018100008B53122F4210068FFF7C8FF012008BD98
:10182000006801225821C1E7006801224821BDE774
:10183000006802220821B9E7006801220821B5E703
:1018400010B50446002221210068FFF7AFFF206891
:10185000FC222021FFF7AAFF206840222421FFF765
:10186000A5FF20680C222321FFF7A0FF206800229B
:101870002221FFF79BFF012010BD10B50122044675
:101880000B210068FFF792FF20B120681D2209217B
:10189000FFF78CFF00F0010010BD044B0246D3F8A7
:1018A0000C0F08B1802181E7704700BFC87100208C
:1018B00010B5B020FFF7F1FF4020FFF7EEFF00204A
:1018C000FFF7EBFF1020FFF7E8FF4FF48064013CC7
:1018D0000020A4B24AF05BFD002CF8D110BD10B579
:1018E0000446A1F15000C0B2FFF7D7FF04EB44005B
:1018F000400004EB440400F00E00FFF7CEFFC4F3F9
:10190000C3001030BDE81040C7E708B55038C0B27A
:10191000FFF7C3FF0020FFF7C0FFBDE8084010201D
:10192000BBE738B500221F2334210120FEF7A4FDB8
:101930003C4BC3F80C0F10B90024204638BDAE2034
:10194000FFF7ABFF04460028F6D0D420FFF7A5FF31
:101950008020FFF7A2FFA820FFF79FFF3F20FFF79F
:101960009CFFD320FFF799FF0020FFF796FF402050
:10197000FFF793FF8D20FFF790FF1420FFF78DFFF7
:10198000A120FFF78AFFC820FFF787FFDA20FFF7C3
:1019900084FF1220FFF781FF8120FFF77EFFCF2019
:1019A000FFF77BFFD920FFF778FFF120FFF775FFE6
:1019B000DB20FFF772FF4020FFF76FFFA420FFF747
:1019C0006CFFA620FFF769FFAF20FFF766FFA62098
:1019D000FFF763FFAE20FFF760FF2020FFF75DFFFA
:1019E0000020FFF75AFFB020FFF757FF4020FFF716
:1019F00054FF0020FFF751FF1020FFF74EFF4FF478
:101A00008065013D0020ADB24AF0C1FC002DF8D147
:101A10008120FFF742FFC820FFF73FFFAF20FFF70D
:101A20003CFF8AE7C871002008B5FFF7BFFE014BF5
:101A3000187008BDF01000202DE9F0411E4690F905
:101A400010301546142253430E4A52F8038083681F
:101A50009A0704460F4602D440694AF05DFD3946B4
:101A600040464BF0DBFE33462A46002140464BF011
:101A70006DFEA3689B0702D42046FFF767FE012096
:101A8000BDE8F081B0000020F7B50779012F1646B8
:101A90000AD0022F15D18468E40758BF41F08001B5
:101AA00003B0BDE8F040C7E7826802F00102CDE96B
:101AB00000620A46417C90F91000F9F753FA03B02E
:101AC000F0BD0020FBE707B552BAADF804200223B1
:101AD00001AAFFF7D9FF024B187003B05DF804FBB1
:101AE000F010002010B50A4C002384F8103F84F851
:101AF000111F84F8122F032304F57162FF21FFF7F1
:101B0000C3FF00280CBF6FF00C00002010BD00BF09
:101B1000C871002010B50B4C002384F8103F130A45
:101B200084F8111F84F8123F84F8132F042304F55E
:101B30007162FF21FFF7A8FF00280CBF6FF00C00B7
:101B4000002010BDC8710020024A00680023512106
:101B50009AE700BFD8810020024A006801230021D3
:101B600092E700BFD88100202DE9F0411E4690F990
:101B700010301546142253430E4A52F803808368EE
:101B80009A0704460F4602D440694AF0C5FC39461C
:101B900040464BF043FE33460022294640464BF078
:101BA000D5FDA3689B0702D42046FFF7CFFD012097
:101BB000BDE8F081B0000020F7B50779012F164687
:101BC0000AD0022F15D18468E40758BF41F0800184
:101BD00003B0BDE8F040C7E7826802F00102CDE93A
:101BE00000620A46417C90F91000F9F7E1F903B070
:101BF000F0BD0020FBE713B5062304466A460068E3
:101C00000221FFF7D9FFB8B1BDF9003007EE903AD5
:101C1000BDF90230F8EEE77AC4ED077A07EE903AA4
:101C2000BDF90430F8EEE77AC4ED087A07EE903A91
:101C3000F8EEE77AC4ED097A02B010BD13B50223BD
:101C400004466A4600680321FFF7B6FF10B900207A
:101C500002B010BD9DF90130002BF8DA206807238F
:101C60006A461221FFF7A8FF0028F0D09DF9022054
:101C70009DF8013043EA022313EB430348BF0333CB
:101C80009B1007EE903A9DF904209DF8033043EA3B
:101C9000022313EB4303F8EEE77A48BF03339B10AC
:101CA0009DF90620C4ED047A07EE903A9DF80530C0
:101CB00043EA022313EB4303F8EEE77A48BF03330A
:101CC0009B10C4ED057A07EE903AF8EEE77AC4ED82
:101CD000067ABDE738B504460068FDF77DFE0C23A3
:101CE0000546021D19462068FFF766FFA870B8B1C7
:101CF000B5F9043007EE903AF8EEE77AC4ED077ACA
:101D0000B5F9063007EE903AF8EEE77AC4ED087AB6
:101D1000B5F9083007EE903AF8EEE77AC4ED097AA3
:101D200038BD38B504460068FDF756FE0D2305465C
:101D3000C21C0C212068FFF73FFFA870B8B1B5F9AD
:101D40000A3007EE903AF8EEE77AC4ED077AB5F973
:101D50000C3007EE903AF8EEE77AC4ED087AB5F960
:101D60000E3007EE903AF8EEE77AC4ED097A38BD06
:101D700013B503230C46006801AA2221FFF71CFFBC
:101D800030B1BDF9053003EB83031B12E63323802A
:101D900002B010BD13B5062304466A4600681F2131
:101DA000FFF70AFFD0B1BDF80030DBBA07EE903A7A
:101DB000BDF80230F8EEE77ADBBAC4ED047A07EE3C
:101DC000903ABDF80430F8EEE77ADBBAC4ED057A54
:101DD00007EE903AF8EEE77AC4ED067A02B010BD4D
:101DE00013B5062304466A4600682521FFF7E4FE82
:101DF000D0B1BDF80030DBBA07EE903ABDF8023042
:101E0000F8EEE77ADBBAC4ED077A07EE903ABDF850
:101E10000430F8EEE77ADBBAC4ED087A07EE903AC0
:101E2000F8EEE77AC4ED097A02B010BD13B50223CB
:101E30000C46006801AA1D21FFF7BEFE98B1BDF84F
:101E40000430DFED0A6ADBBA07EE903AB8EEE77AC3
:101E5000C7EE267A9FED067A77EE877AFDEEE77A6F
:101E600017EE903A238002B010BD00BFCFF7534168
:101E700000007A4370B5066805463046FDF7ACFDB4
:101E80000E230446021D3B213046FFF795FEA0704D
:101E9000B8B1A389DBBA07EE903AF8EEE77AC5ED60
:101EA000077AE389DBBA07EE903AF8EEE77AC5EDF8
:101EB000087A238ADBBA07EE903AF8EEE77AC5EDA6
:101EC000097A70BD07B50223006801AAF621FFF761
:101ED00073FE20B1BDF80430024A5BBA138203B02E
:101EE0005DF804FBD060002007B50323006801AA59
:101EF000F621FFF761FE80B19DF805309DF80420C2
:101F000007491B0243EA02439DF806201343B1F937
:101F10003020C2F10802D3404B6303B05DF804FBEC
:101F2000D060002037B50623F7210068144C6A46BC
:101F3000FFF742FE1349D8B19DF801209DF800300B
:101F40009DF80350120142EA03329DF8023042EA42
:101F500013129DF804308A651B0143EA05339DF88E
:101F6000055043EA151344E93A238B6303B030BDAF
:101F700054F8E83C8B6554F8E43C8B63F6E700BF0B
:101F8000C0820020D060002007B50323006801AAAA
:101F90001946FFF711FEA0B19DF804309DF8051019
:101FA0009DF904201B0443EA01239DF80610002A32
:101FB000ACBF00224FF07F420B431343024AC2F8EA
:101FC000143103B05DF804FBD060002007B5032393
:101FD000006801AA0021FFF7EFFDA0B19DF80430D1
:101FE0009DF805109DF904201B0443EA01239DF888
:101FF0000610002AACBF00224FF07F420B43134370
:10200000024AC2F8103103B05DF804FBD060002032
:1020100013B5044600680379022B0CBF432103214A
:1020200006236A46FFF7C8FD18B9E086A06302B030
:1020300010BDBDF800305BBAE386BDF802305BBA74
:102040006387BDF804305BBA2387F0E713B500233C
:10205000C38683630446062300686A460321FFF7AC
:10206000ABFD78B1BDF8003003EB4303E386BDF967
:1020700002305B4203EB43032387BDF8043003EBDC
:102080004303638702B010BD07B5012301AAFF21F6
:102090000068FFF791FD03B05DF804FBF7B5054656
:1020A0000068FDF799FC00230370042304460DEB40
:1020B00003022868FF21FFF77FFD10B9002003B05D
:1020C000F0BD286804236A46FF21FFF775FD00284C
:1020D000F4D09DF804309B09023B012BEED9BDF8EA
:1020E0000420BDF80630BDF80050BDF8021052BA09
:1020F00043F6FF77C2F30D02BA42DFD0002ADDD0EB
:102100005BBAC3F34A1340F2FF76B342D6D0002B3A
:10211000D4D06DBAC5F30D05BD42CFD0002DCDD0C2
:1021200049BAC1F34A11B142C8D00029C6D0561BE2
:10213000002EB8BF7642FF2EC0DC5E1A002EB8BF5C
:102140007642FF2EBADC01262A440B443241334149
:102150002670C4F80520C4F80130B0E737B505464D
:102160000068FDF739FC00230370042304460DEBDF
:1021700003022868FF21FFF71FFD40B19DF80430DE
:102180009B0907D00B4A04210320FBF725FC002004
:1021900003B030BDBDF80420BDF8063052BA5BBABA
:1021A00092B2C3F34A1301212170C4F80520C4F888
:1021B0000130EDE74D06070807B5022301AAFFF736
:1021C000FBFC044B1870BDF8040040BA80B203B0A9
:1021D0005DF804FBF010002038B515460C4A0B0AD8
:1021E00082F8103F82F8111F022302F57162FF216D
:1021F0000446FFF749FC30B101232A46FF2120465F
:10220000FFF7DAFC10B96FF00C0038BD0020FCE7D6
:10221000C87100202DE9F041104D05F57168164692
:10222000002485F8111F02234246FF21074685F846
:10223000104FFFF729FC18B96FF00C00BDE8F081D2
:1022400002234246FF213846FFF7B6FC0028F3D0B0
:10225000B5F8103F5BBA33802046EFE7C871002025
:102260002DE9F341744D0468DFF8D8810023064658
:1022700085F8FE302D27B9B218F8012B204601371A
:10228000FFF730FC882FF6D1402287212046FFF748
:1022900029FC00238DF806309DF80630002B6FD006
:1022A000012286212046FFF71DFC002287212046BF
:1022B000FFF718FC092208212046FFF713FC002233
:1022C0000B212046FFF70EFC002851D137680DF195
:1022D00006025E213846FFF79DFFBDF80630B3F5D4
:1022E000D77F00F0A58059D8512B00F09F804DD8A2
:1022F0001D2B70D01E2B00F099803068212149F0F1
:1023000018FF34680DF10602DE212046FFF782FF38
:10231000BDF806309FED497A2822C3F309035343E1
:1023200007EE903AF8EEE77A454A67EE877A0021A1
:10233000FCEEE77A82F8101F17EE903A6C2182F8D3
:10234000111F190E82F8121F190C82F8131F190A97
:1023500082F8141F82F8153FFF2102F571620623EF
:102360002046FFF791FB306840228721FFF7BAFB38
:10237000B0FA80F0400985F8FE0002B0BDE8F081B7
:102380000DF10601204649F065FF85E7AD2B4FD0E2
:10239000D62B01D0602BB0D121241DE040F2E132D8
:1023A000934247D00CD840F2D922934242D040F217
:1023B000E122934202D0B3F5E67F9ED164240BE084
:1023C00040F28F42934203D040F29152934294D113
:1023D0004FF4FA7400E00F2400288ED10A224B211A
:1023E0003846FFF77FFB0F2260213846FFF77AFB64
:1023F0000D2263213846FFF775FBB8226921384664
:10240000FFF770FB40F60D7278213846FFF782FB2C
:1024100040F60E627A213846FFF77CFB00287FF4F5
:102420006CAF2146384649F084FE66E71424D3E7B2
:102430003224D1E7C824CFE7D06000209A99893FA1
:10244000C8710020085F060837B5134D95F8FE30B7
:102450000446FBB100680DF1050149F0FBFE9DF853
:1024600005307BB10DF1060220689621FFF7D2FE00
:102470000A22BDF80630B3FBF2F3084A9360012349
:1024800085F8FF3020680122862103B0BDE8304086
:10249000FFF728BB03B030BDD0600020F010002053
:1024A00013B5022301AA044651210068FFF784FBFB
:1024B000114AE8B1BDF804305BBA9BB2D360D3686F
:1024C000B3F5C87F02DD4FF0FF33D3600B4B0C4AEE
:1024D000196852F8E03C32338B4207D242F8E01CD4
:1024E00020680023E83A5121FFF7CEFA02B010BD70
:1024F0006FF00103E9E700BFF0100020042D002079
:10250000C082002007B50223006801AA0021FFF75E
:1025100053FB0F4B83F80401B0B1BDF804300D4AF2
:102520005BBA9BB2B3F5FA6F3FBF0A21B3FBF1F37D
:1025300007EE903AF8EEE77A2BBF4FF0FF33FDEE4F
:10254000E77A1361C2ED047A03B05DF804FB00BFC3
:10255000D0600020F01000202DE9F0412C4C00212B
:10256000054603230068A4F1DC02FFF725FB294997
:10257000002848D034F8DC3C14F8DACC5BBA9BB2C3
:1025800007EE903AF8EEE77AF2EE046A87EEA67A62
:10259000A4F1DC0703200023BDEEC77A81ED427A67
:1025A00001381FD19C450CD1D1F808312BB1D1F89D
:1025B00008214FF6FF739A4203D14FF0FF33C1F861
:1025C0000831154B1A6854F8D83C323393421DD267
:1025D00044F8D82C2868114ABDE8F0410123312184
:1025E000FFF752BA17F8012B082653405AB2002AB7
:1025F000BBBF520082F007025B00D3B2A8BFDBB2C0
:10260000013EF3D1CCE76FF00103D8E7BDE8F081DC
:10261000C0820020D0600020042D0020D88100203E
:1026200013B502230C46006801AA0021FFF7C4FA83
:1026300060B15CB19DF805309DF90420DB0903EB26
:10264000830302EB820203EB4203238002B010BD3E
:10265000F8B590F910301546142253430D4AD75857
:1026600083689A0704460E4602D4406949F054FF35
:10267000314638464BF0D2F801230022294638462D
:102680004BF064F8A3689B0702D42046FFF75EF87E
:102690000120F8BDB000002073B50379012B164668
:1026A0000AD0022B15D18368DB0758BF41F08001A7
:1026B00002B0BDE87040CBE7826802F00102CDE9CC
:1026C00000620A46417C90F91000F8F771FC02B0F4
:1026D00070BD0020FBE713B504466A460068082178
:1026E000FFF7DAFF9DF80030DB0602D4002002B0CD
:1026F00010BD206806236A460021FFF75DFA002816
:10270000F4D09DF801309DF800209DF80410DFED15
:10271000496A1B0203EB02439DF802201C021A4483
:102720009DF8033048BF02F17F42090201EB0341EB
:1027300007EE902A9DF80530F8EEE77A0B4409027F
:1027400048BF03F17F4387EEA67A07EE903AF8EE92
:10275000E77A394BC7EEA63AB3F96A20B3F9741099
:10276000D3ED196AD3ED187AB8EEE66A06EE902A30
:10277000B3F96C2003EE101AB3F9681005EE902A35
:10278000B3F96E2004EE901A2C4905EE102AB3F925
:10279000702011F8D41C04EE102AF8EEE44A112936
:1027A000F8EEE77AF8EEE66AF8EEE55AB8EEC55AC2
:1027B000B8EEC44AB3F9722064EEA34A67EE232A46
:1027C0002CD1B8EEC33AA7EE034AE4EE075AA5EEC1
:1027D000876AE6EE077A06EE102AB8EEC66A77EE4A
:1027E000A47AA7EE065AE5EE076AB3F95C20E6EE96
:1027F000A27A07EE102AB3F95E20C3ED1E7A07EE27
:10280000902AF8EEE77AB8EEC77A67EEA37AF6EE8A
:10281000006AE7EE267AC3ED1F7A68E7E7EE045A0E
:10282000E7EE056AA5EE876AE6EE077A77EEA47A08
:10283000DBE700BF00007848D0600020C0820020A5
:102840002DE9F34116460DF107021D46074688465D
:10285000FFF722FF9DF8074006EA0403AB4209D0C8
:1028600024EA06022A434146384602B0BDE8F04158
:10287000FEF79CBF02B0BDE8F0811FB504460023FF
:1028800000688DF807300DF107022721FFF704FFDC
:1028900060B19DF807301B0708D52068062302AAFF
:1028A0002821FFF789F920B9E086A063002004B051
:1028B00010BDBDF90830002BB8BF03339B10E38671
:1028C000BDF90A30002BB8BF03339B102387BDF935
:1028D0000C30002BB8BF03339B106387E7E71FB5AD
:1028E00000210446C18681630DF107020068FFF7ED
:1028F000D3FE10B9002004B010BD9DF807301B07AF
:10290000F8D52068062302AA0121FFF755F900280F
:10291000F0D0BDF808305BBAE386BDF80A305BBA88
:102920002387BDF80C305BBA5B426387E3E730B5C1
:10293000002585B00446C58685630DF10702006851
:102940000621FFF7A9FE10B9002005B030BD9DF8A3
:1029500007305B07F8D52068062302AA2946FFF74F
:102960002BF90028F0D0BDF80830E386BDF80A3016
:102970002387BDF80C306387E7E707B50DF1070241
:10298000FFF78AFE034B18709DF8070003B05DF84F
:1029900004FB00BFF0100020F8B5144E144F41F0B6
:1029A000010200210446FFF73FF8356847F8D05C84
:1029B00013212046FFF7E1FF10F007000BD00122A2
:1029C0000B212046FFF730F8002220461146FFF782
:1029D0002BF8012008E057F8CC2C002AE8D0336807
:1029E0009BB25B1B9A42E3D2F8BD00BF042D0020CE
:1029F000C082002010B50C460121FFF7BEFFC0F3D6
:102A000000132370C0F3C003A370C0F3800363708E
:102A1000C0F38013C0F3C010E370207110BD2DE926
:102A2000F8430F46502114460546FFF7A6FF013034
:102A30004000C0B2208046212846FFF79EFF2C4E62
:102A40002378013080B273434FF47A78A08003F585
:102A5000FA734FF4FA69B3FBF8F25121B3FBF9F3BF
:102A600000FB02332846B3FBF8F3E360FFF7A4FB57
:102A7000C2B2C0F30F2023788240013292B2734376
:102A8000E28003F5FA732846B3FBF8F1B3FBF9F3E0
:102A900002FB01337021B3FBF8F32382FFF76DFFD4
:102AA00001304000C0B2608071212846FFF784FBEE
:102AB000C3B2C0F30F2083400133FA789BB2238165
:102AC00012B1E2889B1A2381A3782089734303F50E
:102AD000FA734FF47A724FF4FA65B3FBF2F1B3FB79
:102AE000F5F300FB0133B3FBF2F36382BDE8F88337
:102AF000002F3A002DE9F047DB4FDFF87483DFF851
:102B000074934FF4FA738AB0044600268921006852
:102B100047F8CC3C88F8FC60FFF72FFF40F001023B
:102B2000D2B220688921FEF77FFF324620688821D3
:102B3000FEF77AFF206801228021FEF775FF2068EA
:102B40000122FF21FEF770FF324631462068FEF772
:102B50006BFF91212068FFF710FF314607F8C80C82
:102B600001222068FEF760FF32462068FF21FEF751
:102B70005BFF324620688021FEF756FF6021206807
:102B8000FFF7FBFE40F01202D2B220686021FEF790
:102B90004BFF206820224421FEF795FF2068FF228A
:102BA0000121FEF741FF2568012280212846FEF71A
:102BB0003BFF0122FF212846FEF736FF3246314611
:102BC0002846FEF731FF0622FF212846FEF72CFF9C
:102BD00083212846FFF7D1FE40F00402D2B28321C0
:102BE0002846FEF721FF0722FF212846FEF71CFF9B
:102BF000012281212846FEF717FF01228021284665
:102C0000FEF712FF6B2294212846FEF70DFF324695
:102C100083212846FEF708FFD9F8006047F8D06CFA
:102C200083212846FFF7A9FE002800F046830122F1
:102C300028468321FEF7F8FE92212846FFF79DFEE5
:102C40000022C0F3C716814681212846FEF7ECFE1C
:102C500006222846FF21FEF7E7FE83212846FFF7DC
:102C60008CFE832100F0FB022846FEF7DDFE28469D
:102C70000122FF21FEF7D8FE284601220021FEF79F
:102C8000D3FE28460022FF21FEF7CEFE2846002272
:102C90008021FEF7C9FE062303AAB0212068FEF7B3
:102CA0008BFF20680122FF21FEF7BEFE2068002274
:102CB0004F21FEF7B9FE20682C224E21FEF7B4FE0C
:102CC00020680022FF21FEF7AFFE2068B422B62163
:102CD000FEF7AAFE0025002E18BF0C2609F07F097A
:102CE0002A460120C5F3C40C0CF128035FFA85FEC7
:102CF0000DEB030C76451CF81C3C05F0070102D8CF
:102D0000914540F0E58200FA01F123EA01030CF855
:102D10001C3C0135302DE5D1062303AAB0212068E3
:102D2000FEF7B2FE514B01221870FF212068FEF71A
:102D30007BFE002211462068FEF776FE2068002206
:102D4000FF21FEF771FE206800220921FEF76CFECC
:102D5000206800221021FEF767FE20680022112162
:102D6000FEF762FE206801222421FEF75DFE206846
:102D7000FF222521FEF758FE206800227521FEF76C
:102D800053FE20680122FF21FEF74EFE20682C2210
:102D90004E21FEF749FE206800224821FEF744FE3E
:102DA000294620682022FEF73FFE20680022FF21EE
:102DB000FEF73AFE294620680922FEF735FE206814
:102DC00000225421FEF730FE206804223121FEF754
:102DD0002BFE206803223221FEF726FE2068832284
:102DE0004021FEF721FE206825224621FEF71CFE29
:102DF000206800226021FEF717FE206800222721AC
:102E0000FEF712FE206806225021FEF70DFE206814
:102E100000225121FEF708FE206896225221FEF77B
:102E200003FE206808225621FEF7FEFD2A46206890
:102E30005721FEF7F9FD206800226121FEF7F4FD1D
:102E4000206800226221FEF7EFFD20680022642145
:102E5000FEF7EAFD206800226521FEF7E5FD206807
:102E6000A022662108E000BFC0820020F0100020F0
:102E7000D0600020042D0020FEF7D6FD206801223E
:102E8000FF21FEF7D1FD206832222221FEF7CCFD82
:102E9000206814224721FEF7C7FD2068FF22492140
:102EA000FEF7C2FD206800224A21FEF7BDFD206822
:102EB0000022FF21FEF7B8FD20680A227A21FEF7E2
:102EC000B3FD206800227B21FEF7AEFD20682122A1
:102ED0007821FEF7A9FD20680122FF21FEF7A4FD5D
:102EE000206834222321FEF79FFD20680022422122
:102EF000FEF79AFD2068FF224421FEF795FD206829
:102F000026224521FEF790FD206805224621FEF786
:102F10008BFD402211462068FEF786FD20680622C0
:102F20000E21FEF781FD20681A222021FEF77CFD8C
:102F3000206840224321FEF777FD20680022FF2110
:102F4000FEF772FD206803223421FEF76DFD206834
:102F500044223521FEF768FD20680122FF21FEF79B
:102F600063FD206804223121FEF75EFD20680922FE
:102F70004B21FEF759FD206805224C21FEF754FD38
:102F8000206804224D21FEF74FFD20680022FF211A
:102F9000FEF74AFD206800224421FEF745FD206827
:102FA00020224521FEF740FD206808224721FEF738
:102FB0003BFD206828224821FEF736FD20680022CC
:102FC0006721FEF731FD206804227021FEF72CFDF9
:102FD000206801227121FEF727FD2068FE22722160
:102FE000FEF722FD206800227621FEF71DFD2068F5
:102FF00000227721FEF718FD20680122FF21FEF74D
:1030000013FD206801220D21FEF70EFD206800222D
:10301000FF21FEF709FD206801228021FEF704FD53
:103020002068F8220121FEF7FFFC20680122FF2121
:10303000FEF7FAFC206801228E21FEF7F5FC2068DD
:1030400001220021FEF7F0FC20680022FF21FEF79C
:10305000EBFC206800228021FEF7E6FC04222068B9
:103060000A21FEF7E1FC256884212846FFF785FC4C
:10307000842100F0EF022846FEF7D6FC01222068EA
:103080000B21FEF7D1FC256801A92846FFF7B2FC09
:1030900005AA01A92846FFF7C2FC9DF80430002BC1
:1030A00000F01C81089D05F684559DF80630002B24
:1030B00000F01781089B03F2B22305EB43059DF84E
:1030C000073023B1BDF8243003F525731D449DF866
:1030D000083023B1BDF8263003F226231D44E82230
:1030E000206847F8C45C0121FEF79EFC2068294651
:1030F00049F0CCF8012220681146FEF795FC2068C3
:103100004021FFF749FC002800F0DF802068012102
:103110000222FEF789FC20680021FFF73DFC002811
:1031200000F0D3802068DFF8D491E8220121FEF777
:103130007BFC206820224421FEF7C5FC256801A9FC
:103140002846FFF757FC05AA01A92846FFF767FCA8
:10315000502257212846FEF767FC082256212846B0
:10316000FEF762FC082250212846FEF75DFCBDF800
:1031700024004FF47A7A48F20E660AFB0060B0FB36
:10318000F9F080B2FEF7FAF9512102462846FEF71F
:103190009AFC089B0AFB0366574B9E429DBFB6FBF9
:1031A000F9F202F1FF32D2B2FF2246212846FEF7A1
:1031B0003BFC57F8C41C284649F068F80121284612
:1031C000FFF7DBFB0222064601212846FEF72CFC16
:1031D00000212846FFF7E0FB324601212846FEF792
:1031E00023FC246801A92046FFF704FC05AA01A9D5
:1031F0002046FFF714FC482211462046FEF714FC37
:10320000082247212046FEF70FFC032232212046E8
:10321000FEF70AFC072230212046FEF705FC0122BA
:10322000FF212046FEF700FC202230212046FEF739
:10323000FBFB0022FF212046FEF7F6FB062220467C
:103240007021FEF7F1FBBDF826304FF47A7246F696
:10325000440002FB03004DF28803B0FBF3F09DF83D
:10326000073080B21BB1BDF81A30184480B2FEF7A7
:1032700085F9712102462046FEF725FC57F8C41C4B
:10328000204649F003F801212046FFF776FB022291
:10329000054601212046FEF7C7FB00212046FFF727
:1032A0007BFB2A4601212046FEF7BEFB642347F83C
:1032B000CC3C012388F8FC3007E0D9F800309BB201
:1032C0009B1BB3F5FA7F7FF6ABAC0AB0BDE8F08785
:1032D0000B41DB0744BF0132D2B21AE540F6363566
:1032E000E3E69DF80530002B3FF4E9AE089B03F5BB
:1032F00025731D44E3E600BF1B280D011C0C0100D3
:10330000F8B53B4F97F8FC300446002B37D0394DC9
:1033100015F8C06C012E33D0022E4FD07EBB006852
:1033200001228021FEF780FB20680122FF21FEF7A9
:103330007BFB206832463146FEF776FB15F8C82C39
:1033400020689121FEF770FB206801223146FEF7CC
:103350006BFB20683246FF21FEF766FB2068324691
:103360008021FEF761FB206801223146FEF75CFBFD
:10337000214B1B6845F8D03C012305F8C03CF8BD43
:1033800000680021FFF7F9FAC20711D555F8CC2CD7
:10339000002AF4D0184B55F8D01C1B689BB25B1A5E
:1033A0009A42ECD2154B4FF0FF325A600023E4E70B
:1033B000114B1B6845F8D03C0223DEE7006813215F
:1033C000FFF7DBFA4307E1D01E212068FEF7F4FE89
:1033D000012206460B212068FEF726FB0A23B6FBD6
:1033E000F3F6064BB6B25E60012387F8FD30DDE7E9
:1033F000D0600020C0820020042D0020F0100020AA
:1034000010B5EFF31181102383F312884FF0E023FE
:10341000C9B29C691A6912F4803F0D4A1EBF01208F
:10342000C2F8040F9C690B4B1868D2F8043F81F373
:103430001188D2F8081F4FF47A72034402FB01F09E
:10344000001BB0FBF1F00021E3FB020110BD00BF47
:10345000C8710020042D0020124B5B68C3F30803E1
:1034600030B4EBB9EFF31183D3B90F490F4B4FF0E1
:10347000E0250A68AC6908688242FAD1D3F8000FE7
:103480008442F6D8D3F8081F4FF47A7303FB01F097
:10349000001BB0FBF1F00021E2FB030130BC7047E0
:1034A00030BCADE700ED00E0042D0020C871002025
:1034B00010B5074C14F8B70C40B1FFF7CDFF54F826
:1034C000B03CC01AC0F5FA5020EAE07010BD00BF51
:1034D000C082002010B5044630B1036823B1DB6818
:1034E00013B1BDE810401847FFF7B6FFD4E9042335
:1034F0009042994134BF0120002010BDF8B5064626
:103500000D46FFF7A9FF04460F46FFF7A5FF021B74
:1035100061EB0703B242AB41F7D3F8BD38B50D46B6
:103520000446FFF7C5FF011E02DDC917FFF7E6FFDE
:10353000064B2068002203F8B72C492113F8B63C4B
:103540002A46FEF739FB012038BD00BFC0820020AB
:103550002DE9F341384C54F8A83CC0F8363034F823
:10356000A43C438714F8B83C012B064600F136080A
:10357000A4F1A8070CD0022B26D0A3BB0122022164
:1035800047F0EBFC012304F8B83C14F8A25C10E00F
:10359000FFF78EFF14F8A25C58B969463046FFF772
:1035A000BDFF9DF8003008B19B0706D1002304F849
:1035B000B83C284602B0BDE8F0810722032130461E
:1035C00047F0CBFC0223F2E7FFF772FF0028DCD1C3
:1035D00069463046FFF7A2FF9DF80630054610B158
:1035E00013F0080205D0002504F8B85C04F8A25CCA
:1035F000DFE734F9A01C6846FBF768FC404234F969
:103600009E1CF0860DF10200FBF760FC34F99C1C57
:10361000308701A8FBF75AFCD6F8363044F8A83CAE
:1036200040427087B8F80430BB80012304F8B82CFE
:1036300004F8A23CBDE700BFC082002010B50446DC
:10364000013C00D210BD4FF47A700021FFF756FF05
:10365000F6E738B50568044600212846FCF77AF9F4
:10366000B62214212846FEF7A1F86420FFF7E6FFF2
:10367000812210212068FEF799F80120FFF7DEFF74
:10368000152120688022FEF791F80120FFF7D6FF70
:1036900020680321BDE83840FCF75CB938B50568FF
:1036A000044600212846FCF755F9B6227E2128461B
:1036B000FEF77CF86420FFF7C1FF00227C21206820
:1036C000FEF774F86420FFF7B9FF04227D2120681B
:1036D000FEF76CF86420FFF7B1FF8C2240212068D0
:1036E000FEF764F80120FFF7A9FF022241212068BC
:1036F000FEF75CF80120FFF7A1FF20680221FCF72C
:1037000029F94FF40063A38138BD10B50446406920
:10371000FCF786FC0120FFF791FF6069FCF77BFC5A
:10372000BDE810400A2089E773B50468B6227E21FF
:1037300005462046FEF73AF86420FFF77FFF022196
:103740002046FCF707F92046FFF7DFFF00227C2127
:103750002046FEF72BF80120FFF770FF00225921C9
:103760002046FEF723F80120FFF768FF5E238DF85F
:10377000073094F91030142253433D4AD658A368B9
:103780009A0702D4606948F0C7FE01230DF10702D1
:103790000021304649F0DAFF4FF4A473354A002186
:1037A000304649F0D3FFA3689B0702D42046FDF7BB
:1037B000CDFF0A20FFF742FF012259212046FDF7E5
:1037C000F5FF0120FFF73AFF8C2240212046FDF74C
:1037D000EDFF0120FFF732FF032241212046FDF7D4
:1037E000E5FF0120FFF72AFF234EA96B234A95F836
:1037F0003500B6FBF1F1032389B2FBF7F5FC4388F2
:10380000B6FBF3F62E640279422142F0C002204654
:10381000FDF7CCFF0120FFF711FF082243212046CE
:10382000FDF7C4FF0120FFF709FF042258212046BD
:10383000FDF7BCFF0120FFF701FF0A2253212046BC
:10384000FDF7B4FF0120FFF7F9FE00227C2120469E
:10385000FDF7ACFF0120FFF7F1FE06227D21204697
:10386000FDF7A4FF012002B0BDE87040E6E600BF0E
:10387000B0000020635F060840420F00AC600608FD
:10388000F8B5816B0468294A294FB7FBF1F1054669
:10389000062389B290F83500FBF7A6FC0021438887
:1038A000B7FBF3F706462F642046FCF753F8802257
:1038B0006B212046FDF77AFF6420FFF7BFFE03224D
:1038C00068212046FDF772FF6420FFF7B7FE012252
:1038D0006B212046FDF76AFF0F20FFF7AFFE18228D
:1038E0001B212046FDF762FF0F20FFF7A7FE1822DD
:1038F0001C212046FDF75AFF0F20FFF79FFE32796B
:103900001A212046FDF752FF0F20FFF797FE72792C
:1039100019212046FDF74AFF6420FFF78FFE20465D
:103920000321BDE8F840FCF715B800BFBE600608EB
:1039300040420F00F7B505230468816B654A664F66
:10394000B7FBF1F1054689B290F83500FBF74CFC66
:1039500000214388B7FBF3F706462F642046FBF7A8
:10396000F9FF002276212046FDF720FF0F224E218D
:103970002046FDF71BFF0F20FFF760FE72794F21F5
:1039800002F00F022046FDF711FF0F20FFF756FE51
:103990007279502102F00F022046FDF707FF0F2039
:1039A000FFF74CFE5221FF222046FDF7FFFE0F20BD
:1039B000FFF744FE95F83510072941D0474E96F899
:1039C0000C01FBF75DFC0546012276212046FDF740
:1039D000EDFEAA780C212046FDF7E8FE2A790D219C
:1039E0002046FDF7E3FEAA79AB88120142EA1322D2
:1039F000D2B20E212046FDF7D9FE4FF4807196F821
:103A00000C01FBF73DFC0546022276212046FDF71E
:103A1000CDFEAA78520002F0FE0203212046FDF7F7
:103A2000C5FE2A7904212046FDF7C0FEAA79AB889D
:103A3000120142EA1322D2B205212046FDF7B6FE5A
:103A4000002276212046FDF7B1FE032214212046F4
:103A5000FDF7ACFE0F20FFF7F1FD002263212046A9
:103A6000FDF7A4FE6420FFF7E9FD0822652120464A
:103A7000FDF79CFE0DF1070264212046FEF70CFEC7
:103A80009DF8072022F0100242F0600264212046D7
:103A90008DF80720FDF78AFE0F20FFF7CFFD0DF10F
:103AA00006024D212046FEF7F7FD9DF8062002F0A4
:103AB0003F0242F040024D2120468DF80620FDF7DE
:103AC00075FE0F20FFF7BAFD03212046FBF742FFEA
:103AD00003B0F0BDE260060840420F00D060002055
:103AE000F8B5816B04682D4A2D4FB7FBF1F10546FF
:103AF000062389B290F83500FBF776FB0021438856
:103B0000B7FBF3F706462F642046FBF723FF80221E
:103B10006B212046FDF74AFE6420FFF78FFD072248
:103B200068212046FDF742FE6420FFF787FD002252
:103B30006B212046FDF73AFE6420FFF77FFD01224E
:103B40006B212046FDF732FE0F20FFF777FD18228C
:103B50001B212046FDF72AFE0F20FFF76FFD1822DC
:103B60001C212046FDF722FE0F20FFF767FD32796A
:103B70001A212046FDF71AFE0F20FFF75FFD72792C
:103B800019212046FDF712FE6420FFF757FD20465D
:103B90000321BDE8F840FBF7DDBE00BFBE600608AC
:103BA00040420F009CE710B57822044600210068CF
:103BB000FDF7FCFD0520FFF741FD202201212068D3
:103BC000FDF7F4FD0520FFF739FD002202212068F2
:103BD000FDF7ECFD6420FFF731FD012010BD10B5AD
:103BE000072204460A210068FDF7E0FD0520FFF7E3
:103BF00025FD242241212068FDF7D8FD0520FFF78F
:103C00001DFDC02242212068FDF7D0FD0520FFF7F1
:103C100015FD012010BD10B50122044610210068D9
:103C2000FDF7C4FD48B11420FFF708FD2068A0226D
:103C3000BDE810401121FDF7B9BD10BD13B5044614
:103C400000210068FBF786FE0021204647F06CF952
:103C50001420FFF7F3FC0F21204647F065F90A20F6
:103C6000FFF7ECFC01AA03231021204646F058F987
:103C70000A20FFF7E3FC9DF80420174B803223F85D
:103C8000A02C9DF80520803223F89E2C9DF806205C
:103C900000218032204623F89C2C47F045F90A2069
:103CA000FFF7CCFC0DF1030201230221204646F070
:103CB00037F901230DF103020921204646F030F9BE
:103CC0002046122147F030F920680321FBF742FE1D
:103CD000012002B010BD00BFC082002008B50068FE
:103CE00001220921FDF762FDBDE808406420A5E43A
:103CF00080B506460A2501210846FCF74DFD002146
:103D00000846FCF749FD771C4FF03208052457EAB6
:103D1000040307D14FF47A70FFF790FC013DEAD11C
:103D2000FDF7C9FC0120FCF725FD0020FCF722FD72
:103D30000120FDF768FC4046FFF780FC0120FCF7FE
:103D400019FD0020FCF716FDFDF75DFC4046FFF76E
:103D500075FC44B1013CDAD14FF4FA70FFF76EFC08
:103D60004FF0FA08D3E7013FD1E737B505680446BD
:103D700000212846FBF7EEFD15227E212846FDF79F
:103D800015FD6420FFF75AFC11227E212068FDF703
:103D90000DFD0520FFF752FC20680DF107020321FD
:103DA000FEF77AFC9DF8073003F03C03142B02D099
:103DB0000620FFF79DFF0C2240212068244DFDF7CF
:103DC000F5FC0120FFF73AFCA16B224A94F835007C
:103DD000B5FBF1F1032389B2FBF706FA4388B5FB83
:103DE000F3F52564027920684221FDF7DFFC01200C
:103DF000FFF724FC082241212068FDF7D7FC0120B1
:103E0000FFF71CFC002243212068FDF7CFFC0120B6
:103E1000FFF714FC102251212068FDF7C7FC012098
:103E2000FFF70CFC0A2253212068FDF7BFFC01209C
:103E3000FFF704FC802256212068FDF7B7FC012023
:103E4000FFF7FCFB20680321FBF784FD03B030BDC6
:103E500040420F0000610608F0B5816B0568514AC9
:103E6000514FB7FBF1F185B00446062389B290F8B3
:103E70003500FBF7B9F900214388B7FBF3F7064695
:103E800027642846FBF766FD80226B212846FDF754
:103E90008DFC9620FFF7D2FB032268212846FDF710
:103EA00085FC9620FFF7CAFB03226B212846FDF70D
:103EB0007DFC0F200021FFF721FB10226A212846FC
:103EC000FDF774FC0F200021FFF718FB00226C2186
:103ED0002846FDF76BFC0F200021FFF70FFB7279DE
:103EE00019212846FDF762FC0F200021FFF706FB91
:103EF00018221B212846FDF759FC0F200021FFF74F
:103F0000FDFA18221C212846FDF750FC0F20002145
:103F1000FFF7F4FA32791A212846FDF747FC012011
:103F20000021FFF7EBFA03212846FBF713FD206879
:103F3000062302AA4321FDF73FFED0B1BDF80830A9
:103F4000DBBA07EE903ABDF80A30F8EEE77ADBBA52
:103F5000C4ED077A07EE903ABDF80C30F8EEE77A38
:103F6000DBBAC4ED087A07EE903AF8EEE77AC4EDD2
:103F7000097AD4ED087AFDEEE77ACDED017A9DF964
:103F8000043001330CD1D4ED077AFDEEE77ACDEDA4
:103F9000017A9DF90430013302D10620FFF7A8FE13
:103FA00005B0F0BDBE60060840420F0018B10368BE
:103FB0005B6803B11847FF20704718B103689B681E
:103FC00003B118470020704770B450B106798E4293
:103FD00007D34579954204D30368DB680BB170BC05
:103FE000184770BC704710B440B184798C4205D337
:103FF00003681B6913B15DF8044B18475DF8044B67
:10400000704718B103685B6903B11847704718B16E
:1040100003681B6A03B118470020704730B50A4691
:1040200058B1041D00F1140320686168154603C5EA
:1040300008349C422A46F7D1012030BD10B50C4609
:1040400070B92D2300202375094B2061C4E90000BD
:10405000C4E90200C4E90633302384F8203010BDDF
:104060000368DB6A002BECD098470028E9D0F6E71C
:104070008F3B070838B5054D441E14F8011F01B9E0
:1040800038BD55F8980CFBF727FCF6E7C0820020F6
:1040900070B50E4C0E4605460D48FFF7EBFF334654
:1040A0000C4954F8980C2A4649F0D0FB54F8980C67
:1040B000FBF706FC14F8943C3BB1012304F8933C55
:1040C00014F8923C013304F8923C70BDC082002089
:1040D00070060708F9F8000808B50648FFF7CAFF98
:1040E000054B33F8900C18B1BDE80840FFF7A6BAAD
:1040F00008BD00BF555D0708C082002010B5074C01
:1041000002460B4654F8980C054949F09FFB54F8B9
:10411000980CFBF7D5FBBDE81040DDE7C08200201E
:10412000F9F8000808B5FFF7A5FFBDE80840D3E798
:1041300010B504460948FFF79DFF2046FFF79AFF98
:10414000074B13F8942C3AB1012203F8932C13F87F
:10415000922C013203F8922C10BD00BF70060708A4
:10416000C082002010B504460348FFF783FF2046B5
:10417000BDE81040D6E700BF7C0607080CB48306F4
:1041800007B500D551B9049805A90191FFF7B6FF0D
:10419000012003B05DF804EB02B070470020F8E79F
:1041A000024B014653F8980CFBF796BBC0820020E7
:1041B0000CB407B510F0400009D069B92320FFF70F
:1041C000EFFF049805A90191FFF798FF012003B0C4
:1041D0005DF804EB02B070470020F8E70FB413B5A8
:1041E000094C0A4954F8980C04AB53F8042B01937A
:1041F00049F02CFB54F8980CFBF762FB02B0BDE8C9
:10420000104004B0704700BFC0820020F9F80008D9
:104210000FB407B504A951F8040B0191FFF76EFF25
:1042200003B05DF804EB04B070470FB407B504A900
:1042300051F8040B0191FFF72BFFFFF74DFF03B07F
:104240005DF804EB04B0704770B5C379164603F00F
:1042500007028CB00446062A4FD8DFE802F00414A7
:1042600017191C1E49000D7813F0C00347D0402BCE
:104270003CD12946204615F0A9FD002859D00CB0A4
:10428000BDE87040AAE791F90050EDE70D88EBE733
:10429000B1F90050E8E70D68E6E791ED000A6846DD
:1042A000FAF764F801462848FFF798FFF6B1E3797A
:1042B0003F2B1BD8204615F0E1FC00EE100A6846A3
:1042C000B8EEC00AFAF752F801462048FFF786FF19
:1042D000204615F0E3FC00EE100A6846B8EE400AEE
:1042E000FAF744F801461948FFF778FF0CB070BDA3
:1042F00015480CB0BDE8704070E70025B4E7042A0B
:104300000CBF134813482946FFF768FF002EEDD075
:10431000E3793F2BEAD8204615F0B0FC054620464D
:1043200015F0BCFC02460C4829460CB0BDE87040B4
:1043300054E76946204615F06FFB08486A4629464F
:10434000FFF773FFD2E700BF560F0708550F0708A6
:10435000CD060708B73A0708285F0708810607084F
:104360002DE9F04F8FB001F020034C4C00938146B3
:104370000F464FF000084A4B53F8980CFBF7A0FA91
:1043800094F807B00BF038034B4549D1204615F09F
:10439000FDFBFAF73BFA8568204615F023FC8246C0
:1043A0002E18204615F05EFC0BF007020146062A87
:1043B0006CD8DFE802F0044045494E525E0015F823
:1043C0000A200978511A4A424A41009B03B13ABB7C
:1043D00002A92046019215F01FFB7B0615D5019A14
:1043E0009AB9304802A9FFF7F9FE2F4902A849F00F
:1043F000E5FB00284CD115F80A30202B48D12B487A
:104400003146FFF7EBFEFFF767FE294802A9FFF7E9
:10441000E5FE002231462046FFF716FFFFF75CFE5F
:1044200008F1010840F28523984504F10C04A2D15B
:104430000FB0BDE8F08F15F90A2091F90010C1E71F
:1044400035F80A200988BDE735F90A20B1F90010CE
:10445000B8E755F80A200968B4E796ED007AD1ED7F
:10446000007AB4EE677AF1EE10FA0CBF0122002256
:10447000ABE72046019115F011FC0199421C304632
:104480004EF0EAFFB0FA80F252099EE700229CE764
:10449000002231462046FFF7D7FEB4E760630608E6
:1044A000C08200209E060708EB5E0708D60C0708AE
:1044B0009F06070838B50D46044615F0D3FB2A467B
:1044C00001462046BDE83840BEE6F8B5C47914F090
:1044D000C003064602D0402B15D0F8BD15F0DEFB18
:1044E00004F00704062C054604D10146BDE8F84057
:1044F00012488DE6304615F0C1FB2A460146BDE85C
:10450000F8400F4884E615F051FC05460D480E4E64
:104510000E4FFFF7AFFD00242B79A34202D8BDE870
:10452000F840D9E514B13046FFF7A4FD2B683846B2
:1045300053F82410FFF752FE0134EDE7A9060708EF
:10454000B9060708D0060708E0060708550F070850
:1045500008B50548FFF78EFD044B53F8980CBDE8ED
:104560000840FBF7ADB900BF7C060708C0820020F9
:1045700000485AE6E206070813460A460146014883
:1045800053E600BFEE06070820B10078B0FA80F0CD
:1045900040097047012070472DE9F04F87B003466E
:1045A000FFF7F2FF054618B107B0BDE8F04FDFE7AF
:1045B0005D49DFF8A8A1DFF870B105AA18464EF0F2
:1045C000A4FF2F4681462C46A8464FF0FF36B9F18E
:1045D000000F12D14FFA86F948461FF071FE10B154
:1045E0004568002D79D1B8F1000F55D14F483146BB
:1045F000F9F7BFF907B0BDE8F08F032D07D8DFE862
:1046000005F0020E132D4846F9F7A0FF064605AA4D
:10461000594600204EF079FF01358146D7E74846DC
:10462000F9F794FF8046F2E74149484650F0D1FF40
:1046300020B94049484650F0CCFF08B144F001048D
:104640005146484650F0C5FF28B93B49484650F00E
:10465000C0FF0028DBD044F00204D8E7484649F008
:1046600007FB032816D199F80020382A12D199F8AF
:104670000120452A0CD04E2A0CD1002299F8023094
:10468000312B03D0322B05D142F002021743BEE793
:104690000422F3E7FF22F9E7002C08BF03240023DC
:1046A000E4B2CDE9008402971A46194648461FF045
:1046B000C5FF054610B92148314699E720484246D2
:1046C0003146F9F756F931461E48F9F752F91E4BB3
:1046D000294653F88C0C44F023F81C483146F9F76E
:1046E00048F95CB16979A14208D019482246F9F726
:1046F00040F92B68E1B29B69284698475FB1A979D8
:10470000B94208D013483A46F9F733F92B683946CD
:10471000DB6928469847EB6A002BD4D00E48F9F79E
:1047200028F90023EB62CEE7AE5707080E0707080B
:10473000001D0708EB4007083C200708360707085C
:1047400055070708E3070708C0820020720707081B
:104750008A070708AA070708CD0707080B070708F5
:104760002DE9F04F85B00546FFF70EFF044630B146
:104770000021012005B0BDE8F04F44F081B8864922
:104780002846F9F7AFFA20B905B0BDE8F04F3DF083
:104790000BBA82492846F9F7A5FA28B9012005B0D5
:1047A000BDE8F04F3DF06EBB7D492846F9F79AFA17
:1047B00098BB7C4B93F9B32F83F8AC0F03F5C4710E
:1047C00091F8D654012D09D0033D052D06D90CB121
:1047D00083F8B32F05B0BDE8F04FC9E691F8D75480
:1047E000A52D00F1010013D1012A0ED16E4983F8E5
:1047F000AC2F002283F8AD0F01F8882C83F8B32F7B
:1048000005B0BDE8F04F3DF085BB013A52B201243E
:10481000782801F11401D3D1D9E72846F9F796FE9B
:10482000614B13F9883C009303FA80F6772E834698
:1048300000F2A7802846FAF7A9FF0746002800F0F3
:104840008C80F9F783FE0124C5B23846FAF79EFF43
:104850000746002800F08480F9F778FE01340190C3
:10486000E4B23846FAF792FF804600287AD0F9F78A
:104870006DFE01340746E4B24046FAF787FF8146F1
:10488000002871D0F9F762FE01340290E4B2484684
:10489000FAF77CFF8246002868D0F9F757FE01340A
:1048A0000FFA80F9E4B25046FAF770FF824600280A
:1048B0005ED0F9F74BFE01340FFA80F8E4B25046AF
:1048C000FAF764FF002855D00390F9F73FFE039AEA
:1048D0000FFA80FA1046FAF759FF0346002857D01E
:1048E00004F0FD04F9F732FE042C7FF473AFC3B279
:1048F000012D03D9EA1E052A3FF66CAF23B1A52B83
:1049000002D0482B7FF466AF26480EB980F8B36F0B
:10491000142202FB06020199C2F84C16A52B02993B
:1049200082F85E56C2F85076C2F85416A2F858962D
:10493000A2F85A86A2F85CA682F85F360AD1009BDC
:10494000194A01335B4402F8883C90F8B33F0133C5
:1049500080F8B33F05B0BDE8F08F0446054674E724
:1049600001907EE7074687E7029090E781469AE745
:104970008046A4E75FFA88F382468046062CB7D0CB
:1049800028E70A487722214605B0BDE8F04FF3E555
:104990000134E4B2F2E700BF11080708170807085E
:1049A000541B0708D0600020C08200201C080708A4
:1049B00010B50346FFF7E8FD30B1FCF773F8BDE82A
:1049C00010400748FFF7AEBB1846F9F7BFFD044695
:1049D00080B2FCF73BF821460248BDE8104017E4DE
:1049E000250807083108070808B50346FFF7CCFD7E
:1049F00040B10C4B0C48002223F8902CBDE8084035
:104A0000FFF790BB1846F9F7A1FD014638B1054BF9
:104A100023F8900CBDE808400448FFF7F9BBBDE857
:104A20000840A5E5C0820020430807085908070888
:104A30002DE9F04F834689B090460C461646002774
:104A40004FF0190A4FF46179B8F1000F4BD030786C
:104A500025787178B378F278854242D165788D42B5
:104A60003FD1A5789D423CD1E578A5EB020CDCF165
:104A7000000545EB0C05CDE90632059114F0F0F880
:104A8000079A069B059901911AFB02921AFB039360
:104A90000392029343790093144A3B4629465846B1
:104AA000FFF786FB207814F0DBF8E3780F4A1AFB57
:104AB00003930393A3781AFB039302936378019300
:104AC0004379009329463B4658460137FFF756FB8A
:104AD000282F04F1040406F10406B5D109B0BDE89D
:104AE000F08F0025C7E74546DCE700BF70080708E0
:104AF000F7B50746FFF748FD044630B12E490022BE
:104B0000012003B0BDE8F04092E73846F9F71EFDFA
:104B10002728054648DC8600781C8DF80740FAF700
:104B200035FE074690B1F9F711FD031E0EDB234A4F
:104B30002146DBB202F2545404EBC10CC8009CF8CD
:104B400005C09C4525D001313D29F5D13846FAF7FD
:104B50001DFE044660B1F9F7F9FC1D2808D8184B72
:104B6000334403F8860C9DF8073001338DF8073085
:104B7000114FB11C0DF1070239442046FAF713FE1C
:104B80009DF80730042B02D0002347F8253003B0EE
:104B9000F0BD0B4B0244334492F8582503F8872CA0
:104BA00001238DF80730D1E706482722214603B0BC
:104BB000BDE8F040E0E400BF39820020C05B060899
:104BC000C0820020860907082DE9F04F3F4FDFF82B
:104BD00004A189B0814690460C46164602F1300B7E
:104BE00094F9045000230C22394802FB03F10956C2
:104BF000A94266D00133042BF6D10C36B34504F13B
:104C00000C04EDD109B0BDE8F08F96F90430D6F868
:104C100000E07279B179307A96F807C007939D4227
:104C20004DD1256875454AD16579954247D1A57919
:104C30008D4244D1257A854241D1E579A5EB0C031B
:104C40005D425D4107EB820207EB8C0C07EB8000B5
:104C500007EB8101D2F83C27DCF83C37D0F83C0761
:104C6000D1F83C170493CDE900E203900291079B31
:104C7000524629464846FFF79BFAE27994F90430F8
:104C800007EB82022946D2F83C270492227A07EBEE
:104C900082024846D2F83C270392A27907EB8202AF
:104CA000D2F83C270292627907EB8202D2F83C27C5
:104CB0000192226800925246FFF760FA9DE70025B4
:104CC000C0E7B8F1000FA0D14546D6E7C05B0608A3
:104CD000DC820020830807082DE9FF410346FFF727
:104CE00053FC30B145490022012004B0BDE8F04139
:104CF0006AE718465E1CF9F729FC044640B21FF02B
:104D00005BFC054630B93E48214604B0BDE8F041A1
:104D1000FFF78BBA0068696801AB03C3A868186025
:104D20003046FAF733FD0446002853D003782B2B86
:104D300005D02D2B43D0F9F709FC019009E001348F
:104D40002046F9F703FC012303FA00F0019B03431B
:104D5000019302262B4F4FF000082046FAF716FD6C
:104D6000044628B3F9F7F2FB274A002352F8041B44
:104D7000884231D00133112BF8D1002307EB830295
:104D8000D2F83C27904213D1B8F1020F26D0B8F1E7
:104D9000030F26D0B8F1010F14BF8DF809308DF83C
:104DA0000A3008F101080136B8F1040FF6B2D4D187
:104DB000012E19D804B0BDE8F041FFF7D9BB01348A
:104DC0002046F9F7C3FB012303FA00F0019B23EA15
:104DD0000003BDE70126BDE7DBB2CFE78DF80C305D
:104DE000DFE78DF80B30DCE701AB03CB28601868F8
:104DF0006960A86004B0BDE8F08100BF0C830020AA
:104E0000A0080708C05B0608FC6206082DE9F04F01
:104E1000834687B090460C46164600274FF0190A85
:104E20004FF46179B8F1000F4DD0B078A5783378A0
:104E3000727896F803C096F804E07179854240D103
:104E400025789D423DD1657895423AD1E578654512
:104E500037D12579754534D165798D4214BF002548
:104E600001251AFB02921AFB0393CDE90103039279
:104E70000091CDE904CE154A3B4629465846FFF736
:104E800097F923790593E378049363780F4A1AFB23
:104E90000393039323781AFB03930293A37801935C
:104EA0006379009329463B4658460137FFF766F978
:104EB000142F04F1060406F10606B3D107B0BDE8CD
:104EC000F08F0025CDE74546DBE700BFB3080708B4
:104ED0002DE9F3478246FFF757FB064630B13E49BE
:104EE0000022012002B0BDE8F0478FE75046F9F7F5
:104EF0002DFB1328054663DC062747430AF1010012
:104F00008DF80760354CFAF741FC04F1800909EB94
:104F10000708064648B1F9F719FB03289FBFE319B4
:104F200083F8850001238DF807303046FAF72EFC10
:104F3000064668B1F9F70AFB1D2809D8062303FBCA
:104F4000054383F882009DF8073001338DF8073060
:104F50000DF1070241463046FAF725FCFAF716FC38
:104F6000064668B1F9F7F2FA3C2809D89DF80730EF
:104F7000062202FB0542013382F883008DF80730D8
:104F80003046FAF703FC68B1F9F7E0FA1D2809D8B2
:104F90009DF80730062202FB0544013384F88400A3
:104FA0008DF807309DF80730062B11D0002349F803
:104FB0000730A8F8043002B0BDE8F047FFF7D8BAD0
:104FC00007481322314602B0BDE8F047FFF7D4BAD4
:104FD00002B0BDE8F08700BF40830020C0820020FF
:104FE000860907082DE9F04F2DED088BDFF814A195
:104FF00097B0074690460C461546002694ED008A69
:10500000B5EE408AF1EE10FA73D0D4ED019A94ED2A
:10501000029AD4ED038AB8F1000F40D095ED000A52
:1050200095ED01BAD5ED02AA95ED03AAB4EE408A3A
:10503000F1EE10FA62D1F4EE4B9AF1EE10FA5DD176
:10504000B4EE6A9AF1EE10FA58D1F4EE4A8AF1EE13
:1050500010FA0CBF4FF001094FF0000912A8F9F740
:1050600085F9B0EE4B0A83460EA8F9F77FF9B0EE4A
:105070006A0A05900AA8F9F779F9B0EE4A0A04908D
:1050800006A8F9F773F9059B049A0390CDE900B3DC
:1050900002923346524649463846FFF789F8B0EE49
:1050A000480A12A8F9F762F9B0EE690A81460EA81B
:1050B000F9F75CF9B0EE490A83460AA8F9F756F900
:1050C000B0EE680A049006A8F9F750F9049B039023
:1050D000CDE901B3CDF80090334652460021384661
:1050E0000136FFF74BF80C2E04F1100405F1100502
:1050F00084D117B0BDEC088BBDE8F08F4FF00009EC
:10510000ACE700BFD1080708F8B50546FFF73CFA41
:10511000064668B1434991F8A2324FF4D47202FBBB
:105120000311BDE8F840002201F58471012059E720
:105130003D4905222846F8F7BBFD78B9394A02F106
:10514000F80392F8A2224FF4D47101FB02330C222F
:105150000021013A43F8101FFBD1F8BD2846F9F7AA
:10516000F5F90B28044656D82846FAF70FFB0646F1
:1051700000283DD0F9F75EF92A4A92F8A2324FF49E
:10518000D470611C434303EB01131A4482ED3E0AC1
:1051900001253046FAF7FAFA064670B1F9F74AF9EE
:1051A000204A92F8A2324FF4D470611C434303EBBF
:1051B00001131A4482ED3F0A01353046FAF7E6FA48
:1051C000064668B1F9F736F9164A92F8A2324FF45A
:1051D000D4714B4303EB04131A4482ED440A0135A6
:1051E0003046FAF7D3FA28B9BDE8F840FFF7C0B95E
:1051F0000546CEE70B4E96F8A272F9F71BF94FF46D
:10520000D4737B4303EB04143444032D84ED450A2B
:10521000EAD1F11885E731460448BDE8F8400B2291
:10522000FFF7AAB9C08200201108070886090708FD
:105230002DE9F347DFF868A081460E4617464FF088
:105240000208002457B337F8243036F8241037F812
:105250000820994220D136F80850A91A4D424D41F4
:10526000CDE900322946234652464846FEF7A0FFC4
:1052700036F80830019336F824300093524623461E
:10528000294648460134FEF779FF042C08F104084A
:10529000D8D102B0BDE8F0870025E1E73D46E7E759
:1052A000E5080708F8B50446FFF76EF9054628B18A
:1052B000BDE8F8402A4900220120B9E729492046E3
:1052C000F8F710FDA8B9284B4FF47A714FF4FA6241
:1052D000A3F8C812A3F8CA22A3F8CC12A3F8CE22CE
:1052E000A3F8D012A3F8D222A3F8D412A3F8D6229E
:1052F000F8BD2046F9F72AF90328064628D82046A3
:10530000FAF744FA044670B1F9F720F90127054687
:105310002046FAF73BFA10B1F9F718F937B9BDE8AA
:10532000F840FFF725B905460746F1E7A5F2EE225A
:1053300040F2DC539A42F2D8A0F2EE229A42EED822
:10534000094B03EB8603A3F8C852A3F8CA02CFE7C0
:1053500029460648BDE8F8400322FFF70DB900BF13
:105360008885002011080708C0820020F608070879
:105370002DE9F04F91B0174607900C4615460026D0
:1053800004F115090DF1240B04224946584650F04A
:10539000FDF800238DF82830D4E90232082B72F191
:1053A00000010DF12C0A55D22F491A465046F8F744
:1053B000FDFA002F56D095F80080237843454ED152
:1053C000D4E90202D5E902139A4208BF884246D1C5
:1053D000227D2B7D9A4242D1042205F115014846D7
:1053E00050F088F800283AD121692B69CB1AD3F103
:1053F000000949EB03091D4B059300230493B5F9FC
:1054000012300393B5F910300293194B194A0798DB
:10541000CDE9008349463346FEF7CAFECDF814B005
:10542000237D0493B4F912300393B4F91030114A78
:105430000798CDE901A314F8203B00934946334671
:105440000136FEF79BFE082E05F1200598D111B01C
:10545000BDE8F08F08495046F8F7A8FAA9E74FF0E1
:105460000009C8E7B946D9E7B73A07081D25070874
:105470001B45070809090708FE0807082DE9F74F2B
:105480000446FFF781F8074630B16F49002201203A
:1054900003B0BDE8F04F6BE76C492046F8F722FCFB
:1054A000014638B968484FF4807203B0BDE8F04F48
:1054B0004FF078B92046F9F749F883B2072B054633
:1054C00000F2B9802046FAF761F9824600284CD0F4
:1054D000F9F73CF801240FFA80F95046FAF756F92B
:1054E00068B14FF00008411E00F1100C464611F85B
:1054F000013F13F0DF0F3BD101270134E4B2FAF78B
:1055000045F9824600284CD0F9F720F801340FFA0B
:1055100080FBE4B25046FAF739F90346002842D03E
:105520000190F9F713F80134019B0FFA80FAE4B205
:105530001846FAF72BF90346002836D00190F9F700
:1055400005F80134019B42B2E4B218460192FAF721
:105550001DF9019A034650B30134E4B2032C28D854
:1055600003B0BDE8F04FFFF703B804468146B4E747
:105570006145C2D0A3F13002D2B2092A05D9A3F104
:105580006102052A07D8573BDAB2360146EA187697
:1055900042EA0818ABE7A3F14102052AADD8373B30
:1055A000F2E78346B6E78246C2E70246CDE7284BDC
:1055B000D4E71FFA89F10229D2D80BF2262189B249
:1055C000B1F5E16FCCD80AF2262189B2B1F5E16FCD
:1055D000C6D8D4B2062CC3D81846019348F048FB6D
:1055E0000428BDD8002FBBD01A4A019B2DB202EB74
:1055F000451102EB4512184D81F8D892C1E9B886E1
:10560000A1F8E8B2A1F8EAA281F8EC4202F53B72F7
:10561000591E033311F8010F2C5C04F00304022C13
:1056200008BF203802F8010F087808B18B42F1D189
:1056300003B0BDE8F08F09480722394603B0BDE842
:10564000F04FFEF799BF00BF9885002011080708AA
:105650001D250708C0820020A96007082A0907083D
:105660002DE9F04FDFF8AC9087B0834690460C46AA
:1056700016460027B8F1000F49D0707A617AB6F962
:105680000AC0B6F90CE096F808A08142D6E90032CB
:105690003BD12168994238D16168914235D1B4F942
:1056A0000A10614531D1B4F90C1071452DD1257A1C
:1056B000A5EB0A014D424D41CDE90032CDE9020C86
:1056C000CDE904EA3B464A4629465846FEF770FDB6
:1056D000237A0593B4F90C300493B4F90A30039398
:1056E000637A02936368019354F8103B00934A462F
:1056F0003B46294658460137FEF740FD112F06F17B
:105700001006B7D107B0BDE8F08F0025D4E74546B5
:10571000DEE700BF370907082DE9F74F0446FEF71B
:1057200033FF054630B14E490022012003B0BDE8E9
:10573000F04F95E74B492046F8F7D4FA30B94FF0CF
:10574000FF3003B0BDE8F04F3EF0FEBF2046F8F753
:10575000FDFEC3B2102B834607D9434810222946C9
:1057600003B0BDE8F04FFEF707BF2046FAF70EF88A
:105770000646E8B1F8F7EAFE012482463046FAF719
:1057800005F80646B8B1F8F7E1FE01348146E4B207
:105790003046F9F7FBFF064600285AD0F8F7D6FE48
:1057A0000128804609D903B0BDE8F04FFEF7E0BEFE
:1057B00004468246E2E78146EAE70134E4B2304635
:1057C000F9F7E4FF0646002845D0F8F7BFFE00F5DC
:1057D000B473B3F5347F0746E5D80134E4B23046FC
:1057E000F9F7D4FF0346002837D00190F8F7AEFE52
:1057F00000F5B472B2F5347F0646D4D80134019B6B
:10580000E4B21846F9F7C2FF034640B10190F8F739
:105810009DFE0134051E019B18BF0125E4B2184608
:10582000F9F7B4FF08B10134E4B2062CBBD10F4B39
:105830004FFA8BFB03EB0B13C3E9F6A983F8E18363
:10584000A3F8E273A3F8E46383F8E05303B0BDE880
:10585000F08F8046B3E70746C1E70646D1E700BFB1
:10586000988600201108070857090708C082002001
:105870002DE9FF47DFF87090804617460D46164623
:105880004FF0000A77B3337829789942D6E901209E
:1058900026D16968914223D1AC68211A4C424C410F
:1058A000CDE9012000934A46534621464046FEF783
:1058B0007FFCAB6802936B68019315F80C3B009377
:1058C0004A465346214640460AF1010AFEF756FC75
:1058D000BAF1080F06F10C06D4D104B0BDE8F08788
:1058E0000024DDE73C46E4E7680907082DE9F843B2
:1058F0000446FEF749FE054628B1BDE8F8432E49A7
:1059000000220120B4E72D492046F8F7EBF90146C3
:1059100028B9BDE8F843284860224EF043BF20462E
:10592000F8F714FEC3B2072B064606D929462448C9
:10593000BDE8F8430722FEF71FBE2046F9F726FF11
:10594000074628B3F8F702FE051E18BF01250124FB
:105950003846F9F71BFF0746E0B1F8F7F7FD0134C9
:105960008046E4B23846F9F711FF0746A0B1F8F7D0
:10597000EDFD01348146E4B23846F9F707FF08B17E
:105980000134E4B2032C09D0BDE8F843FEF7F0BDC2
:105990000446DDE78046E5E78146EDE7094B76B250
:1059A0000C2202FB063686F8E854C6F8EC84C6F8EA
:1059B000F094BDE8F88300BFA8870020110807080D
:1059C0007D090708C08200202DE9F04FDFF88490A0
:1059D00091B007468846164600240DF12C0A04EBC8
:1059E000840508EB050358F805001B790290514621
:1059F00002A88DF80C3042F0F1FE4EB373197059C5
:105A00001B790490052204A902A88DF814304FF0E8
:105A100071FD0DF1180BB0FA80F5594604A86D0917
:105A200042F0DCFECDF800B023464A46294638460F
:105A3000FEF7BEFB2346CDF800A04A46294638466D
:105A40000134FEF79BFB802CC9D111B0BDE8F08F6B
:105A50003546EFE78C0907082DE9F04F89B0054678
:105A6000FEF792FD044630B163490022012009B0DF
:105A7000BDE8F04FA8E72846F8F768FD7F280646FE
:105A800000F3B2802846F9F781FEB3005A4A039327
:105A900006EB8603D118D450584B0C71CDE9014365
:105AA0000546A346A146A2462746A046029B05AA54
:105AB00013F8010B029394460023AE4615F8011B20
:105AC00019B1884201D00A2B0CD120336B444FF01E
:105AD0000005884203F80C5C08D009B0BDE8F04F1F
:105AE000FEF746BD0CF8011B0133E6E708F1FF3372
:105AF0000EF10105032B31D8DFE803F0591B026ECC
:105B00004FF0010C12F8011B61B33D48002310F85F
:105B100001EB8E455AD00133082BF8D139480023C8
:105B200010F801EB714553D10CFA03F349EA03096C
:105B3000E8E7012112F8013BA3B14E2B3CD0452BE5
:105B40003CD0532B3CD0572B3CD0552B3CD0442B36
:105B5000F0D1052301FA03F31F43EBE705A8F8F79B
:105B6000F5FC834608F101085FFA88F8B8F1050FE3
:105B70009CD10399244B019A3144581803F5A96329
:105B80000B4402F00F0204F00F0444EA071442EA47
:105B90000B123F1180F8482580F849A580F84A95F6
:105BA000DC701F7109B0BDE8F04F2EF015BF05A8DD
:105BB000F8F7CCFC0190D5E70023CBE70123C9E738
:105BC0000223C7E70323C5E70423C3E79A46A5E7F3
:105BD0000133072BA4D195E705A8F8F7B7FC1028E7
:105BE0000446A8BF0024BDE708487F22214609B02B
:105BF000BDE8F04FFEF7C0BC0888002040630608EF
:105C0000456306084D630608C08200208609070820
:105C10002DE9FF47DFF86C90804617460D46164683
:105C20004FF0000A67B333882A889A4226D16C88DD
:105C30007288A21A54425441F2780292B2782146F4
:105C4000CDE90032404653464A46FEF7B1FAEB78BA
:105C50000293AB78019335F8043B00934A465346D0
:105C6000214640460AF1010AFEF788FABAF1100F00
:105C700006F10406D6D104B0BDE8F0870024DBE7C6
:105C80003C46E4E7960907082DE9F0410546FEF792
:105C90007BFC044628B1BDE8F041244900220120E4
:105CA000B6E72846F8F752FC0F28064636DC2846A9
:105CB000F9F76CFD1E4FDFF884800546A0362846B4
:105CC000F8F744FC37F8023B98421FDC012C08EB44
:105CD000860311D0022C12D0A3F8480528462C21A7
:105CE0004FF027FC054668B10135012301346BB143
:105CF000032CE4D1BDE8F08183F84A05EEE783F890
:105D00004B05EBE7A21E53425341EFE7094B00223C
:105D100043F82620BDE8F041FEF72ABC214606489C
:105D2000BDE8F0410F22FEF727BC00BF888A0020A3
:105D3000546306080888002086090708C0820020EE
:105D40002DE9F04FDFF8B49085B00646884614463A
:105D50004FF0000B062303FB0BF505F5307500270C
:105D600018F805A0002C44D0625DAAEB0200414265
:105D70004141CDE900725B464A4630460391FEF749
:105D800017FA0399CDE9007A5B464A463046013757
:105D9000FEF7F4F9062F05F10105E1D10BF1010B36
:105DA000BBF1060FD6D1DFF854904FF4397518F8CF
:105DB00005B0A5F5397AF4B1635DABEB0302574248
:105DC0005741CDE900A34A46062339463046FEF73F
:105DD000EFF90623CDE900AB4A4639463046FEF7D7
:105DE000CDF9013540F2ED239D42E0D105B0BDE88B
:105DF000F08F2146C6E72746EBE700BFA809070852
:105E00007FB50346FEF7C0FB044630B119490022B6
:105E1000012004B0BDE8704092E71749164E6A466B
:105E200018464DF072FB01AD80B1032C03D1FEF793
:105E30009FFB04B070BDF8F789FB6A4645F8040B78
:105E40003146002001344DF060FBEDE7032CEED12C
:105E5000DDE90145039E29463246E0B22EF01CFFE3
:105E60000028E4D0054833462A462146FEF7D0F9FB
:105E7000DFE700BF08880020AE570708A809070819
:105E80002DE9FF47DFF89890804617460C461646E6
:105E90004FF0000A002F41D0B6F90030B4F90010DD
:105EA000B6F90220B6F9040096F906C0994233D13A
:105EB000B4F9021091422FD1B4F9041081422BD1D0
:105EC00094F90610A1EB0C0569426941CDE9003255
:105ED000CDE9020C53464A4640460D46FEF768F9A6
:105EE00094F906300393B4F904300293B4F9023004
:105EF000019334F9083B00934A46534629464046ED
:105F00000AF1010AFEF73AF9BAF1120F06F1080692
:105F1000C0D104B0BDE8F0870021D7E73D46DFE7F8
:105F2000BC09070830B585B00546FEF72DFB0446D1
:105F300010B32E490022012005B0BDE830409FE794
:105F40002D2B03D0A3F13002092A4AD8042C04DDFA
:105F500005B0BDE83040FEF70BBB2846F8F7F6FA6F
:105F600004AB621C03EB440424F80C0C15F8013F4D
:105F7000303B092BFAD914462B78002BE0D1052CA5
:105F8000E6D1BDF80430BDF90450112BE0D8BDF9BD
:105F90000600A0F5FA739BB2B3F5FA6FD8D8BDF935
:105FA0000810A1F5FA739BB2B3F5FA6FD0D8BDF91A
:105FB0000A209042CCDC9142CADBBDF90C4004F1CE
:105FC0007D039BB2FA2BC3D8094B03EBC503A3F89F
:105FD0003608A3F83818A3F83A2883F83C4805B0E7
:105FE00030BD202BB4D101352246C4E7F68A00200B
:105FF000C0820020034B9A780021101A997018BFB4
:10600000012070476085002010B5114B014603F157
:10601000180253F8044B41F8044B9342F9D11B8802
:106020000B800B4900F11A0351F8044B43F8044B61
:106030009142F9D111881980054B343053F8041B73
:1060400040F8041B9342F9D11B88038010BD00BFA8
:10605000A0810608104A117A537A0B43D17C0B4376
:1060600051780B4391780B43D1780B4311790B4353
:10607000917B0B43917E0B4392F823100B4392F8D4
:106080002F100B4305D192F84100013818BF0120B1
:1060900070470120704700BF68CC002070B5234CCA
:1060A00094F8523005460E4643B1D4E91623904287
:1060B00071EB030324BF002384F85230636F1C4844
:1060C000984710F0010320D080F00203C3F340038F
:1060D00084F85230D4E91A325B1946EB0206C4E95F
:1060E0001636012384F88830430744BF012384F81F
:1060F0008930D4F89030ED1A002D0FDD012384F89B
:106100008830012000F0010070BD8207ECD594F8C2
:106110005220002AE8D084F85230E5E794F888301D
:10612000002BEED194F88900ECE700BF68CC00208A
:10613000C8CC00202DE9F04F80468FB017460C46A2
:1061400016464FF0000A23780793B4F9029063785B
:106150002068A2880893237994F905B00A90ADF8D5
:106160002C200993B9F1000F3DD0002F40D03068AA
:10617000BDF828500C9080B2B288ADF8342085422A
:1061800031787378B6F9022096F804E02ED1914563
:106190002CD1BDF82C50BDF83400281A4542454199
:1061A000CDE901320091CDE903EB124A534629466D
:1061B0004046FDF7FDFF099B0E4ACDF810B0CDE932
:1061C0000293089B0193079B009329465346404640
:1061D0000AF1010AFDF7D2FFBAF1240F04F1060417
:1061E00006F10606AFD10FB0BDE8F08F0025D7E766
:1061F0003D46E0E7240C07082DE9F04F9BB091469F
:106200000E900F930C46154600260F9B5A1C01D08A
:10621000B34266D1A446BCE80F0010AF0FC7DCF84C
:1062200000303B6023790993237C0B9394F9113060
:106230000C93A37C94F80C8094F813A00A92074660
:106240000D93B9F1000F5AD0AE46BEE80F000DF124
:10625000540CACE80F00DEF80020149BCCF80020B2
:10626000534033F07F43864695F804B0A96895F80B
:106270000CC0E87C3FD1099A5A453CD177453AD1C8
:10628000E04538D10A9A8A4237D1AAEB0003594235
:1062900059410A9B1B4A0E98CDF81CA0CDE90583F5
:1062A000099B03930D9B02930C9B01930B9B009303
:1062B000049733468B46FDF77BFF0A9B114A0E98E5
:1062C000CDF81CA0CDE90583099B03930D9B029398
:1062D0000C9B01930B9B0093049733465946FDF7A3
:1062E0004DFF0136402E04F1140405F114058CD144
:1062F0001BB0BDE8F08F0021CBE71946C9E7CB46BC
:10630000DBE700BF3B0C07082DE9F04F074687B0DD
:1063100016460C4615464FF0000BD4E9009AD4F807
:10632000088066B3A8688045D5E9002125D191454C
:1063300023D1AAEB010359425941CDE9019A114AEF
:10634000CDF800805B4638460591FDF731FF059991
:106350000C4ACDF800805B46CDE9019A38460BF136
:10636000010BFDF70BFFBBF1080F04F10C0405F165
:106370000C05D2D107B0BDE8F08F0021DDE7314632
:10638000E6E700BF5C0C07082DE9F04FA1B0174607
:1063900010900C4615460026A646BEE80F000DF1EB
:1063A000480CACE80F0023680B939EE80700238A93
:1063B0000C93638A0D93A38A0E93E38A94F8048066
:1063C000D4F808B094F80CA094F818900F938CE8C7
:1063D0000700002F5CD0AE46BEE80F000DF1640C44
:1063E000ACE80F009EE807008CE8070095F818C09D
:1063F00029682879AB682A7BCC4547D1804545D1AF
:106400000B98884242D1924540D19B453ED1169A85
:106410001D9B9A423AD117991E9BCB1A594259415A
:106420000F9B08930E9B07930D9B06930C9B194A99
:106430001098CDF80CA0CDE904B30B9BCDF80090DB
:10644000CDE9018333461191FDF7B2FE11990F9BFF
:1064500008930E9B07930D9B06930C9B0D4A109877
:10646000CDF80CA0CDE904B30B9BCDF80090CDE99D
:10647000018333460136FDF781FE042E04F11C042E
:1064800005F11C0588D121B0BDE8F08F0021C7E7D8
:106490003946DCE76D0C07082DE9F04FDFF864A002
:1064A000DFF864B085B00646894615461F460024CD
:1064B000002F01DBA7421CD119F80480FDB12B5D30
:1064C000A8EB03020AEB83035142DB6900935141BD
:1064D00023465A4630460391FDF76AFE03990AEBBC
:1064E00088085A46D8F81C30009330462346FDF7FA
:1064F00045FE01340E2CDBD105B0BDE8F08F2946F6
:10650000EDE700BFA08106088F0C0708F0B589B041
:10651000044647F0ADFB10F0FF020BD1394B9978E0
:10652000394B4FF4D47000FB0131012009B0BDE8B4
:10653000F040FFE5354905222046F7F7B9FBA0B941
:10654000304B9A78304B4FF4D47101FB0233304A10
:1065500015689488062606FB00F299180130242855
:106560009D508C80F7D109B0F0BD20462949294EB5
:1065700001AA4CF0CAFF4FF0FF33079302AD00248D
:1065800078B1062C02D1FDF7F3FFECE7F7F7DEFF59
:1065900001AA45F8040B3146002001344CF0B5FF48
:1065A000EEE7042CEFDD029B232BECD8039E112E8B
:1065B000E9D8049D3B2DE6D8059C04F57A72B2F526
:1065C000FA6FE0D80698FF28DDD807994A1C402AC0
:1065D000D9D80C4A92784FF4D4777A43062707FB30
:1065E00003220D4B134483F8D4000C4883F8D06089
:1065F00083F8D150A3F8D24083F8D510FFF786FF77
:10660000B1E700BF608500208884002011080708DA
:10661000D0810608AE570708B88300201D2507085B
:1066200070B5054608460E4647F022FB3146044643
:1066300002462846F7F73CFB60B92B5DA3F1300218
:10664000092A06D923F02003413B192B01D9013433
:10665000281970BD0020FCE72DE9F0418AB00446FE
:106660000D4647F005FB10F0FF000FD13E4B1A78A6
:106670003AB94FF0FF333D4901200AB0BDE8F0417F
:10668000BAE56B1C6DD02B460246F4E7384905226B
:106690002046F7F70DFB38B934484FF47E710AB045
:1066A000BDE8F04145F062BF20463249314E6A46AE
:1066B0004CF02BFF01AD002478B1092C02D1FDF77D
:1066C00057FF4EE0F7F742FF6A4645F8040B3146A4
:1066D000002001344CF019FFEEE7092CEFD10199AD
:1066E0003F29ECD8DDF808E0BEF1010FE7D8DDF86E
:1066F0000CC00CF10103402BE1D8049F362FDED8EB
:10670000059E072EDBD8069D1B4A05F5742303F56D
:1067100010739342D3D8079C072CD0D8089800F563
:10672000742303F510739342C9D8099AFF2AC6D877
:10673000124B4FF0140808FB013309B2C3F8A00054
:106740000F4883F8A8E083F8A9C083F8AA7083F8FB
:106750009C60C3F8985083F8A44083F8AB20FFF7FF
:106760007BFF0AB0BDE8F0812C82002000CD002024
:1067700011080708AE57070880841E0068CC002067
:106780001D2507084FF0FF3166E770B586B0044657
:1067900047F06EFA10F0FF0205D12249012006B041
:1067A000BDE87040B0E5204905222046F7F780FAA1
:1067B00038B91C4840F2FF3106B0BDE8704045F0E2
:1067C000D5BE20461949194E01AA4CF09EFE02ADD5
:1067D000002478B1042C02D1FDF7CAFE1FE0F7F7C0
:1067E000B5FE01AA45F8040B3146002001344CF0F7
:1067F0008CFEEEE7042CEFD1029A072AECD80C4B62
:106800000C480C2101FB0233039AC3F8A025049A1B
:10681000C3F89825059AC3F89C25FFF7B6FF06B084
:1068200070BD00BF00D2002011080708AE5707084E
:1068300068CC00201D2507082DE9F0438DB00446E3
:1068400047F016FA10F0FF0205D13E4901200DB0C5
:10685000BDE8F04398E53C4905222046F7F728FAC1
:1068600038B938484FF47E710DB0BDE8F04345F0BB
:106870007DBE20463549354E01AA4CF046FE02AD9C
:10688000002478B10A2C02D1FDF772FE57E0F7F729
:106890005DFE01AA45F8040B3146002001344CF09E
:1068A00034FEEEE70A2CEFD1DDF80880B8F1030FD3
:1068B000EAD8DDF80CE0BEF1010FE5D8DDF810C034
:1068C000BCF1070FE0D8059F214A07F5742303F5B3
:1068D00010739342D8D8069E072ED5D8079D05F58C
:1068E000742303F510739342CED8089CB4F5004F7F
:1068F000CAD20998B0F5004FC6D20A99B1F5004F37
:10690000C2D20B9AB2F5004FBED2124B4FF01C0907
:1069100009FB0833A3F80A060F4883F810E683F84A
:10692000FCC5C3F8F87583F80466C3F80056A3F8ED
:106930000846A3F80C16A3F80E26FFF77DFF0DB04E
:10694000BDE8F08360D2002011080708AE570708A1
:1069500080841E0068CC00201D2507082DE9F04F1B
:10696000A1B0CDE90C011546002414AE0D9A02EB3E
:10697000441263010DF1400C02F1200E10685168C1
:10698000674603C708327245BC46F7D1002D00F0B8
:1069900081802B4418AF03F1200C186859683A46DF
:1069A00003C2083363451746F7D19DF840300B9377
:1069B0009DF860100B98BDF842709DF84480BDF8BA
:1069C00046909DF848A0BDF84AB09DF84C30BDF8FF
:1069D0004E2081425CD1BDF86210B94258D19DF879
:1069E0006410414554D1BDF86610494550D19DF819
:1069F000681051454CD1BDF86A10594548D19DF8F1
:106A00006C10994244D1BDF86E10914240D11CA93E
:106A100014A8CDE90E3247F0D1F8DDE90E32B0FA14
:106A200080F14909CDE905B30B9B0093CDE9072619
:106A3000CDE9039ACDE90178174A0C980B912346CA
:106A4000FDF7B6FB0B99BDF84E3007939DF84C301F
:106A50000693BDF84A3005939DF848300493BDF87D
:106A6000463003939DF844300293BDF842300193C1
:106A70009DF840300093084A0C980896234601344C
:106A8000FDF77CFB082C7FF471AF21B0BDE8F08FDF
:106A90000021C7E72946D6E7A70C07082DE9F041F2
:106AA00090B0044647F0E4F810F0FF0205D14549E4
:106AB000012010B0BDE8F04150E74349434F01AA1F
:106AC00020464CF022FD41496A464CF01EFD06AEC0
:106AD0000024354600286ED0092C61D13A4901AA1C
:106AE00000204CF012FD0646002869D047F0C0F89F
:106AF000044638B10F2828BF0F242246314602A889
:106B00004CF02EFD04F14003DDF818800DEB03047A
:106B1000B8F1070F4FF0000304F8383C4DD8DDF80A
:106B20001CE0BEF11C0F48D8DDF820C0BCF1FF0FFF
:106B300043D8099F1C2F40D80A9EFF2E3DD80B9C9E
:106B40001C2C3AD80C98FF2837D80D99022934D834
:106B50000E9AFF2A31D81E4B03EB481303F5CF637F
:106B600003F8084C03F810EC23F80ECC03F80C7C67
:106B700023F80A6C23F8060C03F8041C23F8022CF3
:106B800002AC224603CAAA4218605960144603F1B7
:106B90000803F6D10F48FFF781FF10B0BDE8F08180
:106BA000F7F7D4FC6A4646F8040B39460020013456
:106BB0004CF0ABFC8EE7092C90D0FDF7D9FCECE74C
:106BC00004469FE7D0D2002037260708AE570708B3
:106BD00068CC00201D25070838B5064D002455F85F
:106BE00034000134FDF746FAFDF776FA352CF6D17C
:106BF00038BD00BFD881060830B5274885B0FDF7FD
:106C000039FAF4F7E5FD28B9244805B0BDE830406D
:106C1000FDF788BAF5F7A8F808B92148F5E7F5F7C0
:106C2000ADF80268037D81790446407C0290207CA7
:106C30000190608A009052081A48FDF7CFFAE51DCE
:106C40000C3415F8010BFDF7ABFAA542F9D1164C3F
:106C50001648FDF70FFA6378022B06D007D9032BED
:106C600010D11348FDF706FA0CE01248FAE704F5D4
:106C700080541148FDF7FEF994F8B431022B06D088
:106C8000032B06D005B0BDE83040FDF725BA0B4810
:106C9000E8E70B48E6E700BFDB0C0708E50C070850
:106CA000F30C0708020D0708A84E0020300D070856
:106CB000400D0708460D0708530D0708590D070832
:106CC000720D07082DE9F3473549DFF8D49001AA82
:106CD0004CF01BFC4FF0000A4FF0FF35564654466F
:106CE0005746A84678B9BAF1040F3DD0BAF1050F5E
:106CF00044D0BAF1030F13D02A492B464246012053
:106D000041F04AFE0EE0BAF1040F09D8DFE80AF0BC
:106D1000030D12171C00F7F719FC804603281BD936
:106D2000FDF726FC02B0BDE8F087F7F70FFC05463B
:106D3000A628F4E7F7F70AFC07463F28EFE7F7F73E
:106D400005FC04463F28EAE70378482B03D0562B7E
:106D5000E6D1012600E0002601AA494600200AF1FA
:106D6000010A4CF0D2FBBDE70F4BA72202FB0852F1
:106D700003EB4203B3F86867C6F34036A72303FB6F
:106D80000855A401084B04F47C6407F03F0703EBAB
:106D900045033C4344EA4634A3F86847C2E700BFD2
:106DA000AE570708D0D3002068CC00202DE9F3416E
:106DB0002649DFF8988001AA4CF0A7FB002504467D
:106DC0002F464FF0FF366CB9022F0BBF20492049E8
:106DD0008D55334612BF2246334622460120FFF727
:106DE0005BFB04E037B1012F12D0FDF7C1FB02B00D
:106DF000BDE8F0812046F7F7A9FB0D280646F4D838
:106E000001AA414600204CF080FB01370446DAE736
:106E100010482146F6F766FF05460028F0D00E48D8
:106E20002146F6F75FFF60B10C482146F6F75AFF9E
:106E300048B10B482146F6F755FF0028D5D1032568
:106E4000DEE73D46DCE70225DAE700BFAE5707087C
:106E500074800020840D07088E2407080E4E070852
:106E6000FB5307082DE9F04F2DED028B4D484E4D99
:106E70009FED4E8A8BB0FDF7CBF90027B946BA4695
:106E80004B4B4C4A196800238B4227DB01371D2FDF
:106E900005F14805F4D14849484BD1E90021520990
:106EA00042EAC1624649186809684FF47A73B0FB38
:106EB000F3F34448FDF7ACF90A2299FBF2F302FB25
:106EC000139000909AFBF2F13F4802FB11A2FDF7EC
:106ED0009FF90BB0BDEC028BBDE8F08F52F8040BAC
:106EE000A84201D00133CFE7AC6A4CB107EE904A1B
:106EF000B8EEE77AC8EE077AFDEEE77A17EE904A29
:106F0000AB6B0893D5E90C637609E96B46EAC36677
:106F10005B090993089B4FEAE47B6143A4FB030CE4
:106F200003FB0B1141F28833C01841EB0C014FF405
:106F30007A72002347F006FD099A804604FB02F1AD
:106F4000A4FB060C41F28833C01806FB0B1141EB81
:106F50000C014FF47A72002347F0F4FC2B6C01967D
:106F6000042F4FF47A72B3FBF2F306934FF00A0347
:106F700018BF814490FBF3F203FB1200CDE904201B
:106F800098FBF3F203FB1283CDE90223089B0093E5
:106F90002A680E482346394618BFC244FDF738F91F
:106FA00074E700BF890D0708C80800200024744951
:106FB000386A012090690120086A0120106A0120C6
:106FC000186A0120050E0708270E0708D00D0708CC
:106FD0001FB50A4B03930A4B02930A4B01930A4BCA
:106FE00000930A4A0A4B0B490B48FDF711F90B496C
:106FF0000B4805B05DF804EBFDF70AB91D2507083D
:10700000760E07087F0E0708880E0708F8010708A4
:10701000550E07080B0207085B0E0708940E0708B9
:10702000A40E0708F8B50C480C4E0D4F0D4DFDF79A
:10703000EFF80D4B1A68C2F500729200002422B1DD
:1070400056F824103846FDF7E3F80134222C02D01C
:1070500055F82420F3E7F8BDAD0E07088083060835
:10706000C30E0708583C00205434002070B5124B62
:1070700093F8A02CD2B1192A94BF104B1049114893
:10708000114D124E98BF03EB82034FF0000498BFDE
:10709000D3F86812FDF7BCF8214655F8042B3046AA
:1070A0000134FDF7B5F8082CF6D170BDBDE870408D
:1070B0000748FDF737B800BF68CC0020A08106085C
:1070C000D10E0708D90E07080CD90020F10E0708C9
:1070D000000F07082DE9F84F054646F0C9FDDFF817
:1070E000EC800446D8F80090C0B93048304D314F9C
:1070F000FCF7C0FF012655F8041B59B10B783BB1D2
:1071000006FA04F313EA090F02D03846FDF766F8D1
:107110000134F0E7BDE8F84FFCF7DEBF0246264930
:107120002846F6F7C5FD78B92448214C214DFCF7D7
:10713000A1FF54F8041B0029ECD00B78002BF8D0E9
:107140002846FDF74BF8F4E72B78DFF864B02D2BD9
:1071500003BF013504F1FF344FF0010A4FF0000A7C
:1071600000265BF8047B1FB9BDE8F84F41F01ABB5D
:10717000224639462846F6F79BFDA8B90120B040C3
:10718000BAF1000F0AD0F7F737FB0D48FCF772FF92
:1071900039460C48BDE8F84FFDF73AB840EA090017
:1071A000C8F800000848F1E70136DAE7170F0708CA
:1071B00070840608905D0708210F0708260F07084E
:1071C000320F0708550F07083B0F0708843E0020C1
:1071D0002DE9F84F054646F04BFDDFF8F4800446F4
:1071E000D8F8CC6CC8B93148314DDFF8D480FCF701
:1071F00041FF0127E3B205EB8302D2F8541341B1FA
:1072000007FA03F3334202D04046FCF7E7FF0134AC
:10721000F0E7BDE8F84FFCF75FBF02462549284676
:10722000F6F746FD60B92448244C254DFCF722FFB3
:1072300054F8041B0029ECD02846FCF7CFFFF7E7F1
:107240002B78DFF878B02D2B03BF013504F1FF3424
:107250004FF0010A4FF0000A4FF000095BF8047B81
:107260001FB9BDE8F84F41F09DBA2246394628467D
:10727000F6F71EFDB8B9012303FA09F3BAF1000FBE
:107280000CD026EA03030F48C8F8CC3CFCF7F2FE0A
:1072900039460D48BDE8F84FFCF7BABF33430B48F9
:1072A000C8F8CC3CF2E709F10109D7E7170F070846
:1072B000A0810608210F0708260F0708F484060896
:1072C000905D0708320F0708550F07083B0F0708A6
:1072D00068CC00202DE9F047814646F0C9FC494EB4
:1072E0000446376800BB4848484D494EFCF776FFD6
:1072F0004FF00C0808FB04F35A5D0123013A934058
:107300003B4206D020461BF0CFFB01463046FCF73F
:1073100065FF0134182CEDD117B93E48FCF7AAFEE1
:10732000BDE8F047FCF7D8BE02463B494846F6F7B1
:10733000BFFC054678B93948FCF79CFE2C46344D15
:1073400020461BF0B1FB013401462846FCF746FFFE
:107350001A2CF5D1E4E799F800302D2B03BF09F181
:10736000010904F1FF344FF0010A4FF0000A002533
:1073700028461BF099FB2246804601464846F6F710
:1073800097FC002836D1BAF1000F1CD0182D17D069
:10739000192D0AD1736822483360FCF76BFE414611
:1073A0002048BDE8F047FCF733BF1F4B0C2202FB1F
:1073B000053393F890230123013A93403B43EAE7D6
:1073C0006FF07F43E7E7182D03D1C6F800A01748F8
:1073D000E3E7192D01D17760F9E7134B0C2202FB8B
:1073E000053393F890230123013A934027EA0303DE
:1073F0003360ECE701351A2DBAD1BDE8F04741F012
:10740000D1B900BFAC800020430F070830850608C3
:10741000540F07084D0F0708210F0708590F0708D9
:10742000320F0708550F0708A08106083B0F070811
:107430002DE9F341044646F01BFC04283DD1661EAD
:107440002546E71C16F8010FF6F71AFCBE4230700D
:10745000F8D1DFF87880271D15F8016B40463146DA
:107460004EF067F820B1314628464EF062F820B160
:1074700002B0BDE8F041FDF77BB8BD42ECD120463B
:1074800022F0EAFE0F48FCF7F5FD0F490F480023F4
:1074900011F8012F10F8014B08326A440133042B14
:1074A00002F8084CF4D1002309488DF804306946ED
:1074B000FCF7AEFE02B0BDE8F0810028E2D0FDF797
:1074C00057F8DFE7640F070838D9002068860608F8
:1074D000560F070808B504460648FCF7CBFD064BD7
:1074E0001868F8F7EDF9054B18681DF0F3F9204618
:1074F00007F0E0F86A0F0708288200203482002095
:10750000034808B5FCF7B6FD0120FFF7E3FF00BF15
:10751000760F070808B50C4B93F8D02C012A12D12E
:1075200093F8D53C062B0AD00A2B04D00748BDE8B7
:107530000840FCF79FBD23F0CDF80548F7E721F0A0
:107540005FFF0448F3E708BD68CC00208F0F0708F1
:107550009E0F0708B80F070808B50A48FCF7E2FDB8
:10756000094B1868F8F7ACF9084B002483F8F24C83
:10757000C3F8344D064B1C7013F00CFF2046FFF788
:10758000A9FF00BFD10F07082882002068CC002087
:10759000F974002008B5214B214C1D68D4F8400D2A
:1075A0001DF098F928461DF095F9D4F8400D417961
:1075B0008B0704D4036841F002019B6998470021BE
:1075C0000846F9F7E9F800210120F9F7E5F8D4F8C1
:1075D000400DF9F7E4FF78B101210020F9F7DCF85C
:1075E000D4F8400DF9F7FCFF01462846F9F7D4FF1F
:1075F00000210846F9F7D0F82846F9F7D0FF00280F
:10760000E5D001210846F9F7C7F82846F9F7E8FF61
:107610000146D4F8400DF9F7BFFFD4E734820020CB
:1076200068CC0020F7B50546FCF7AEFF044620B154
:1076300003B0BDE8F040FCF79BBF28461E491E4F33
:1076400001AA4BF062FF2646254640B90B2D18D9FA
:1076500001461A480B22FCF78FFF03B0F0BD44B17E
:10766000012C0AD001AA3946002001344BF04DFF0D
:10767000EBE7F6F76BFF0546F4E7F6F767FF06461C
:10768000F0E7022C0ED1A6F57A73B3F57A7F05D90F
:107690000B484FF4FA624FF47A71DCE7094B03EBC5
:1076A00045039E80074B084803EB45032946B3F981
:1076B0000420FCF7ADFDD0E7AE57070886090708A0
:1076C000D3270708386A0120FB0F070870B5044666
:1076D000FCF75AFFC0B11F4B1E68013630461BF045
:1076E000E3F934460546E8B901341A2CA8BF002452
:1076F00020461BF0D9F90546A0B9B442F4D1BDE843
:1077000070401548FCF70EBD2046F6F71FFF0446F3
:107710001BF0CAF9054628B921461048BDE870405B
:10772000FCF776BD0B4B1C601DF08EFB2A460C4807
:107730002146FCF76DFD192C9DBF0A4B0C2202FB64
:1077400004330020BDE8704098BF93F890031DF00B
:1077500093BB00BF04120020081007081C10070884
:1077600032100708A081060870B51D4990B00522A7
:1077700004464DF0EBFE70B91A4A13782BB901217B
:107780001170194A1370194A1370194810B0BDE8E6
:107790007040FCF7C7BC1749032220464DF0D6FEC7
:1077A000C0B9104E104D3378104C7BB12B786BB1B3
:1077B0002278114901A8F6F7F9F801A8FCF735FD80
:1077C000002333702B70237010B070BD0B48FCF792
:1077D000A9FCF5E70A4810B0BDE87040FCF725BDEC
:1077E000011907082C8200202D8200202E82002003
:1077F00047100708751B07085D100708A010070849
:10780000B410070870B5124E337890B0A3B1114D83
:107810002B788BB1104C1149227801A8F6F7C6F8E5
:1078200001A8FCF702FD0E48FCF7FFFC00233370B3
:107830002B70237010B070BD0A48FCF71BFC22F0BF
:10784000EFFCF6F7E5FE22F0F5FC0020FFF742FE24
:107850002C8200202D8200202E8200205D1007083F
:10786000C3100708E11007082DE9F0478CB0074660
:1078700010F8013B202BFAD00025204CDFF8848043
:10788000DFF88490DFF884A02E466946204612F087
:10789000C3F8394668464DF09CFEE0B16946404663
:1078A000FCF79CFC4946684646F088F900BB204638
:1078B00012F0D8F9124B01460078202814BF504628
:1078C0001846FCF78BFCFCF707FC2046FCF7FDFD97
:1078D000FCF702FC0136013540F285239D4204F19C
:1078E0000C04D2D10EB940F05DFF0CB0BDE8F087BA
:1078F00000212046FCF7DEFDE5E700BF60630608D7
:10790000D60C0708A3060708EB5E0708560F070802
:107910002DE9F04F2DED028B8FB00578202D064616
:1079200000F10100F9D0304646F0A2F9044618B142
:10793000012822D12A2D20D199489A4DDFF884823E
:10794000FCF7F0FB002640F28527284602A912F03A
:1079500063F802A94046FCF741FC0136284621465F
:10796000FCF7A8FDFCF7B8FBBE4205F10C05ECD115
:107970000FB0BDEC028BBDE8F08F3D2130464DF0DD
:10798000D8FD002800F005810346994613F8012D23
:10799000202AFAD0A9EB060901308046074610F8E4
:1079A000013B202BF9D07F4D4FF0000A5FFA89F997
:1079B00040F2852B02A9284612F02EF802A846F0C4
:1079C00057F902A9024601903046F6F771F9754B56
:1079D000044658BB019A4A4528D10C2202FB0A33BF
:1079E000DB7903F00706062E2FD14046F6F74EF955
:1079F0006D4902A846F0E2F820B16C4902A846F0B1
:107A0000DDF8E0B998F80030222B18D1404646F056
:107A10002FF908EB000313F8013C222B0FD1821E33
:107A200008F10101284612F0DDF9A1E70AF1010A87
:107A3000DA4505F10C05BDD140F0B4FE98E74046AB
:107A400046F016F941460246ECE713F0C0030AD0AF
:107A5000402B6AD05648FCF76BFB2846FCF735FDF7
:107A6000FCF73AFB84E798F80030002BF2D051493C
:107A700040464DF09EFD0446404646F0F9F88442EB
:107A8000E8D14046F6F7D6FC2846B0EE408A12F020
:107A9000F5F807EE900AF8EEE77AF4EEC87AF1EE20
:107AA00010FAD7D8284612F0F9F807EE900AF8EE47
:107AB000677AF4EEC87AF1EE10FACBDB052E1AD114
:107AC00018EE104A3C4902A846F078F848B93B4BFA
:107AD00093F8771DE2B2914203D0002C45D183F890
:107AE000DB4D284612F0BEF8052E43D8DFE806F03D
:107AF00041414B4B4D4F042E12D13A4617F8013BF2
:107B0000202BFAD0092BF8D0013A00240A2112F8D0
:107B1000013F303BDBB2092BD4D801FB0434F6E73C
:107B20004046F6F713FD0446CCE7284612F03EF92E
:107B300090F804B0814627462346A246BB4500D9AB
:107B40001BB1BAF1000F85D0BCE7D9F8003041462F
:107B500053F82700F6F7C6F8002805BF3C46012376
:107B600000234FF0010A0137E8E7012283F8DB2DFB
:107B7000B7E7047002A91248FCF730FB0021284641
:107B8000FCF798FCF4E60480F4E70460F2E7046094
:107B9000F0E730460FB0BDEC028BBDE8F04F63E676
:107BA000E810070860630608EB5E0708FA1007088C
:107BB00034110708051107081311070868CC0020C5
:107BC00029110708A30607082DE9F8432BF0C8FB85
:107BD00020B9BDE8F8434948FCF74CBA4848494C3D
:107BE000494E4A4FDFF87081FCF79CFA0025637814
:107BF000FF2BA94605F1010576D02278FF2A73D024
:107C000029463046FCF704FB2378A178062B5AD886
:107C1000DFE803F004343A42594A5200072954D8A5
:107C20003B4B03EB8103D3F8D0243846FCF7F0FA42
:107C3000A1794046FCF7ECFAE1793648072997BF6D
:107C4000334B354A03EB8103D3F85425FCF7E0FAB4
:107C5000324B334803EB091303F62C69B3F82E1E9D
:107C6000FCF7D6FAB9F8021001F00301012936D069
:107C7000022940D02B48FCF7CBFA33E02A4A2B4BA1
:107C8000002908BF1A46D0E7062920D8204B03EB6D
:107C90008103D3F8F024C8E707291AD81C4B03EB5B
:107CA0008103D3F80C25C0E7092914D8184B03EB3E
:107CB0008103D3F82C25B8E779B11D4A1D4B022961
:107CC00018BF1A46B1E71C4AAFE71C4AADE71C4A89
:107CD000ABE71C4AA9E71C4AA7E71C4AA5E71C48D2
:107CE000FCF720FAFCF7F8F9402D04F110047FF4BA
:107CF0007EAFBDE8F8831748F2E700BFD31107084D
:107D0000021207088CDA0020121207082612070850
:107D1000A08106084E1207087311070868CC0020DE
:107D20005F120708961207086E110708631107080B
:107D3000B5110708C31107084411070857110708B0
:107D40007B1107088B1107089A110708A71107086C
:107D50007412070884120708351207082DE9F04F3E
:107D60002DED028BA3B0BE4B0393BE4B0293BE4BD3
:107D70000193BE4BBE4ABF49BF480093BF4BC04CA6
:107D8000C04DC14FFCF744FAC049C148FCF740FA66
:107D9000C04BC14819684FF47A73B1FBF3F1FCF79B
:107DA00037FA06A8F6F796F806A916A844F0EAFBF3
:107DB00016A9BA48FCF72CFA22F0B2FF6423B0FBF4
:107DC000F3F103FB110094F82D3105EB830382B22C
:107DD000D3F87435009394F82C31B14889B2FCF78C
:107DE00017FAB04BB0481968B04BB1FBF3F1FCF790
:107DF000F5F9D7F81C80002605F2845904F5977A26
:107E000005F5B46B0123B34013EA080F0BD059F802
:107E1000263043B11AF806205BF8261053F82220CA
:107E2000A348FCF7DBF90136072EEBD1FCF754F938
:107E3000A0489E4EFCF776F909A8F2F702FC0999D2
:107E40009D48B1FBF6F1FCF7E3F90A999B48B1FBB9
:107E5000F6F1FCF7DDF90B999948B1FBF6F1FCF767
:107E6000D7F90C999748B1FBF6F1FCF7D1F923F05B
:107E700063F905EB8000D0F8C815059123F066F989
:107E800005EB8000D0F8C88523F070F905EB800081
:107E9000D0F8C89523F08EF905EB8000D0F8C8A57E
:107EA00023F0ACF905EB8000D0F8C8B523F0F4F965
:107EB00005EB8000D0F8C86523F0D4F905EB80000D
:107EC000CDE900ABD0F8C83505997F48CDE902630C
:107ED00042464B46FCF79CF97C4B1B68DE031CD5E5
:107EE0007B4B93F80080B8F1000F16D07948DFF88B
:107EF0004492DFF844A24146FCF78AF90026B9F91A
:107F00000220314650460136FCF768F9F3B2984535
:107F100009F11009F3D8FCF7DFF80020FEF76CFE3A
:107F20006D4B6E4A1E886E4B6E491B686E48DFF8BB
:107F30000C92DFF80C82DFF80CA2DFF80CB2C3F56C
:107F400000739B00FCF764F9684A694B6948D31ACF
:107F5000694AB6B231461288FCF75AF96748FCF70D
:107F6000E1F8042659F8041B6548FCF737F9654821
:107F7000FCF780F818F8011B002940F0F0816248F6
:107F8000FCF778F86148FCF775F85AF8041B0029EB
:107F900040F0E9815C48FCF7C5F8013EE2D1398C3C
:107FA0005B48FCF71BF95B490A6F5AB107EE902A50
:107FB000DFED596AF8EEE77A86EEA77AFDEEC77A2A
:107FC00017EE902AD1F800315BB107EE903ADFED61
:107FD000526AF8EEE77A86EEA77AFDEEC77A17EED8
:107FE000903A896A59B107EE901ADFED4B6AF8EEC4
:107FF000E77A86EEA77AFDEEC77A17EE901A00911F
:10800000B4F83C114548464F464EDFF84091FCF726
:10801000FFF84548FCF72EF83B684FF001081E407A
:10802000002E40F0A481FCF757F83B68580140F15E
:108030008F800DA811F04AFE002840F089800D9B2A
:10804000B3F5217F9DBF39480C2202FB0300304667
:1080500016A911F0E1FC364816A9FCF7E6F877E01E
:108060001D250708760E07087F0E0708880E0708EB
:10807000F80107080B0207085D0E0708550E0708F0
:1080800060DD0020A0810608386A0120940E0708F0
:10809000A60E0708042D0020D8120708F2120708C0
:1080A00003130708200100202813070840420F008F
:1080B0003813070840130708551307086713070804
:1080C000791307088B1307089D130708306A0120EE
:1080D0002C6A0120F0130708302E00200000022037
:1080E0005434002000180000241407080080000801
:1080F000004000085C140708823E00209614070820
:10810000A9140708B11407084F0F0708C714070878
:10811000D1140708C808002000247449E114070896
:1081200088690120C0FFFD7F1E15070860630608EF
:1081300035150708AC3D0020151407087887060898
:1081400095DE0020D0600020C0140708550F0708F6
:108150003B68190510D500203BF03CFF420706465E
:1081600003D5A049A048FCF753F8F30740F112816A
:108170009E499D48FCF74CF89D48FBF77BFFD4F8DF
:108180004011002900F014810B7B4A7B99488968D3
:10819000FCF724F8FBF7A0FF9748FBF76BFFD4F838
:1081A0004401FBF70AFF002800F006810DA9D4F86E
:1081B0004401FBF743FF9DF848109DF85430149A92
:1081C0008E48FCF70BF8119911B18D48FCF706F8B1
:1081D0000F9911B18B48FCF701F8FBF77DFF8A4B33
:1081E0001B68180640F1AC802BF0BAF8002800F0AC
:1081F000A7808648FBF73EFF8548D0F8443DB3F59D
:10820000487F00F0E78000F2DB80B3F5167F00F0D6
:10821000E380B3F52F7F00F0E1807E497E4AB3F51D
:10822000FA7F08BF114690F8482D90F8493D90F824
:108230004B0D072896BF05EB80000020D0F84806BC
:1082400000907648FBF7CAFF00210F202BF094F82E
:1082500010B17348FBF7C2FF724E9FED738AFBF7B4
:108260003BFFF1797148FBF7D3FF738C07EE903A2F
:10827000F8EEE77AC7EE887A17EE900A45F064FECA
:1082800002460B466A48FBF7C3FFF38B07EE903AB2
:10829000F8EEE77AC7EE887A17EE900A45F054FEBA
:1082A00002460B466348FBF7B3FF338C07EE903A68
:1082B000F8EEE77AC7EE887A17EE900A45F044FEAA
:1082C0000B4602465C48FBF7A3FF5C48FBF7A0FFA8
:1082D0005B48FBF727FF5B48FBF724FF94F8483126
:1082E00019070AD594F8502194F851115648C2F351
:1082F000C002C1F3C001FBF78BFF94F848315A0765
:108300000AD594F8502194F851115048C2F38002D4
:10831000C1F38001FBF77CFF94F848319B070AD535
:1083200094F8502194F851114948C2F34002C1F326
:108330004001FBF76DFF94F84C114648FBF768FFCE
:10834000454B1B7833B105EB83054448D5F86816D7
:10835000FBF75EFF23B0BDEC028BBDE8F08F584603
:10836000FBF73CFF0EE65846FBF752FF15E696FA80
:10837000A6F3B3FA83F308FA03F2062B26EA020601
:108380007FF74EAE05EB83034846D3F8CC15FBF7D9
:1083900025FF45E6B7077FF5EFAE31491248FBF7F9
:1083A00037FFB6073FF4E8AE2E48FBF731FFE3E6B0
:1083B0002D48FBF75FFEEDE62C48FBF75BFE0CE774
:1083C000B3F5617F0CD01349294AB3F57A7F08BF12
:1083D000114628E7274926E7274924E7274922E7C6
:1083E000274920E749150708540F070865150708AE
:1083F000A5150708AB150708C4150708CA1507080F
:10840000E8150708F1150708843E00200D16070837
:1084100068CC002073110708AD120708131607086F
:108420003A160708247100200000C8425A160708AF
:1084300065160708701607087D1607088A160708CC
:108440009F160708C0160708CC160708DE1607088F
:10845000EF16070801170708828000201817070881
:108460007915070892150708B815070800160708B8
:10847000D0120708C2120708B4120708BB12070877
:10848000C91207082DE9F3411A481B4C1B4E1C4F1B
:10849000DFF87080FBF7BCFE0025E2792168A37944
:1084A00094F808C006EB820201F13F41D2F8800641
:1084B000A28806EB830301F57E01890AB2FA82F2F3
:1084C000D3F8E0314131C2F11F02BCF1000F0CD0F2
:1084D000CDE900C04046FBF79BFE0135312D04F18C
:1084E0000C04DAD102B0BDE8F08100903846FBF709
:1084F0008FFEF2E73217070814750020A0810608E6
:108500005E1707084E17070810B5F3F723FC124C47
:10851000D0B11248FBF726FE1148FBF7ABFD2068EF
:10852000F7F7CEF94FF47A70FBF788F80D4B18681F
:108530001CF0D0F90C4B1878F8F734FD022101201B
:10854000F2F75CFDF9F7A4F80848FBF793FD206803
:10855000BDE81040F7F7B4B9288200206C1707086F
:108560006A0F0708348200202C6A01208C17070844
:108570002DE9F0410446254E254DDFF8B08000205E
:10858000FDF738FD2348FBF7EDFDB17822480131B6
:10859000FBF73EFE21462020FBF7E2FE1F48FBF7DB
:1085A000E1FDB3781E4A4FF4D47707FB0353D3EDB4
:1085B000047AF5EE407AF1EE10FA0CBF01210021A9
:1085C0002046FBF7DBFDB1787943103108EB01025F
:1085D00020462944FCF706FD1248FBF7C3FDB3789B
:1085E000114A07FB03532046B3F9D210B1FA81F1C7
:1085F0004909FBF7C3FDB1787943D03108EB01029B
:1086000020462944BDE8F041FDF794BD6085002077
:1086100088910020BB170708C9170708DC1707084F
:10862000EF170708FE17070811180708B88300207E
:10863000A0F2DC50164BB0F5FA7FA8BF4FF4FA70E9
:10864000984210B5B8BF18460C46114640F00DFAD6
:1086500000B207EE900A9FED0F7AF8EEE77AE4B2E7
:1086600087EE870AFBEE096AE0EE006A07EE904AA1
:108670009FED097AF8EE677AA7EEA67AF3EE097A0B
:1086800020EE070A80EE270A46F0ECFF00B210BD8C
:108690000CFEFFFF0000C84200401C452DE9F84FCA
:1086A000864D95F859012DED028BB0EE408A78B3D6
:1086B000834E844F00244FF0060805F5AA7995F8FB
:1086C000843108FB0373234493F8FE3653B1012B26
:1086D0000DD00134042C06F10206F0D1BDEC028B62
:1086E000BDE8F88F09EB44039B8E3380F1E7032C40
:1086F00001D00023F9E7744B1B68DB0405D412F0AA
:108700001DFE00B2714B5885E3E740F2DC50F9E7FB
:108710006E4C21F0C1FDD4F82CA0D5F8907195F8DD
:1087200094811AF4807B14BF7E7B3E7A42463146A8
:10873000FFF77EFFA0848146012021F0ADFD424677
:108740003146FFF775FF8046E084022021F0A4FD4A
:10875000BBF1000F77D0B97B95F89521FFF768FF43
:10876000464236B22685BBF1000F6ED0FB7B6422F9
:1087700013FB09F393FBF2F3A3843B7C13FB08F395
:1087800093FBF2F3E3847B7C13FB06F393FBF2F39E
:10879000238512F09BFD95F85831608543B9B4F9F3
:1087A0002830626AC5F88821A5F88C31A5F88E01B9
:1087B0001AF0400F92D0B4F9343007EE903AF8EE48
:1087C000E77AB2EE047A87EE878AB5F99E3107EE32
:1087D000903AF8EEE77A38EE678ADFED3D7ABDEE43
:1087E000C88A18EE103A1BB208EE103AB8EEC88AE2
:1087F00028EE278AB0EE480AF4F73CFCF0EE408AF7
:10880000B0EE480AF4F7D4FBB4F9263006EE903AFD
:10881000B4F9243007EE103AF8EEE66AB8EEC77AFB
:1088200067EE007A20EE660AE6EEA87AA7EE280A3E
:10883000FDEEE77ABDEEC00A10EE103AA38417EE03
:10884000903AE3844AE7797A86E7224F97F8A0BC0A
:10885000B0EE480ABBF1120F4FF00001484608BFC6
:10886000C7F8A49C12F0EAFBBBF1120F00B208BFDC
:10887000C7F8A80CA084B0EE480A4FF001014046AA
:1088800008BFC7F8AC8C12F0D9FBBBF1120F00B2D5
:1088900008BFC7F8B00CE084B0EE480A4FF0020100
:1088A000304608BFC7F8B46C12F0C8FBBBF1120F1A
:1088B00000B2208508BFC7F8B80C6AE760DD002069
:1088C0005C6A0120A0810608346A0120386A012010
:1088D00035FA8E3C68CC00202DE9F041DFF8F081BC
:1088E000754DD8F800309F6A744B1B6813F0100F59
:1088F00086B040F0A88095F83830002B00F0A380B7
:108900006F4CD4F8A83104F5D0709847002800F0D7
:108910009A8094F8FF31002B43D1022385F8583018
:10892000B4F9003207EE903AB4F90232F8EEE77A81
:10893000C4ED727A07EE903AB4F90432F8EEE77AB1
:10894000C4ED737A07EE903AF8EEE77AC4ED747AE4
:108950005C4903AAA1F10C0041F028FF03A994F897
:10896000E421084622F08EFB03A822F04DFB94ED93
:108970006E0A5549544C03A841F025FF04F17808CC
:108980000026B4EC010AD5F8383584ED020A4046D9
:1089900098470136032E04ED010A08F5C078F0D19E
:1089A00051E095F85830012BD2D1D4F8BC31039363
:1089B000D4F8C031049303A9D4F8C431059305F168
:1089C0005800F4F773FE95F85830012B4FF000066D
:1089D0006AD0022B5FD0039604960596DDED037AEC
:1089E0009DED047ADDED056AC4ED727A84ED737A4B
:1089F000C4ED746AFDEEE77ABDEEC77AFDEEE66A75
:108A000017EE903A17EE102A16EE901A1BB212B219
:108A100009B2A4F80032A4F80222A4F8041201203A
:108A2000CDE900210421294AF4F7D6FFD8F8003017
:108A300000200021C3E90C01C3E91001C3E90E01C4
:108A40002E646E64AE64EB695B0621D51C4C94F811
:108A50005032EBB1FE173146384645F0DDFED5ED1C
:108A6000106A94ED997A07EE900AA7EEA67AD4E9F7
:108A70009C32D5ED116A84ED997A94ED9A7ADB19DE
:108A8000A7EEA67A46EB0206C4E99C3684ED9A7AF4
:108A900006B0BDE8F0812B6F0393D5F888300493BE
:108AA000D5F8A030059399E7C4F8C861C4F8CC6143
:108AB000C4F8D061C4E700BF386A0120886901208A
:108AC00060DD002028DF0020786A01201E180708DA
:108AD000286A0120034B012283F88022022283F8B6
:108AE0008122704760DD002070B50D4E35782D1A5B
:108AF00018BF01250328044634BF0446002420463D
:108B0000F5F7C8FE074A347002F282231A2104FBEB
:108B10000133C2F8903119F0CDFD284670BD00BF79
:108B20006085002060DD0020022810B50C4618D8B2
:108B3000FFF7DAFF0B48FBF715FB0B4B0B481978D7
:108B40000131FBF765FB21460820FBF709FC2146B4
:108B50001020FBF705FC21462820BDE81040FBF75C
:108B6000FFBB10BD45180708608500205518070891
:108B700038B5154C154DAC4213D30020F5F78AFEDD
:108B8000134821F069FB134A136843F48003136010
:108B900000BF114B1878FFF7A7FFBDE838402BF056
:108BA0001BBFB4F90230002B4FF00001204607DA5A
:108BB000F5F760FE01212046F5F75CFE0221204614
:108BC000F5F758FE1434D6E7A8620708F8670708D7
:108BD0006A180708843E00206085002010B504460E
:108BE0000A48FBF747FAFFF7C3FF21F019FBF5F737
:108BF0000FFD21F01FFB064B0649002220461A708C
:108C0000FDF70EFD08B9FEF765FC10BD73180708E7
:108C10002D8200203919070810B5064B5C78241AFC
:108C200018BF0124032828BF0020587022F03AF80A
:108C3000204610BD60850020022810B50C4610D8D3
:108C4000FFF7EAFF0748FBF78DFA074B074859780B
:108C50000131FBF7DDFA21461820BDE81040FBF793
:108C60007FBB10BD89180708608500209918070888
:108C70002DE9F04F0D468DB0B6490746FDF7D0FC03
:108C80000646002840F0B780B3493846FDF7C8FCD7
:108C90000646002840F0B180B0493846FDF7C0FCD8
:108CA0000646002840F0AB80AD493846FDF7B8FCD9
:108CB0000646002840F0A580AA493846FDF7B0FCDA
:108CC000002806460ABF012410243E466D4205F0E6
:108CD00020052C43A44DA54F95F800A095F80290CF
:108CE00095F80180DFF8F8B25F45C0F08C80FFF79F
:108CF0003FFF5046FFF7F8FE4846FDF77BF9404638
:108D0000FFF78AFF9A493046FDF78AFC08B144F024
:108D1000400414F01103019300F05C829548FBF7C6
:108D200021FA0020FEF754F99348FBF71BFA934809
:108D3000FBF7F8F904F03003302B02D19048FBF731
:108D400011FA9048904FFBF70DFA9048FBF70AFA9A
:108D50004FF0FF338E4A8F492046FDF79DFB8E482A
:108D6000FBF700FA8D4A8E492046FDF789F88D48B9
:108D7000FBF7F8F98C4A8D492046FCF779FD8C48C1
:108D8000FBF7F0F98B4A8C492046FCF769FC8B48CD
:108D9000FBF7E8F98A4B1E688A4BD3F800908A4BA0
:108DA00000939B4669EA06034FF0000A02935BF8C2
:108DB000043B002B34D01A78D2B1029A03934FF0BF
:108DC000010808FA0AF812EA080F14BF012100216D
:108DD0003A462046FBF7ECF966EA090212EA080F68
:108DE000039B3A4614BF012100212046FBF7C6F938
:108DF0000AF1010ADBE7012468E7022466E7082498
:108E000064E7042462E77B88C3F30B021B04D7E901
:108E1000011048BF02EB42024AF0A2FB143763E79D
:108E20001F46DFF8C0A169EA06030293009B53F8CE
:108E300004BB0093BBF1000F25D09BF8002002B3C8
:108E40004FF0010808FA07F819EA080F0BD066EA94
:108E5000090212EA080F5B46524614BF01210021A5
:108E60002046FBF7A5F916EA080F0AD0029B13EA81
:108E7000080F52465B4614BF012100212046FBF734
:108E80007DF90137D2E75148DFF85CA1FBF76AF9B9
:108E90004F4AD2F800804F4A126888EA02025E46C2
:108EA000D343DFF848B10093009B0127B7403B4212
:108EB00014BF4FF001094FF0000918EA07070CBF73
:108EC00052465A463046039219F0EEFD039A02903C
:108ED000034649462046FBF76BF90136002F0CBFCD
:108EE0005A465246029B49462046FBF747F9182E40
:108EF000DAD13948DFF8F8A0DFF8F880DFF8F89029
:108F0000FBF730F9354BD3F8D8720026F3B20AEBF1
:108F10008302D2F854B3BBF1000F6FD00121994006
:108F200039405B460CD04A4600212046FBF726F923
:108F30005B464A4600212046FBF73AF90136E5E751
:108F4000424620460091FBF719F900995B464246DC
:108F5000F1E700BFC318070845180708BB17070843
:108F600089180708CA18070860850020A862070842
:108F7000CE180708DB180708E3180708FB180708CE
:108F80000719070842190708921907084C1907081A
:108F900074800020B09400205C190708F68A002035
:108FA000868B00206C190708A8870020048F0020FA
:108FB0007519070898860020648F00208919070812
:108FC000883E0020843E002070840608A919070806
:108FD000A4940020AC800020B019070860DD0020B8
:108FE000F86707089E190708B8180708AE18070899
:108FF000A0810608C5190708B91907089848FBF7A2
:10900000B1F8DFF82CC39748974ACDF820B0CDF8D7
:1090100010B0042601271CF8013F10F801EB03F102
:109020003001694401F820EC12F8011F01F1300809
:10903000E84408F810EC002F00F0EF80A3EB010EDD
:10904000DEF1000141EB0E01013E0F46E3D1874AFC
:109050008DF8146008AB2046FBF7AAF804AB39463C
:10906000824A2046FBF78AF88148FBF77BF8814A61
:1090700081492046FBF7A8FD8048FBF773F8804A3A
:1090800080492046FCF7A0FC7F48FBF76BF87F4A3D
:109090007F492046FCF7BCFD7E48FBF763F8784A21
:1090A00078492046FCF74CFE7B48FBF75BF87B4A8F
:1090B0007B492046FBF7BCFC7A48FBF753F87A4A19
:1090C0007A492046FBF7A2FE7948FBF74BF8794A2C
:1090D00079492046FCF7ACF87848FBF743F8784A22
:1090E00078492046FCF744F97748FBF73BF8774985
:1090F00020463FF0C5FB7648FBF734F84FF0FF33CE
:109100001A46744920463FF047FC7348FBF72AF89B
:109110004FF0FF33714A72492046FDF76DF87148F0
:10912000FBF720F8704A71492046FDF7EDF87048CA
:10913000FBF718F86F4A70492046FDF725F96F488C
:10914000FBF710F86E4A6F492046FDF707FC6E48A2
:10915000FBF708F821463046FBF702F9E7065ED533
:109160002146304695F8009095F802806F78FFF719
:10917000DBFC21460120FFF7D7FC21460220FFF748
:10918000D3FC2046FFF7F4F921463046FFF754FDA3
:1091900021460120FFF750FD21460220FFF74CFD3C
:1091A0004846FFF7A1FC4046FCF724FF3846FFF78E
:1091B00033FD5648FAF7D6FF554809F10101FBF790
:1091C00027F8544808F10101FBF722F85248791CAE
:1091D000FBF71EF80026A00703D528782146FFF7E5
:1091E000A3FC210704D5AB7813B92046FFF7C0F9DB
:1091F000620703D568782146FFF71EFD019B13B176
:109200004648FAF7AFFF2EB14548FAF7ABFF45489D
:10921000FAF788FF444C454D1CE0394614E728789E
:109220002146FFF781FCAB7813B92046FFF7A0F980
:1092300068782146FFF700FD0126CCE76388C3F379
:109240000B021B04D4E9010148BF02EB42024AF0C1
:1092500087F91434AC42F1D30DB0BDE8F08F00BFF4
:10926000D21907086886060838D90020E8190708C7
:10927000EF1907080C830020D0930020F519070888
:1092800008880020168C0020FA190708888A002018
:10929000968E0020041A0708131A07083982002046
:1092A000049400201F1A07084083002058930020D0
:1092B000361A07088885002078910020471A070889
:1092C0009885002078900020531A070860E000205D
:1092D000721A0708C0E90020831A070800CD002091
:1092E000F8EE0020961A070800D20020F8F30020BC
:1092F000B41A070860D2002058F40020D11A0708D9
:10930000D0D20020C8F40020C3180708E61A0708C6
:10931000091B07081C1B07082D1B0708401B070813
:10932000591B07086F1B0708A8620708F86707089A
:109330003CE0002000219BE4012199E42DE9F04F5D
:10934000CA4CDFF864A385B0C94B9C42C0F07C8155
:10935000C84CC94D2078FFF7C7FB6078FFF75CFC6D
:10936000A078C64CFCF746FEB4F81022B4F8EC31F5
:10937000C34804329A42A4BF5A1FA4F81022B4F87A
:109380001222043A9342A8BF053395F88127A8BF5B
:10939000A4F8123295F880379A4224BF002385F84A
:1093A0008037F5F729FAB74B1A68B74B934312D1B8
:1093B00000212520F0F75CFD064660B10021272042
:1093C000F0F756FD38B1026833689A4203D14FF482
:1093D0008030F5F711FA0027DFF8B0823E464FF0F3
:1093E000FF0948F2B83A58F827004308810801F00D
:1093F000333103F077330B44C10801F01131C31A44
:109400005B1A03EB131310F0010203F00F33B3FBED
:10941000F9F1C1EB012118BF0136A3EB010318BF1D
:10942000F6B2012B40F28881022B00F07C81974834
:109430000D2143F09BF8B5F8AC37B5F8AA27643B8B
:109440009342A8BF1346A5F8AA3700BF95F8223863
:1094500013B9082385F82238002010F037FCDFF814
:109460004CB2DBF80030002800F06F8123F08063FD
:10947000D4F89021CBF80030019211F05FFF8046C4
:1094800011F00EFF019A1FFA88F311780093A0EBF8
:1094900008034B43642193FBF1F37D4913FA88F3EE
:1094A000A5F8383800271678A7EB06090FFA89F9CE
:1094B000B9F1000FB24640F34B81C6F16406F6B233
:1094C00053780391CDE9013211F0EAFE019B039933
:1094D00009FB09FC03FB0CFCC3F1640316FB06F655
:1094E0000AEB8A0A9CFBF6F633440A2209FB03F3D3
:1094F00093FBF2F303EB4A0A0FFA8AFAA0EB080097
:109500004FF47A73174400FB0AFA9AFBF3FA009BB4
:10951000029ABFB29A446E2F21F802ABC3D121F058
:10952000DBFB18F071FE302200215A484BF03AF96B
:1095300010F0A0F994F8583123BB5749C4F878319A
:1095400091F83E0084F885316422C82612FB006041
:10955000C4F85C0191F83F0084F8863112FB006288
:10956000C4E95823C4E95A33C4E95C3391F8412073
:1095700084F85931C4F888314FF07A7384F8842123
:10958000C4F88C31DBF8003044499B060A6800F1CE
:10959000E280B5F87607B5F874370343B5F8780775
:1095A00003431BB2002B40F0D680B5F97A37B3F5F0
:1095B000805F40F0D080B5F97C37B3F5805F40F034
:1095C000CA80B5F97E37B3F5805F40F0C48022F4DD
:1095D00000720A6021F098FAB5F86C18DFED307A65
:1095E000304A07EE101AB8EEC77AB5F86E18C7EE13
:1095F000276A02F2545307EE101AB8EEC77AC3ED89
:10960000006AC7EE276AB5F8701807EE101AB8EEB0
:10961000C77AC3ED016AC7EE276AB5F8721807EE7C
:10962000101AB8EEC77AC3ED026AC7EE276AC3ED17
:10963000036A95F8743882F8643518F04BFB05B06E
:10964000BDE8F04F3AF070BDB4F90230DFF8608049
:10965000002BA7BF002637460326012700257919CE
:10966000C9B28E4226D214346EE600BFA862070843
:10967000F86707086085002058EE002060DD0020B4
:1096800020631406843E0020400001000C8300206B
:10969000746F012094F6002068CC0020306A01200D
:1096A00000401C46386A01200140000888690120FA
:1096B00000800008534603F1060BC3454ED21A88BA
:1096C000002A4BD003EB020CC44547D2052A45D9EA
:1096D0002088B3F802E0C0F30B00864521D1587909
:1096E00000F0030088421CD12946204693F80490DC
:1096F0000092F5F7BFF82188009AB9EB113F0ED11F
:1097000061886068C1F30B03063A9A42A8BF1A4603
:10971000090448BF03FB0500594649F021FF013504
:109720009DE76346C7E712B110EA0A0F04D141F082
:109730009DFD00283FF47BAE03370C2F7FF453AE22
:10974000013E022E7FF677AE71E643F080638FE62E
:1097500008BF0126B4E642F400723AE729462046E3
:10976000F5F788F8DBE710B5144C94F88132022B3A
:1097700018D120F055FDF4F74BFFFFF7DFFD20F087
:1097800059FD01201BF0B6FB0D4B0E491B6803F57C
:109790009C530022083384F88022C1F87C3884F876
:1097A000812210BD012BFCD120F03AFDF4F730FFEF
:1097B00020F040FD002384F88132F2E760DD0020D4
:1097C000042D002058EE002010B50446FFF78CF958
:1097D00038B120F025FDF4F71BFFFFF7AFFD20F0B7
:1097E00029FD601CC0B2BDE810401BF083BB38B53A
:1097F0000C4D04462046FAF7C7FE38B10A4B0B4819
:109800001978BDE838400131FAF702BD2046F4F777
:109810009DFE0138022804D8C0B2FFF7D5FF2C46C0
:10982000E8E738BD1D25070860850020091B0708EB
:1098300010B50446FFF7F0F938B120F0F1FCF4F769
:10984000E7FEFFF77BFD20F0F5FC601CC0B2BDE831
:1098500010401BF04FBB38B50C4D04462046FAF7BC
:1098600093FE38B10A4B0B485978BDE838400131B6
:10987000FAF7CEBC2046F4F769FE0138022804D876
:10988000C0B2FFF7D5FF2C46E8E738BD1D25070815
:10989000608500202D1B070810B50446FCF7AAFBC5
